:0C0000000C94C30C0C9400000C94000045
:10000C000C9400000C9400000C9400000C94000064
:10001C000C9425610C9400000C9400000C941015A9
:10002C000C9400000C9400000C9400000C94000044
:10003C000C9400000C94CB140C9400000C94DB5D1D
:10004C000C9400000C94175E0C9400000C940000AF
:10005C000C9400000C9400000C9400000C94000014
:10006C000C9400000C9400000C9400000C94805F25
:10007C000C9400000C94C3600C9400000C940000D1
:10008C0000000100020004000800100020004000E5
:10009C008000000100020004000800100020004055
:1000AC00008000010204081020408000B803C10B3E
:1000BC0080100000BC03C10B821F0000C603C10BE3
:1000CC0081030000CE03C10B01040300D803C20B53
:1000DC0001060500E203C40B01800000EE03CB0B0C
:1000EC00020F0000F603C50B020F0000FE03C70B46
:1000FC00020FD0120604C90B011000001004190CD9
:10010C00011000001A04CA0B000100002204CD0BE0
:10011C00010801002C04CE0B030801003A04CF0B9C
:10012C00030700004204E50B017F3F004C04E40B85
:10013C00010400005604D00B030400005E04E30B22
:10014C0001641E006A04D10B000100007604D20B7E
:10015C00000100008204E20B010200008E04D30BAC
:10016C00000100009C04D40B020F0000A804D60B65
:10017C00020FE703B204180C0163000010051A0CFF
:10018C00011000001A051B0C01020200BE04D80B62
:10019C0003080100C404D90B03080000CA04DA0BDD
:1001AC0003080000D004DB0B03080000D604DC0BB2
:1001BC0003080000DC04DD0B03080000E204DE0B86
:1001CC0003080000E804E60B040A2E00F004F00B10
:1001DC00040A2E00F804FA0B040A2E000005040C85
:1001EC00040A2E0008050E0C040A2E000000000064
:1001FC00FF000000220500022A0504043005080750
:10020C0036050C0536058C063C0580094405100B9B
:10021C004C05500C560540035E05140A6805180879
:10022C0070051C0100000002280060009800D0003E
:10023C0008014001210C58002D0B2D002B0B2B001D
:10024C004D0A4D00808182838400002188898A8B2D
:10025C008C8D8E8F310B312041424300320B32207A
:10026C0044454600330B3320474849004D0A4D00A6
:10027C0000000000340B34204A4B4C00350B352069
:10028C004D4E4F00360B3620505152002B0A2B008E
:10029C0000000000370B372053545500380B382022
:1002AC0056575800390B3920595A2F002D0A2D005A
:1002BC0000000000430C430000000000300B302015
:1002CC00202E2C002C0A2C00000000003D0A43526A
:1002DC000000000000004A01460032002100004BE3
:1002EC00004A01460032004D000096004A014600CB
:1002FC003200540000E1004A01460032003D00008B
:10030C00F0000000320050002D0000F000500032D0
:10031C00005000470000F000A000320050004B00DD
:10032C0000F000F000320050002B00005800B40028
:10033C00040038003800213803006A61000087008F
:10034C00C800640032003D4603006E65696E000013
:10035C000800C80064003200215603004B004A011B
:10036C00460032004D00000001000100E600630071
:10037C004D0000000000A0001B00007105D700A07C
:10038C00001A020071056900000018040073056969
:10039C00001E01190600730550726F64756B742092
:1003AC000000537061727465202000005F494400A6
:1003BC005F5273323332494400005F526F74617480
:1003CC0065005F54617374656E5800005F5461730F
:1003DC0074656E5900005F44656661756C744B659D
:1003EC0079002A436F64653000002A436F646531DD
:1003FC0000002A436F64653200002A4D61784D6F0E
:10040C0064756C005F4572774D6F64756C002A548F
:10041C006973636845005F4D795465726D4E720067
:10042C005F4D61737465725465726D7300005F4546
:10043C004D6F646500005F454372656457747200CC
:10044C005F5273304D6F646500005F5634756E6497
:10045C0035005F50756C736554696D6500005F41C4
:10046C00736B43726564697400005F53656E64441A
:10047C006562697400005F4372656469744D6F64F2
:10048C0065005F4372656469744D617374657200D5
:10049C002A5461626C655374617274002A546162EF
:1004AC006C65456E64002A4669727374426F6E50B7
:1004BC0000002A4A6F6231002A4A6F6232002A4ACF
:1004CC006F6233002A4A6F6234002A4A6F62350029
:1004DC002A4A6F6236002A4A6F6237005F45727291
:1004EC006F7231005F4572726F7232005F457272CB
:1004FC006F7233005F4572726F7234005F457272B7
:10050C006F7235005F4672656967616265005F4BAB
:10051C006F6D6D61000054617374657200004C69FD
:10052C00745A00004C656974540050756C7300006B
:10053C00546173742030000073657269656C6C00D3
:10054C0073657269656C20320000546173742032DB
:10055C00000054617374207061720000466F6C6708
:10056C00655400005377697463680000706F72748F
:10057C00696F6E696572656E00002E666F6C6765DB
:10058C000000506F7274696F6E656E2073696368DA
:10059C0065726E00436865662D4D656E75004B2067
:1005AC006C697374656E00004B206C6F65736368C7
:1005BC00656E00004B20647275636B656E00542091
:1005CC006C697374656E000054206C6F657363689E
:1005DC00656E00005420647275636B656E00537910
:1005EC007374656D0000506F7274696F6E004B729E
:1005FC006564697465004B7265642E436C7200000F
:10060C006D616E2E506F7274696F6E0054657374E9
:10061C000000506172616D657465720050726F6498
:10062C00756B746500004B656C6C6E65720056657D
:10063C006E74696C6500436F6C6F7273000030A050
:10064C000531AA0532B40533C00534CA0535D405C5
:10065C0036E00546EA0541F20543FA054402064A2E
:10066C000C060000000030EA05371806391E063863
:10067C002806423206453A066342060000004572DF
:10068C00726F72004F70742E0000496D70756C7330
:10069C00000054696D656F7574008A062F0C000597
:1006AC0000009006320C000300009606300C00058A
:1006BC0000009E06310C001400002E202C3041420C
:1006CC00433144454632474849334A4B4C344D4EEE
:1006DC004F35505152365354553756575838595A3E
:1006EC002F390500C11100000300D90B00000300D5
:1006FC00C1110300170E0300D90B00000500E00820
:10070C0000000A00C1110A00170E0A00D90B0A00DA
:10071C00C1110A00170E2800D90B000000000000C0
:10072C0000000000000000000000000000000000BD
:10073C0000000000070C182022204D994D4011405C
:10074C0048914720222018C007000000070C1F3FCB
:10075C00EE3F7277727FFF7F777F783FEE3F1FC04F
:10076C0007000000000000000C183DEE3F3FEE3F7C
:10077C001FC80F070002000000000000000000006E
:10078C00000207080F1FCE3F1FC80F070002000012
:10079C000000000000000007080F0F880F376F7F64
:1007AC007FFF7F3260070F80000000000000000216
:1007BC00000207080F1FCE3F3FEE3F1AC0070F8005
:1007CC000000000000000000000000000006000F08
:1007DC000F0006000000000000000000FFFFFFFFFC
:1007EC00FFFFFFFFFFF9FFF0F0FFF9FFFFFFFFFF37
:1007FC00FFFFFFFF0000000000000600091088103A
:10080C00108810090006000000000000FFFFFFFF29
:10081C00FFFFF9FFF6EF77EFEF77EFF6FFF9FFFF4A
:10082C00FFFFFFFF000000000E01006A1E3328616D
:10083C0061886133001E000000000000000000070A
:10084C008C0C186618186C0C078003030C0F030033
:10085C0003000000020003038C0302CC020280029E
:10086C0002000E1E001E0C00000000000C000E0BFF
:10087C0008090CC40E0B4C0938C478784C3103CCE5
:10088C00030180000000020202271FCC18306770A1
:10089C00306C181FC227020002000000000000107C
:1008AC0000181C001E1F081F1F001E1C0018100023
:1008BC00000000000000000088010388070F881F5B
:1008CC000F88070388010080000000000000020769
:1008DC00080F1FC0020200020200021FC80F07000F
:1008EC0002000000000819198819198819198819AB
:1008FC00198819198000198819000000000E1F367C
:10090C00CC6666CC6636CC1E06CC0606CC0606CC6F
:10091C000600000000081F30C03030081F30CC30FB
:10092C001F8C0000CC301F80000000000000000075
:10093C000000000000000000000000000E1F1FEE71
:10094C001F0000000200070F8C1F020002020002B1
:10095C000200021FC80F0700021FC00000000207A0
:10096C00080F1FC002020002020002020002020075
:10097C00020000000000020200020200020200025B
:10098C000200021FC80F0700020000000000000058
:10099C00000001080101CE3F01C801010000000068
:1009AC000000000000000000000004000C1C0E3FC2
:1009BC001C000C04000000000000000000000000FF
:1009CC000000000000000000400040400040400ECD
:1009DC007F000000000000000000088C1838EF7F3A
:1009EC0038EC180880000000000000000000000037
:1009FC00000000000207080F1FCE3F7FF000000030
:100A0C0000000000000000000000000F7F3FEC1F02
:100A1C000F80070200000000000000000000000032
:100A2C0000000000000000000000000000000000BA
:100A3C00000000000600060F000F0F000F0F00064D
:100A4C000600060000000600060000000000001969
:100A5C00881919881900000000000000000000002F
:100A6C00000000000006060666063FFC0C0CC819C8
:100A7C00198C7F3300333300000000000600061F82
:100A8C008C3F3600363F8C1F06CC063FC81F060035
:100A9C0006000000000000001338387E3801C8033F
:100AAC0007000E1C0E3870EE600000000000070DF1
:100ABC00881919801B0E001E3E063333C8313BC605
:100ACC001E0000000E000E0E000606000C000000BA
:100ADC000000000000000000000000000380060E73
:100AEC00000C1C001C1C001C1C001C0C000E06081E
:100AFC00030000001C00060700030388030388039F
:100B0C0003880303000706001C000000000000001F
:100B1C000C3636C81F0F0C3F0F081F36CC360000A2
:100B2C0000000000000000000000060006060C3F5C
:100B3C003FC0060600060000000000000000000098
:100B4C00000000000000000000000000000E0E007D
:100B5C000E06000C000000000000000000000C3F1E
:100B6C003FC000000000000000000000000000007A
:100B7C00000000000000000000000000000E0E004D
:100B8C000E00000000010000370000EC010380079C
:100B9C000E001C3800706000000000000F8E3F300B
:100BAC00676060FB616333666C33787036303FE8A6
:100BBC000F0000000300071F001F030003030003C6
:100BCC000300030300031FEE1F0000001FCE3F7045
:100BDC007360607E0001C80307000E1C00387FFFA5
:100BEC007F0000001FCE3F7073600037000FEC0FCA
:100BFC000063006037703FEC1F00000001CC03075E
:100C0C00CC0E1CCC3870CC607FFF7F00CC0000CCAD
:100C1C00000000007FFF7F600060600C7F3FE700FA
:100C2C000033006037703FEC1F00000003CC070E50
:100C3C00001C3800307FCE7F7073606037703FECE3
:100C4C001F0000007FFF7F00660000CC00018801C0
:100C5C000300030600060C000C0000000F8C1F386C
:100C6C00E630306E381FCE3F7073606037703FECEB
:100C7C001F0000001FCE3F7073606037703FFF1F76
:100C8C00006E0001C8031F001E00000000000000E1
:100C9C0000000E000E0E00000000000E000E0E00F4
:100CAC00000000000000000000000E000E0E00000E
:100CBC000000000E000E0E000606000C00CC010316
:100CCC0080070E001C3800381C000E07080301CCEE
:100CDC0000000000000000000000000E3F3FE0009C
:100CEC00000E3F3FE0000000000000003000381C08
:100CFC00000E07080301CC010380070E001C38000E
:100D0C00300000001F8C3F70E66060EC0103800730
:100D1C000600060600000600060000001FCE3F304D
:100D2C006B676FBB6D6DBB6D6DBE6F67C0703FCC7D
:100D3C000F0000000600060F000F0F081919881984
:100D4C0030CC3F3FC6606066600000007F087F616A
:100D5C00CC6060CC617F8C7F60E660606E607FC829
:100D6C007F0000000F8C1F38E63060006060006070
:100D7C00600060306E381FC80F0000007F087F6174
:100D8C00CC6060666060666060666060CC617F802D
:100D9C007F0000007FEE7F6000606000607F887FD6
:100DAC006000606000607FEE7F0000007FEE7F607F
:100DBC0000606000607F887F6000606000606000A1
:100DCC00600000000FCE1F38603060006063EE637F
:100DDC006066603066381FEE0F0000006066606071
:100DEC0066606066607FEE7F60666060666060660D
:100DFC00600000001F881F0600060600060600069D
:100E0C000600060600061F881F0000000066000092
:100E1C006600006600006600006660606C703FC88B
:100E2C001F000000606E6061C86367006E7C007C10
:100E3C006E0067638C6160E66000000060006060BB
:100E4C0000606000606000606000606000607FEEC9
:100E5C007F000000606E7070EE7979E66F6F6666E9
:100E6C006666606066606066600000006066707058
:100E7C0066786C666C66666663666361EE6060E6F7
:100E8C00600000000F081F39CC306066606066603F
:100E9C0060666030CC391F800F0000007F8C7F6053
:100EAC00E66060666060EC7F7F8060600060600080
:100EBC00600000000F081F39CC306066606066600F
:100ECC0060666333CC391FE60F0000007F8C7F60B7
:100EDC00E66060666060EC7F7F8067638C6160E6D3
:100EEC00600000001F8C3F70E6606000703F8C1F3C
:100EFC0000E600606E703FC81F0000003FCC3F064C
:100F0C000006060006060006060006060006060099
:100F1C000600000060666060666060666060666027
:100F2C00606660606C303FC81F00000060666060E7
:100F3C006C3030CC3019881919800F0F000F060057
:100F4C0006000000606660606660606660606666F1
:100F5C0066666F79EE7070E6600000006066603067
:100F6C00CC3019800F0600060F081930CC306066A3
:100F7C006000000060666030CC301988190F000FDB
:100F8C000600060600060600060000007FEE7F0045
:100F9C00CC000180030600060C00183000307FEEF8
:100FAC007F0000001F881F18001818001818001860
:100FBC001800181800181F881F000000000040605F
:100FCC00007038001C0E0007038C0100E700003095
:100FDC00000000001F881F018801018801018801A1
:100FEC000188010188011F881F0000000200070F03
:100FFC008C1D38E77060300000000000000000001D
:10100C0000000000000000000000000000000000D4
:10101C000000000000000000007FFF7F00000707B9
:10102C00000706000603000000000000000000009E
:10103C0000000000000000000000000C1F3FE60054
:10104C001FEE3F6066607FEE3F0000006000606056
:10105C00006060086F7FCE70606660606E607FC8F5
:10106C007F00000000000000000000081F3FC67059
:10107C006000606006703FC81F0000000066000042
:10108C00660000661F3FEE716066606066703FEE42
:10109C001F00000000000000000000081F3FC67089
:1010AC007FEC7F6000703FC81F00000007880F1C9A
:1010BC0000181800187F007F180018180018180066
:1010CC0018000000000000000000000E1F3FE6703A
:1010DC00606E703FE61F006E003FC83F60006060AE
:1010EC00006060006F7F8C7160CC6060CC6060CC05
:1010FC006000000000000006000600000E0E000656
:10110C000600060600061F881F00000000000001F4
:10111C008801000803038801018801018801018806
:10112C00191F800F300030300030300831338037D9
:10113C003E003E37083331CC300000000E000E0666
:10114C0000060600060600060600060600061F88B6
:10115C001F0000000000000000000008597FCE7F37
:10116C0066666666666666666600000000000000DD
:10117C00000000083F3FCE303066303066303066BD
:10118C003000000000000000000000081F3FCE707F
:10119C00606660606E703FC81F00000000000000B9
:1011AC00000000087F7FCE6060666070EC7F6F800F
:1011BC0060600060000000000000000E1F3FE67041
:1011CC0060666070EE3F1F66000066000000000065
:1011DC000000000C373FE638300030300030300073
:1011EC003000000000000000000000003F7F806025
:1011FC007F083F0188017F803F0000000000181825
:10120C00001818007F7F00181800181800181F8885
:10121C000F00000000000000000000066060666027
:10122C00606660606E703FE61F000000000000000A
:10123C000000000660606C3030C81919800F0F0078
:10124C0006000000000000000000000666666666EE
:10125C006666666F6C3F39C8100000000000000025
:10126C000000000C6071C83B1F000E1F083B71CCC6
:10127C0060000000000000000000000C3030C819B5
:10128C0019800F0F000606000C0C0018000000005F
:10129C000000000C7F7F800306000C1800307FCC10
:1012AC007F00000003CC070E000C0C000C1C003857
:1012BC001C000C0C000C0E0C0703C00006000606EC
:1012CC0000060600060000060600060600060600DC
:1012DC00060000003C003E070003030003038C01E2
:1012EC0003800303000307003E3C00000000001CC9
:1012FC006C3663800000000000000000000000005D
:10130C000000000000000000000006000F198C30E7
:10131C006066607FEE7F00000000000000001E0091
:10132C0060077E0700F01EF060F77EF7FBDE1F0003
:10133C00E007FF0700F81FF8E0FFFFFF00000F00B9
:10134C00E002EF0200780F78E07AEF7AF7BD1F0029
:10135C00E007FF0700F81FF8E0FFFFFF2300000283
:10136C000000100000050000FE0500182800FE0417
:10137C0000182400F90F00F80F0070001F71802373
:10138C0072802A73111574111C75151B76151A773A
:10139C00181C781521050100FF000000013F2B02ED
:1013AC000010072100000100072300100000FD3091
:1013BC0000073300113068FF0000E50080000100D9
:1013CC0001000102000403301004000008020209AD
:1013DC0000000A00000C00000D00000F00001000BF
:1013EC0000110700120000130000FD500010B01B8C
:1013FC00110700FD5000121E01FD500013001F29A3
:10140C001F00FD5000200000210000FE01002B0CED
:10141C0000FE00002B2000300000310603320002D9
:10142C003507013604043706063805013907073C31
:10143C0000063D070850000051EF00520000533FDA
:10144C0001FE01006000A7FE0000600027610100A2
:10145C006A0000800000810000820000830000848C
:10146C000000850000901000920007930700953F44
:10147C0003970000980000070100FD5000072100B1
:10148C00072300FD5000077301FD00000000000061
:10149C000000F8000000FF000000FF0000007F804B
:1014AC00001E0F80007FE7C0007FFFE0003FFFE0E1
:1014BC000007FFC00001FFC00001FF800001FF001A
:1014CC0003FFFE0007FFFC0007FFF00003FFF00026
:1014DC0003FFFE00001FFFC001FFFFF001FFFFF83C
:1014EC0001FFFFF8007FFFF80007FE00003FFF0040
:1014FC00007FFF80007FFF80007FC100001FE000A5
:10150C00001FF000001FF000000FE0000007C000FB
:10151C000007C0000007C0000007800000030000A7
:10152C0000030000000200000000000000000000AA
:10153C000000E0000000000000039000000000002C
:10154C00000E180000000000003808000000000029
:10155C0000C01800000000000380700000000000B4
:10156C000C01C00000018006300700000003C00F12
:10157C00401C00000006E01DC0700000000C30395B
:10158C00C1C0000000181871C7180000001C0CE145
:10159C00DC7C0000000E07C3F1C4000000070386CA
:1015AC00070600000003800E1C0200000001C01C96
:1015BC00300300000000E03818010080000070705B
:1015CC000FC183C0000038E003E08E6006001DC030
:1015DC000020FC200F000F800030703019800700B5
:1015EC000010003030C00000001800E06060000007
:1015FC000008038060300000000C0E003018000062
:10160C0000043800180C00000006E0000C06000076
:10161C0000038000060300000000000003018000AE
:10162C00000000000180C000C0C060C030C030C0ED
:10163C0030C030C030C030C030C030C030C030E0FE
:10164C0030703018300C30043FFC3FFC2564002B0C
:10165C00003E3E006B65696E204B726564697400D8
:10166C00436F6C6F72546F75636820567320312E04
:10167C0035300049443D00202047433D00202036B2
:10168C00346B004B653A00496E3A0043616C6962F9
:10169C00726174696F6E004F4B00546F74616C20F3
:1016AC00002D2D2D2D0054696E79200054696E7912
:1016BC0020626164006B65696E20454570726F6DC8
:1016CC00004D4F44554C2053544F500044617461AD
:1016DC002000696E69740000533F000066616C73F2
:1016EC00636865722054697363682000546973637E
:1016FC006820766F6E204B20004665686C65722002
:10170C000056656E74696C20616B7469760054695F
:10171C006D656F757400435349204E722000436F02
:10172C00646520006B65696E204B7265646974009A
:10173C0066616C73636865722054697363680054E6
:10174C006973636820766F6E204B005831393931DC
:10175C00303000504C5520203A00436F6465203ADD
:10176C00005469736368203A004D42005053004B9B
:10177C00656C6C6E657220004D31004F310053501A
:10178C000043500044590062757379004D5000209D
:10179C0067657370657272740025640041627265CE
:1017AC0063686E756E67004B656C6C6E65722000BD
:1017BC00546F74616C004D6F64756C2000202000B8
:1017CC00433F0073656300496D7000504C553A20DF
:1017DC00005370617274653A20005072313A2000E7
:1017EC005072323A200046756E6374203A200054D1
:1017FC0079703A20003A20563A2020302B203000C5
:10180C003A003A20544F3A20003A2050733A2000C4
:10181C0053703A004B204D6F6465204A6F62204A2A
:10182C006F62466C616773004B20004D6F646520DE
:10183C00004A6F62202000562020204572722050F2
:10184C00676C20496D7020544F0056200050617514
:10185C007365004B656C6C6E65723A004D49004DBA
:10186C0042004D43004D50004D4C00746573742084
:10187C002E2E004F4E0025303258002530345800A3
:10188C00253664002533642E2530326400253564FA
:10189C0000256400253264002533640044440000B4
:1018AC004B23004253004221004246005423005473
:1018BC004F004952004D5A004251004252004353CE
:1018CC0000565300564300494C00426600004B231F
:1018DC00005423004245004345004241004453005C
:1018EC0043420023502241534349492D492F4F2253
:1018FC002C22312E3030222C323030382D30312DFC
:10190C0030313B0023482245636F222C22312E308C
:10191C0030222C323030382D30312D30313B0023F9
:10192C00532245636F222C22312E3030222C323040
:10193C0030382D30312D30313B00504F0050463275
:10194C00333B5055002564002B302B303B00256475
:10195C000025303258002E3030004F4E00006D699B
:10196C006B726F746F756368000001002D4E414EF1
:10197C0000000100DE0E76190000F894EE27ECBB97
:10198C00F1E0F5BFE5BFE0936C00F8E1F1BDE1BD1E
:10199C008DE0A2E0BB27ED938A95E9F780E090E11A
:1019AC00A0E0B1E0ED930197E9F7EEE7F9E185915D
:1019BC009591009761F0A591B59105901590BF0197
:1019CC00F00105900D920197E1F7FB01F0CFEFEFDD
:1019DC00EDBFE0E1EEBFC0E0D3E00C947C160A99B9
:1019EC0002C0E1E00895E0E008951A931FEFE2E0F1
:1019FC000E94CF6BE3EFE1BB85E38A95F1F7E0EF53
:101A0C00E1BBE4E4E09374000E94D86B0E943D6655
:101A1C00E03091F4E981EE0FE0520E94DD6B41F46D
:101A2C00EDB7FEB7FA93EA931F930E94E26B1F91F6
:101A3C000E944E660E94E66BE0E0E09371000E940B
:101A4C00E66BE12F76C30E94EB6B10E01430F0F4E0
:101A5C0000E00430C8F4A12FECE30E94EF6B0E946D
:101A6C00F36B0E94F86BE15BFF4FFA93EA930E94D1
:101A7C00FD6B0E94FD6BE02FEE0FEE0FE10FEA9372
:101A8C000E94BA4B0F5FE5CF1F5FE0CFECE0E09315
:101A9C000F04E0E0E09310040E94026C0E94534992
:101AAC000E94086C0E940343E030D9F40E940F6C32
:101ABC000E940F6CE6E9F0E00E94146C0E940F6C1F
:101ACC000E940F6C0E94A4460E941E6C0E945A41F8
:101ADC000E94256C0E945A41EEE1F0E00E942C6CB1
:101AEC00E1CF0E94064345C4E881E03011F01C9A16
:101AFC0001C01C9832C00E940F6C0E940F6C0E9497
:101B0C00306CEFE3F0E00E94356C08951A93A091CD
:101B1C000403A43081F4E0910F04E093100410E06E
:101B2C00183048F4ABE01A9FF001E052FD4F0E94D0
:101B3C003B6C1F5FF5CF42C0A0910403A43039F475
:101B4C00E881E0931004E0E0E0930F0406C0E88124
:101B5C00E0930F04E0E0E0931004219608951A93AB
:101B6C00A0910403A43031F110E0143018F50E9458
:101B7C003F6C3196E491EA93DFDFE0E0E0931004F0
:101B8C000E94486C3896FA93EA93EBE0F1E00E94DD
:101B9C004B6C0E944B6CFA93EA930E943F6CE4915D
:101BAC00EA930E943F6C32960E94506C0E94C7438D
:101BBC001F5FDBCF0E94536C0E94586C19910895E3
:101BCC002A970E94687D30E010E000E047ED50E07D
:101BDC0028E0E091190CE03019F020E149E650E0E2
:101BEC003217F0F50E945C6CE13098F10E945C6C4D
:101BFC00E03870F0EEE00E94626CE8E5F6E1FA93F2
:101C0C00EA930E945C6CEF70EF5F0E946A6C07C0F5
:101C1C00ECE0EA9391DFE8E5EE83E0E0EF830E94ED
:101C2C00486C38960E94F36BE7E3F0E00E94E27A8E
:101C3C00E40FF51F0E944B6CFA93EA93EDE2F0E08F
:101C4C00FA93EA930E945C6CEA930E940F6C0E94D8
:101C5C00746C1F5F143011F410E00F5F3F5FC0CF46
:101C6C000E94536C0E9453490E946F7D61960895A7
:101C7C000E947A6CECE0EA935FDF0E94026CEBE06E
:101C8C00EA935ADF0E947E6C0E94836CEAEAF0E0D1
:101C9C000E94886CE0913A0CF0913B0CE491EA9331
:101CAC00E0913A0CF0913B0C31960E948F6C0E94A3
:101CBC00C74301E00E94926C0E94956C11F00F5F7B
:101CCC00F9CF0E94A36C031718F4E0E0E093C00571
:101CDC000E94A36C11E00E94AA6C0E94956C11F0FA
:101CEC00153008F021C00E947E6C0E94AD6CE0E4BF
:101CFC00F0E00E94E27A3496FA93EA93E2EEF0E096
:101D0C000E94886C0E94AA6C0E94B06CE491EA93C9
:101D1C000E94AA6C0E94B06C31960E948F6C0E943B
:101D2C00C7433F5F1F5FD7CF0E94586C0E94717DE5
:101D3C003AC427970E94687D22E354E0A0910403E3
:101D4C00A43011F426E453E010E0143010F00C949D
:101D5C00FA0E00E0051710F00C94F80EE12FEE0FC0
:101D6C00EE0FE00F3E2F0E94AA6C0E94BC6C3196C5
:101D7C00E4910E94626C0E94AA6C0E94BC6C329628
:101D8C00FA93EA930E94CE68ED85E03039F4AF8186
:101D9C00A13210F4E0E0EF83E0E0E887A02FBB274E
:101DAC00E22FE85FF0E00E94E27A3896FA93EA9329
:101DBC000E94AD6CEAE3F0E00E94E27AE55BFF4F33
:101DCC000E94C16C0E944B6CFA93EA930E94AA6C1D
:101DDC000E94BC6CE491EA930E940F6C0E94746C9C
:101DEC000F5FB8CF1F5FB1CF0E94586C0E946F7D00
:101DFC002E96089522970E94C66CA13059F40E9429
:101E0C00CB6CABE2B1E00E940D7B2E2F57E1E2ECE4
:101E1C00F0E008C00E94CB6C0E94CF6C2E2F53E0D8
:101E2C00E7EEF0E0EE83FF830E94D46CA0911908DA
:101E3C00A13081F4E9ECF0E00E94EB6C0E94F26CB2
:101E4C000E94F76CEBE2EA93EBE5F6E10E94506C32
:101E5C000E94C743E3E0F0E00E94EB6C0E94FD6C33
:101E6C000E94F76C0E94026D0E94066D3F5FE0912C
:101E7C00C10BAFEE0E94EC7AF0E0EE83FF8311E031
:101E8C00E091C20B1E17C0F500E0E091C10B0E17DC
:101E9C0088F50E940C6D59F10E94136DE0931004AB
:101EAC000E94926CAE81BF810E94E27A33960E94AE
:101EBC00C16C0E94AD6C0E94E27ADF010E941D6D24
:101ECC000E94206DEA85FB853497FA93EA930E9471
:101EDC00F76C0E94026D0E94066D3A930E94E320FB
:101EEC00EF3F29F0ADE05A9FF0010E94256D3F5F56
:101EFC000F5FCBCF1F5FC4CF0E94536C0E94586CF6
:101F0C00CAC022970E94687DE2E5F7E0EE83FF836A
:101F1C0040E0443190F4AE81BF8111960E942D6D4A
:101F2C001396EFEFEC93AE81BF81EC93EE81FF81C2
:101F3C003496EE83FF834F5FECCFE091C10BA0EFA3
:101F4C000E94EC7A2E2F0E94CB6CA0E4B1E00E9490
:101F5C000D7B5E2F0E94D46C21FE23C00E94326D3B
:101F6C000E94326DEFEAF0E0FA93EA930E94376D2B
:101F7C000E94026D0E94066D0E94086CE6EBF0E078
:101F8C00FA93EA930E94326D0E94F26C0E94376DB4
:101F9C00EFE7EA93EDE5F6E1FA93EA93E0E0F0E09F
:101FAC0011C00E94326D0E94326DE8EEF0E0FA939F
:101FBC00EA93E52F0E943D6DFA93EA930E94026D1D
:101FCC00EAE8FBE0FA93EA930E94C7433F5F11E013
:101FDC00E091C20B1E1710F00C944B1000E0E09136
:101FEC00C10B0E1710F00C9449100E940C6D11F4DB
:101FFC000C944610A0919A0BE0E8EA23E03821F00B
:10200C00A091E20BA23019F40E94136D0AC00E9439
:10201C00406DE03011F4E0E001C0E8E0E0930F0423
:10202C00E7E0E0931004A02FBB27E22FF0E00E9422
:10203C00E27A3396FA93EA930E941D6D0E94AD6C7E
:10204C000E94E27A3396FA93EA930E94F76C0E940C
:10205C00376D0E94026D0E94066D4E2FA0911E08D6
:10206C00E32F0E94456DEA0FFB1F43833A930E94B6
:10207C00E320EF3F29F0ADE04A9FF0010E94256D6F
:10208C003F5F0F5FACCF1F5FA3CF0E94536C0E94CA
:10209C00586C0E94E4350E946F7D28960895E1E00B
:1020AC00E0930D04E2E0E0930E04E0E0E093100412
:1020BC00ECE0E0930F04ECE5F3E00E943B6CEAE00B
:1020CC00E0930F04EAE4F3E00E943B6C0E94534956
:1020DC0008951A93A981A43029F4A0E021FCA1E071
:1020EC00A03009F426C0E9810E944C6D0490E9816E
:1020FC000E94526DE491A02DAE1BA2501A2F0E948B
:10210C00086CE4EBF0E0FA93EA93EB810E94526DD9
:10211C000E94957B3296FA93EA93EAE3F0E00E94F0
:10212C005A6DEFE7EA93EDE5F6E10E94506C0E94E0
:10213C00C7431881229608950E94EB6BE0E0EA9366
:10214C000E94CF180E94406D0E2FE4E3F2E00E9433
:10215C00957B33971E2F0E940F6C0E940F6C0E9470
:10216C00306C0E94616D0A930E94BA4B0E94FD6B09
:10217C000E94666D0E94BF46E2E0E0930E04E0917F
:10218C00980BEF70E09310040E946B6DEFE0E093FE
:10219C001004AA81A13051F40E94736D0E94836CCB
:1021AC000E94A446E0E6F6E10E94786D21FE0DC087
:1021BC00E4E0EA938EDFECE3F2E00E947C6DEEE368
:1021CC00F2E00E947C6D0E946E49A0DC80C0E88128
:1021DC000E94526D0E947C6DEA810E944C6D0E949F
:1021EC007C6D0E94FC46E881EA9373DFCAC11A93A6
:1021FC000A93EC81EA93EBDF1AEEEC810E944C6DB2
:10220C000490EC810E94526DE491A02DAE1BA25063
:10221C000A2FAC81A43029F4A0E021FCA1E0A0306D
:10222C0009F409C01EEAAA81BB811B96E0E0EC937D
:10223C00EC81EA934EDF0E94136DE0931004EC8165
:10224C000E94816DFF93EF930E94326DEE810E948C
:10225C00526D0E94957B31960E945A6D0E94926C31
:10226C00FA93EA93EC85E058EA930E940F6C0E9473
:10227C00876D0E94C743AF91BF91EC93EC810E9494
:10228C00526D0E947C6DEE810E944C6D0E947C6DA3
:10229C000E946E4919810881259608950E948C6DC3
:1022AC000E94CF6C8F010E940F6C0E940F6C0E94D9
:1022BC00306C0E948F6D0E94736D0E94A446EA815F
:1022CC00EA930E94CF180E946B6D0E94966D198143
:1022DC000881239608950E948C6D0E94CF6C8F010B
:1022EC000E940F6C0E940F6C0E94306C0E948F6DCC
:1022FC000E94736D0E94A446EC81FD810E94786D52
:10230C00AA81BB810E945E7D24F4A030E0E1BE076F
:10231C000CF006C0EA81FB81FA93EA930E946341B8
:10232C00AA81BB81A130E0E1BE0724F0A030E1E13D
:10233C00BE070CF00AC0A6EEBBE0EA81FB81E150BF
:10234C00F0410E94A06D0E94A86D0E94966D1981AB
:10235C000881269608950E948C6D0E94CF6C8F0187
:10236C000E940F6C1A930A930E946E49E0E0E0936E
:10237C003C0C099119910895E881EA930E94CF18B9
:10238C000E94B01FE03051F10E94AE6D0E940F6CA4
:10239C000E94B26D0E946B6D0E94B66DE881EA934B
:1023AC000E943021E8830E94BA6D3B9734F00E9462
:1023BC00BA6D0E94C56DE9E40BC0A3EEB6E00E94B5
:1023CC00C96D0E94CC6D0E94D16D0E94D66DE3E761
:1023DC00EA930E944246E2E0E0930E04D2C00E94CF
:1023EC003D68E0E0E0930F04A0910403A43019F4DD
:1023FC00E8E6F3E002C0E4E7F3E0FA93EA930E9424
:10240C00A74308950E94CB460E943D680E949268A3
:10241C00E1E0E0930D040E94AE6DE6E0F0E00E9476
:10242C00DA6DECE6F6E10E94786D0E940F6CE7E045
:10243C00F0E00E94DA6DEFE7F6E10E94786D0E9401
:10244C00DE6DEA930E947041E3E8F6E10E94786D3C
:10245C00E0910403EA930E947041E9E8F6E10E94DE
:10246C00786D08952A971A930A930E940F6C0E9414
:10247C000F6C0E94306CE4E6F0E00E94356C00E0DA
:10248C0010E01530B0F4053020F40E94E36DE0301C
:10249C0009F40DC00E940F6C0E94926C0E94DA6DC0
:1024AC000E94EA6D0E94E36D0E94EF6D0F5F1F5F4B
:1024BC00E8CF0E94F16D0E94A446EFE8F6E10E947D
:1024CC00786DE0913108EA930E9470410E947E6C15
:1024DC000E94736D0E94A446E3E9F6E10E94786DB8
:1024EC00E0912306EA93E5E0EA930E942641E0910D
:1024FC00190CE03079F10E947E6C0E94666D0E948E
:10250C00A446E09128060E94F46D0E94326D0E9450
:10251C00A446E0912806E295EF70E695E695AE2F7D
:10252C00E0912906EE0FEE0FEA0F0E94F46D0E9467
:10253C00836C0E94A446E0912906E295EF70AE2FC1
:10254C00E0912A06E295E07FEA0FEA93E6E0EA934F
:10255C000E9426410E947E6C0E94666D0E94A446D9
:10256C00E0913F0CEA930E947641198108817DC16C
:10257C00E881E064E7B9369A349BFECF349AE4B133
:10258C00F5B121960895E881F981AA81BB81AE1736
:10259C00BF071CF4EA1BFB0B06C0A881B981EA81BA
:1025AC00FB81EA1BFB0B2496089528970E946A7DF9
:1025BC00EFE0E0936100E1E0E09362000E94D86BF1
:1025CC00E5E0E09361000E94D86B0E94FA6DE09305
:1025DC006F05F0937005E0917B05F0917C05E0931D
:1025EC006D05F0936E05E1E0EA93C2DFE0937B05A5
:1025FC00F0937C05EFE0E0936100E8E0E09362008B
:10260C000E94D86BEAE0E09361000E94D86B0E94B4
:10261C00FF6DE0936B05F0936C05E0917905F091FB
:10262C007A05E0936905F0936A05E0E0EA93A0DF90
:10263C00E0937905F0937A050E94FF6DA0916B05EC
:10264C00B0916C05EA0FFB1FA0917905B0917A054A
:10265C000E94046E8F010E94FA6DA0916F05B091DB
:10266C007005EA0FFB1FA0917B05B0917C050E94C1
:10267C00046E9F01E0916B05F0916C050E940B6E4E
:10268C00FF93EF930E94FF6D0E940B6EAF91BF9171
:10269C00EA0FFB1FFF93EF93E0917905F0917A0518
:1026AC000E940B6EAF91BF91EA0FFB1FE093750573
:1026BC00F0937605E0916F05F09170050E94116E14
:1026CC00FF93EF930E94FA6D0E94116EAF91BF9130
:1026DC00EA0FFB1FFF93EF93E0917B05F0917C05D4
:1026EC000E94116EAF91BF91EA0FFB1FE09377052B
:1026FC00F0937805A0917505B0917605E4E1F0E0D2
:10270C000E94B47A0E2EA0917705B0917805E4E181
:10271C00F0E00E94B47AE02919F00E947745A3C03A
:10272C000093710510937205209373053093740513
:10273C00A0916405A63428F4E0916405EF5FE09362
:10274C0064050E94176E989724F40E941C6E98974B
:10275C000CF00EC0A0916405AA3019F4E1E0E093EE
:10276C006105A0916405A83219F4E2E0E0936105DB
:10277C000E94176E999724F00E941C6E99970CF486
:10278C0072C0E0916705EF5FE0936705A0E0B0E0F1
:10279C000E94B07B0E94176E0E94216E0E94286ED0
:1027AC000E942D6E0E94E77A7F936F93FF93EF93B5
:1027BC00A2E0B0E00E94B07B0F01A0E0B0E00E946C
:1027CC00366EAF91BF918F919F910E943D6E0E948A
:1027DC00286EA4E0B0E00E94B07B0E941C6E0E94A8
:1027EC00216E0E94426EAC81BD818E819F81EFE390
:1027FC00F1E060E070E00E94E77A7F936F93FF93C3
:10280C00EF93A6E0B0E00E94B07B0F01A4E0B0E033
:10281C000E94366EAF91BF918F919F910E943D6E39
:10282C000E94426EE0911204E03049F4E885F9858B
:10283C00E0935905F0935A05EC81FD810AC0EC81B7
:10284C00FD81E0935905F0935A050E942D6E0E946C
:10285C007C7AE0935B05F0935C050E941E6C0E94F1
:10286C00256C0E94FF440E94717D2C9608951A934A
:10287C000E94CB46E2E0E0930E04E2E3F0E00E941B
:10288C004B6C0E94476EE7E9F6E10E94786DE4E13B
:10289C00EA930E94CF40E0E9F1E00E944B6EE4E144
:1028AC00EA930E94CF40A0916705A13010F0A89543
:1028BC00FACF10E0143010F00C94BA14E2E0E0936C
:1028CC000D040E944F6EDF010E947C6DFD0132965B
:1028DC000E947C6D0E94BF460E944F6E3496E4911C
:1028EC00EA930E944246E1E0E0930D04A091670553
:1028FC00AF3110F4A895FACFEAE0EA930E94CF40EA
:10290C000E944F6EDF0135960E94957BBF01FD0141
:10291C000E94556EDB010E94C07B0E945C6E0E947F
:10292C00AD6CE8E2F0E00E94E27AE65AFF4F0E94BA
:10293C00476E0E944F6E0E94556E0E94C56DA0910D
:10294C006705AE3110F0A895FACF0E944F6EDF01EB
:10295C000E947C6DFD0132960E947C6DE8E1F0E0F6
:10296C000E94146C1F5FA6CF0E945C6EEAEFF0E031
:10297C000E94476EE3EAF6E10E94786DE0EDF7E025
:10298C000E944B6E0E94CB464CC10E94616E0A9312
:10299C00E4E6E2BF78940E94C14407DEE6B3AFEFF1
:1029AC00EA27E0933108A2E6BBE00E94706EE0914A
:1029BC00620BE77031F4A0910A04E0E4EA27E0939B
:1029CC000A04E091620BEF7131F4A0910A04E3E880
:1029DC00EA27E0930A040E940B660E94CF21E2B31F
:1029EC00EF700E2EA0911408B0911508EFE0F0E0F6
:1029FC00AE27BF27EA23FB230E94957AE029E2BB8E
:102A0C00E0911408E07111F41D9A01C01D98099110
:102A1C00199114C00E94616EE6E0E4BDE0B1E2954C
:102A2C00EF70AE2FE0916300E071EA2B1E2F0E9435
:102A3C00616D0E94A6210E94E5651991E991EFBF95
:102A4C00F991E991B991A9919991899179916991AA
:102A5C00F9901990099018950E940F650E94956540
:102A6C000E94FE500E94EC1E08951A93A8950E9495
:102A7C00D542E13011F00C949C15E091C605E15063
:102A8C001E2FA091C505A13021F40E94766EE03076
:102A9C0009F40CC0ADE01A9FF001E15FFC4FBF01DF
:102AAC00E081E260DB01EC930E947D6EA091C50594
:102ABC00A23011F0A43089F40E94766EE093DB050D
:102ACC000E94826E31F0FD01E15FFC4FE081E2700B
:102ADC0009F403C01A930E948B6EA091C505A33014
:102AEC0019F41A930E949027A091C505A53029F4DA
:102AFC00E091C605EA930E94BD27A091C505A830B8
:102B0C00A9F4E0E0EA93E091C605EF77EA930E941E
:102B1C00A2181E2F1F3F51F0E0E0EA930E94CF4015
:102B2C00E12FE058E093DB05E0932D06E0910A04D9
:102B3C00E078D1F0E0910A04EF77E0930A040E9468
:102B4C009749E0910A04E07131F0E0910A04E270D7
:102B5C00EA930E94A945A0913208A13328F0E2E043
:102B6C00EA930E94FB0C1E2FA0913C0CA13039F46F
:102B7C00E0913D0CF0913E0C0E948F6E09F401C067
:102B8C00EADB6ADF4EC01A930E94CB46E1E0F0E02C
:102B9C000E94506C0E94A44610E00E94996E0E9404
:102BAC000F6C0E94616D0E94A446E0912108E030F8
:102BBC0049F4E6EAF6E10E94786D0E949F6E0E944D
:102BCC00D66D1E5FA0912108A130F0F0E091210894
:102BDC00E150EA930E94FE18A091B30BAD3229F498
:102BEC000E94A86E0E945A7D79F0E3EBFBE00E94F4
:102BFC00A86DE6E0F0E0FA93EA930E94B56E0E94AD
:102C0C00A86E0E94D66D1E5FE0912108EF5FE093E5
:102C1C0021081C3020F4A0912108AB3008F001C031
:102C2C00BECF199108951A930E94CB46E981E030EA
:102C3C0019F4E0E0E0931E08A981A230A9F410E099
:102C4C00A0911E08A13010F01C3008F00DC0E091CE
:102C5C001E08E150E0931E080E94B96E19F40E9400
:102C6C00C76E09F01F5FECCF0E94996E10E00E94B6
:102C7C000F6C0E94616D0E94A446A0911E08A034A6
:102C8C0008F50E94B96E19F40E94C76ED1F0E0915C
:102C9C001E08EA930E94CF180E946B6D0E940F6C65
:102CAC000E94B56E0E94D26E0E94C56DE8E7EA9351
:102CBC000E9442460E94B66D0E94D76E0E94D66D4D
:102CCC001E5F05C0EDEAF6E10E94786D1E5FE09193
:102CDC001E08EF5FE0931E081C3020F4A0911E0824
:102CEC00A13408F001C0C3CF0C94311BE0E0E5BF68
:102CFC00E0936D00E0936C00EBBBEFEFEABBE0E020
:102D0C00E8BBE7BBE5BBEFEFE4BBE0EFE2BBE1BB4D
:102D1C00E0E2E3B9ECEBE2B9E0E0E0936200E093CF
:102D2C006100EFE0E0936500E0936400E0E0E0BF59
:102D3C00E7E0E3BFE4E6E2BFE0E0E1BFEFBDEEBDFC
:102D4C00EDBDECBDE7BDE6BDEBBDEABDE9BDE8BD43
:102D5C00E0937900E0937800E3E0E5BDE6E0E4BDC4
:102D6C00E0E0E3BDE0938B00EAE0E0938A00E0E072
:102D7C00E0938900E0938800E0938100E093800069
:102D8C00E2E1E0938700E4E3E0938600E0E0E09387
:102D9C008500E0938400E0938300E0938200E0934D
:102DAC006A00E0E3EABFE0E4E9BFE8BFE1E4E7BFC3
:102DBC00E0E0E0937D00EBB9E8EDEAB9E6E0E09302
:102DCC009500E0E0E0939000E7E6E9B9E0E0E093FD
:102DDC009B00E8EDE0939A00E6E0E0939D00E0E0D4
:102DEC00E0939800E3E3E0939900E0E8E8B9E0E0D1
:102DFC00E0BDE0E4E7B9E7E8E6B9E0B5EF7EE0BDB9
:102E0C00E0E2E0937000E0E0E0937200E4E4E09331
:102E1C007400EFE1E1BDEFE0E1BD0E94B85D0E94FE
:102E2C00564B0E949A4578940E94564B0E949A45A4
:102E3C00E1E0EA930E947A0D0E94DE6DE53128F004
:102E4C00A9E0B0E0E0E00E94C87BDCDA21E030E0F1
:102E5C00E0E0EA930E94FB0CE0933208EAE0F0E039
:102E6C000E944B6E3F5FA0913208A43511F03A30AE
:102E7C0008F001C0EDCF0E94736D0E947E6C0E9421
:102E8C00A446A0913208A43581F4E1E0EA930E94B3
:102E9C00FB0CE0933208E2EBF6E10E94786DE091D6
:102EAC003208EA930E94424607C0E0E0E093320801
:102EBC00E8EBF6E10E94786D84D0E03059F40E9482
:102ECC00736DE9E0F0E00E94DA6DE1ECF6E10E944E
:102EDC00786D20E0A9E0B0E0E1E00E94C87B2030F2
:102EEC0071F40E94736DEAE0F0E00E94DA6DEDEC93
:102EFC00F6E10E94786DA8950E94E06EFCCF0E94CE
:102F0C00CB360E94736DE9E0F0E00E94DA6DE8EDDB
:102F1C00F6E10E94786D0E94761BE03019F0EEED20
:102F2C00F6E102C0E3EAF6E1FA93EA930E9459460D
:102F3C000E941D66E1E0EA930E94CF4000E010E0A1
:102F4C000436E0E01E0724F40E949565E03009F099
:102F5C0007C0EAE0F0E00E944B6E0F5F1F4FF0CF0E
:102F6C000436E0E01E072CF0A0916705AF3108F0A5
:102F7C007EDC7BDD0E9426320E94A81DFACFFFCF9B
:102F8C000E94E36E17FD02C0103011F4E0E063C341
:102F9C00E12F61C30E94E36E17FD10E01A3008F4B4
:102FAC001F5F0E94F06E57C30E94E36E17FD02C0B4
:102FBC00103011F4E0E04FC311500E94F06EE1E0CC
:102FCC004AC31A930A9310E0E4E6F0E00E944B6EB9
:102FDC00A8950E943D66E03021F4E0EA0E94FB6E69
:102FEC0009F002C001E001C000E00E944E661F5FC4
:102FFC00003011F4153008F001C0E6CFE02F099134
:10300C00199108950E94006F43C40E94006F0E94A2
:10301C000D6F0895A881B9810E945E7D24F4A83EAD
:10302C00E3E0BE070CF005C00E94136F0E94B0666F
:10303C0013C3E0E011C3A881B9810E945E7D24F422
:10304C00A83EE3E0BE070CF005C0EA81E03011F4C5
:10305C00EFEFEA830E94136FED81EA930E94DC6626
:10306C0060C10E946A7D20E030E0283EE3E03E072C
:10307C007CF4A8953A932A93CDDF1E2F1F3F29F09D
:10308C00EFEFEA933A932A93D6DF2F5F3F4FEDCFC2
:10309C000E94717D4FC01A930A93E0E0F0E0E09338
:1030AC00400CF093410CAA81A03468F40E941C6F70
:1030BC00E55FFB4F8F010E94236F1A930A93E0E4A4
:1030CC00FCE00E94266FE091400CF091410C27C16E
:1030DC001A931FEF1F5F1A93DEDFA981BA81EA17DB
:1030EC00FB0711F0113408F001C0F4CFE12F188167
:1030FC0018C11A930A93A091C10BE091C20BEA9FDD
:10310C00F001A0911E08EA0F0E2F013408F00FE316
:10311C0010911E08101758F41A93BDDFAA81BB81B9
:10312C00EA17FB0711F4E12F03C01F5FF3CFEFEF9A
:10313C0019810881249608950E94687D10E010344E
:10314C0018F50E94AD6CE8E2F0E00E94E27AE050E3
:10315C00FC4FAF01E0EAEA93FA0170960E942A6FE5
:10316C00EC713E2FE0EAEA93FA013F960E942A6F37
:10317C000E2FEF81E31719F4EE81E01709F002C06E
:10318C00E12F03C01F5FDBCFEFEF0E946F7D28960E
:10319C0008951A930A93E091890BAA81EA17C1F05A
:1031AC00A03468F40E941C6FE050FC4F8F010E9409
:1031BC002E6F0E94266FEA81E093890B09C0EFEF16
:1031CC00E093890B0E94396F0E943E6FE093940B41
:1031DC00A6C01A930A930E941C6FE050FC4F8F01FB
:1031EC00AA81A03420F40E942E6F0E940D6F97C00C
:1031FC001A930A93E091B20BAA81EA17A1F00E94EC
:10320C00486F40F40E94546F0E94266FEA81E0934D
:10321C00B20B09C0EFEFE093B20B0E945F6F0E94FC
:10322C003E6FE093BD0B7BC01A930A930E94486FCC
:10323C0020F40E94546F0E940D6F71C01A930A9370
:10324C00E091330CAA81EA1761F10E94646F18F5C2
:10325C000E94236F1A930A93E4E3FCE00E94266F0A
:10326C00EA81E093330CE0E0E0932B06A091350C5F
:10327C00A13020F0A091350CA83008F00BC0A8EDBF
:10328C00BBE0E091350C0E946E6FAE0FBF1FEC914E
:10329C00E0932B0606C0EFEFE093330CE0E0E093F5
:1032AC00340C3DC01A930A930E94646F40F40E9440
:1032BC00236F1A930A93E4E3FCE00E940D6F2FC076
:1032CC001A930A93E0912E0CAA81EA17C1F00E947E
:1032DC00716F70F4E0EAEA930E94836C1A930A937C
:1032EC00EFE2FCE00E94266FEA81E0932E0C07C00F
:1032FC00EFEFE0932E0C0E947B6F0E94A3680FC02F
:10330C001A930A930E94716F50F4E0EAEA930E94B8
:10331C00836C1A930A93EFE2FCE00E940D6F198103
:10332C000881239608950E947B6F0E94A368E88110
:10333C00EF5FE093300CD2C124970E94687D0E940D
:10334C00826F0E94A368AA85A03478F5AB85A13062
:10335C0010F0A63008F007C0EB850E946E6F0E943B
:10336C00896F0E949C6FEB85E030F9F4E0E0EE830E
:10337C00EF83E887E98740E050E020E030E025303B
:10338C00E0E03E0784F4F9010E94896F0E949C6F73
:10339C000E94D26E4E0F5F1F0E94D76E0E94A16FCB
:1033AC002F5F3F4FECCF0E94AC6F3FC11A930A9333
:1033BC00AB81A13010F0A63008F01CC0EB810E944C
:1033CC006E6F0E94997A0E94957ADF01EA810E94C1
:1033DC00BD6FE8E0F0E00E94E27AE050FA4E8F0117
:1033EC00E0EAEA930E947E6C1A930A93ECE1FCE00B
:1033FC000E940D6F198108810C94EA1E0E946A7D4F
:10340C00EC810E94C16FE83109F459C00E94C66F6B
:10341C00309729F00E94C66F0E94CB6FEC830E94FC
:10342C00A41F0E2F10E0101710F00C94651A0E94B8
:10343C00CF6F82DFAEE1BCE00E94706EA091200CD9
:10344C00B091210C8091220C9091230C0E94D46F8E
:10345C000E94777AE093200CF093210C6093220C5D
:10346C007093230C0E94CF6FA1DFE0EAEA93EE8108
:10347C000E946E6FEE0FFF1FE050F04F0E942A6FFC
:10348C00E270D9F4ED81E093240C0E94C66F309762
:10349C0051F40E94DE6D0E94DB6FEF5EF84DDF0190
:1034AC000E94E16F02C00E94C66FE093250CF0935E
:1034BC00260C0E94E66F0E94EB6F1F5FB4CF0E9438
:1034CC00717D269608951A930A930E94F16FECE28F
:1034DC00F0E00E94F86F0E94FC6F0E94017010E0F7
:1034EC001034D8F41A9355DEE0912208EA931A931B
:1034FC0023DF0E940A70EA0FFB1F0F010E940A7063
:10350C000E941270DF01CB010E94D76E0E94777A65
:10351C00D0010E94907B1F5FE3CFA0911908A330CC
:10352C00B9F500E00031A0F50E94926C0E94177072
:10353C0069F510E01A3050F5E02FE05DEA93E4EE07
:10354C00F6E10E941C70E12FE05D0E942370E1F413
:10355C000E9428700E942F70EA0FFB1FFF93EF93BD
:10356C000E942F700E9412707F936F93FF93EF93C2
:10357C000E940162AF91BF918F919F910E94777AC7
:10358C00AF91BF910E94907B1F5FD4CF0F5FCACFCA
:10359C0010E01A3090F40E942F700E941270A091CB
:1035AC002908B0912A0880912B0890912C080E9430
:1035BC00777A0E9401701F5FECCF0C94321F249716
:1035CC000E94687DEA85EA9366DD9F01022E032A3C
:1035DC0039F13A932A937CDD1E2F40E050E0E0E075
:1035EC00EE83EF83E887E987AA851A17B1F4012FD8
:1035FC00003498F40A934FDD2E173F0761F4EB85E6
:10360C00EA930A9399DE0E94D26E4E0F5F1F0E94BE
:10361C00D76E0E94A16F0F5FEBCF0E94AC6F05C0FD
:10362C00EB85EA93EB85EA9387DE0E946F7D2C96FF
:10363C0008951A93A895A981A63068F40E94826F08
:10364C000E94A36810E0103430F4E981EA931A93D5
:10365C00ADDE1F5FF8CF1881229608951A9311E002
:10366C00163020F41A93E5DF1F5FFACF67C3E1E051
:10367C00E093340CE093350C31C0A8950E945F6F39
:10368C00EEEAF3E0FA93EA930E947E6C0E943670A5
:10369C00E093BB0B0E943F70E093BC0BE0E0E09327
:1036AC00BD0B1CC0A895E9E8FBE00E944670E9E25E
:1036BC00F0E00E94F86F0E94396FE4EAF3E0FA93AD
:1036CC00EA930E947E6C0E943670E093920B0E94EB
:1036DC003F70E093930BE0EBE093980B21960895E9
:1036EC000E94687D0E944B70E03228F0AAE0B0E0A6
:1036FC00E0E00E94C87B00E085DCA091BE0BB0919D
:10370C00BF0BA633E2E1BE0741F110E01A3030F4F2
:10371C001A93B3DF1A9388DD1F5FF8CF10E01034D3
:10372C0030F41A93BFDF1A9354DD1F5FF8CF10E00B
:10373C00103830F41A939BDF1A93B4DD1F5FF8CF67
:10374C008DDFA9E0B0E0E0E00E94C87BE6E3F2E1A7
:10375C00E093BE0BF093BF0B01E010E0183210F0B9
:10376C000C94091C0E9450709F010E945070AF0174
:10377C000E945A703496E491E03011F0E13069F413
:10378C00D901AC910E945A703596E491EA1720F455
:10379C000E945A700E94617034C0E23091F4DA01D8
:1037AC000E94867BE031A7E2FA0714F4FF2342F46F
:1037BC000E945A7036960E94957BDA01ED93FC9329
:1037CC0020C0E33049F4D901AC91AF3F21F40E9401
:1037DC005A700E94617015C0E43099F4D901AC9113
:1037EC00AF3F79F400E00E945A703596E4910E17C1
:1037FC0040F40E945A700E9461702F5F3F4F0F5F20
:10380C00F2CF1F5FABCF01DC10E0153060F41A93E0
:10381C0057DDA0912F0CA63020F01A9384DD1A935B
:10382C006FDD1F5FF2CFE02F0C94C920E881EF5FB2
:10383C00E883A881A43610F0E0E0E883E8810C94DA
:10384C0046210E94C96DA5E0B0E00E94E27A309654
:10385C000C944621A091370CBB27E091360CA6C0E6
:10386C00F9DF329774F00E946670E091360C0E947A
:10387C006D700E940D6FE091360CEA93D7DFE093E8
:10388C00360C08950E946670E091370C0E946D70A2
:10389C00FA93EA930E94FD660895E4E2FCE00E942C
:1038AC0075700E946670E091370C0E946D700E94DA
:1038BC000D6FE091370CEA93B9DFE093370C089564
:1038CC000E946A7DE0E0E093360CE093370C10E048
:1038DC0030E0343680F5A8950E9466703A93B1DFDB
:1038EC00FA93EA93E4E2FCE00E94266F00E0A091D8
:1038FC00240CA13010F0A03808F001C001E0E12F39
:10390C00E03041F4013029F43093370C3093360C0D
:10391C0011E00FC0E13031F4003019F43093360C63
:10392C0012E007C0E23029F4013019F43093370C5F
:10393C0013E03F5FCECF46C21A93A091CF0BA87075
:10394C00B9F010E0E981FA810E94AD6CAE17BF07A7
:10395C007CF4ED81E093240CEB81FC81E851FC4F6D
:10396C000E947C70E0E0F0E00E94EB6F1F5FEACFFA
:10397C0018810C94CB20E881EF5FE883A881A436F2
:10398C0010F0E0E0E883E8810C944621E881E150F6
:10399C00E883A881A43610F0E3E6E883E8810C9470
:1039AC004621A091390CBB27E091380CF0E0319600
:1039BC000E948170EC59FF4FDF01E4E6F0E00E94B9
:1039CC003F7B08950E94C96DA5E0B0E00E94E27AA9
:1039DC00E050FE4F0C944621E9E2FCE00E94757029
:1039EC00E881EA93BBD10C9446211A933ADBE1E0CF
:1039FC00E093860BA3C1A89510E0143680F41A93BB
:103A0C00A6D1A091290CAF3F31F40E948670AF3F34
:103A1C00EFEFBE0711F01A93DFDF1F5FEECF0E94AE
:103A2C008B70689420F88AC10E946A7D1091390CC1
:103A3C00AD81AA23CAF5E091380CE11719F0AD81DC
:103A4C00AA230AF030C01A9382D10E948670EE81AC
:103A5C00FF81EA17FB0729F4E885A091290CEA17E6
:103A6C0009F01EC00E949170EC81FD810E94817A48
:103A7C00EA17FB0744F40E9496700E949F70E0E0E6
:103A8C00EC83ED830BC00E949670EC83FD83E0E029
:103A9C00F0E00E949F70E0E0E093290C1A935ED155
:103AAC000E94A470C8CF46C0E091380CE11729F0F1
:103ABC00AC81BD810E945E7D0CF01BC01A9347D176
:103ACC000E948670EE81FF81EA17FB0729F4E885D6
:103ADC00A091290CEA1709F009C00E9496700E9467
:103AEC009F701A933BD1E0E0EC83ED830E94A470AD
:103AFC00DBCFAC81BD810E945E7D1CF452DF33971D
:103B0C000CF418C0E885E093290CEE81FF810E942B
:103B1C00A970EC81FD810E949F70E091380CEA93B2
:103B2C001DD1E091380CEA9326DFE093380CE0E0ED
:103B3C00EC83ED83689420F8EC81FD810E94717D0B
:103B4C00299608951A93A091420CA03059F4E09153
:103B5C00450CF091460CFA93EA93E8EBFBE00E94DB
:103B6C00AE7009F40BC0E1E0E093420CE091380C2C
:103B7C00E093440CE091380CE093430CA091420C80
:103B8C00A13011F00C94261EE091390CA091440C3C
:103B9C00EA1711F40C94171EE091440CEA93F6DE2C
:103BAC00E093440CEA93D3D0A091290CA13010F0EF
:103BBC00A03808F035C0E091430CEA93E7DEE093BF
:103BCC00430CA091440CEA1759F1EA93C7D0E09149
:103BDC00E20BE030E9F410E01530D0F4ABE01A9FC2
:103BEC00F001DF01E352FA4FE081E03049F0FD01D2
:103BFC00E452FA4FE081AE2FE091440CEA1709F041
:103C0C0005C00E94B470A091430CA0831F5FE4CF49
:103C1C00E9E2FCE00E947570E091440CEA939ED0BE
:103C2C000FC0E091430CE093390CE0E0E093420CC0
:103C3C00689420F80E941768E093450CF093460CAA
:103C4C007DC01A93A8951091390CE091380CE117AE
:103C5C00C1F00E94BA700E945E7D64F4EB81A09169
:103C6C00290CEA1739F40E948670E981FA81EA1767
:103C7C00FB0709F003C0E12F1881A6C00E94A470B5
:103C8C00E4CFEFEF1881A0C00E9491700E945E7D7E
:103C9C0084F4E0912B06E87031F4E0912F08A091A8
:103CAC00290CEA1731F40E94BE700E94CB6FE034ED
:103CBC0008F001C05CC10C94A421A895E091380CCB
:103CCC00A881EA1761F0E8810E94C37019F0E881BD
:103CDC000C944621E881EA934EDEE883EFCFEFEFB8
:103CEC000C9446211A93A8951091390CE091380C3C
:103CFC00E117E1F00E94BA700E945E7D8CF4E091B5
:103D0C002B06E87031F4E0912F08A091290CEA17EA
:103D1C0039F40E948670E981FA81EA17FB0709F0F1
:103D2C0002C00C948B210E94A470E0CFEFEF0C9496
:103D3C008C211A931091390C1A93BFDF19910895A5
:103D4C00E881EA9318DEE883EA93B7DF99C20E9410
:103D5C0066700E94CA700E94266F92C20E946670A2
:103D6C000E94CA700E940D6F8BC20E946A7D0E94D5
:103D7C008B7010E030E0343628F5A8953A93E7DFE5
:103D8C0000E0A091290CA03808F401E0E12FE0300C
:103D9C0041F4013029F43093390C3093380C11E094
:103DAC000FC0E13031F4003019F43093380C12E0CC
:103DBC0007C0E23029F4013019F43093390C13E0C8
:103DCC003F5FD9CF0E94717D249608951A930A9370
:103DDC00A0911908A43009F43FC010912F0800914C
:103DEC00510CE0913108E03059F0E0932F086894C1
:103DFC0024F80E94D370E0E0E0933008E0E520C0A6
:103E0C00E0913008E03021F0E0932F08E2E518C093
:103E1C00E0E0E0932F08E093510CE091C40BE0300C
:103E2C0031F0E091C40BE150EA930E942419A09167
:103E3C00340CA17039F0E091C40BE0932F08E4E44A
:103E4C00E093510CA0912F081A1721F4A091510C5A
:103E5C000A1711F0689423F80991199108950E949A
:103E6C00D970EBE0EC93EC81D8011696EC93EB81D6
:103E7C00D8011796EC93D8011896E0E0F0E0ED939A
:103E8C00FC93D80112960E94E670D80114960E94F9
:103E9C00E6700E94EB7001C10E94D970ECE0EC93CB
:103EAC000E94EB7034C21A9318E0113108F5E091BE
:103EBC001408F0911508A981BA81EA27FB27BF01E4
:103ECC000E94F770E623F723309781F00E94F77079
:103EDC00A981BA81EA23FB23309731F01A93E0E0F1
:103EEC00EA931A93BCDF02C01A93D6DF1F5FDDCFB3
:103EFC000DC2A0911A0CA93030F0E091590CA09190
:103F0C00580CEA1709F414C0E091590CE03021F474
:103F1C00E3E6EA93C1DF08C0E0911A0CEA93E0E013
:103F2C00EA93E3E6EA939BDFE091590CE093580C9B
:103F3C000895A0919A0BECE1EA230895A0919A0BB5
:103F4C00A07411F0E2E00895A0919A0BA07809F00A
:103F5C00F5C10DC0A091890BAF3F09F4EFC1E9DFAA
:103F6C00E43009F4EBC1E5DFE03109F4E7C1E1E04D
:103F7C0008950895A881AF3F11F4E0E081C1D9DF25
:103F8C00E43011F4E1E07CC1E0E07AC1A881A23018
:103F9C0019F4CFDFE83011F0E1E072C1E0E070C15C
:103FAC00A881B981AC91A130A8F0A881B981AC915C
:103FBC00A43180F4A881B981EC910E940271EB5F6D
:103FCC00FC4FE081EF770E2EA881B9811296EC910F
:103FDC00E01509F002C0E1E011C1E0E00FC1A881D9
:103FEC00A13118F0E881E051E883E8810E94077163
:103FFC000E941171A091D00BA13018F0A881A430AF
:10400C0009F006C0E6E9F0E00E94957B0E94117170
:10401C0037C1A881A13010F0A63008F006C0E881A5
:10402C000E941C71E15CF94F2AC1E0E029C1A88112
:10403C00A13010F0A63008F006C0E8810E941C7177
:10404C00EC5BF94F1CC1E0E01BC10E946A7DEC8166
:10405C00EA93EDDFEF731E2F1030E1F0EC81EA9361
:10406C00E6DFE0743E2FE12FE150A1E00E948D7A53
:10407C00A0912306EA230E2F303011F4003009F002
:10408C0002C0E1E008C0303011F0003009F402C089
:10409C00E1E001C0E0E00E94717D259608950E9448
:1040AC00687D00E00530A0F50A930E9466190E9415
:1040BC002171A7E10A9FF001EE5CF94F0E94467056
:1040CC00E4E1F0E00E94F86FE091300CDA015096D8
:1040DC00EC93A0912F0CEFE3EA23AE2FE091320C7E
:1040EC00E295E07FEE0FEE0FEA0FDA015596EC93B6
:1040FC00E091300CE1503E2F3F3F41F0E091310C0C
:10410C000E94DB6FDA015196ED93FC930F5FCACFDF
:10411C0010E01034C0F51A930E94CF181A932ADFBE
:10412C00E13079F5E0919D0BEA9373DFE1500E2FAE
:10413C000F3F39F10E942171E12FDA011396EC93B4
:10414C00E0919D0BDA011496EC93E091A30BF091A6
:10415C00A40BDA011696ED93FC930E94D46FA4E69F
:10416C00B0E080E090E00E94E77ADF01CB01E091C3
:10417C00A30BF091A40B0E943D6EDA011A96ED93FD
:10418C00FC931F5FC6CF0E946F7D26960895A09169
:10419C001908A23031F0A83021F0A73011F0A53069
:1041AC0009F40AC00E94F16FEFEFF0E00E94F86F83
:1041BC0076DFE0E0E093A20608951A93E981E058D7
:1041CC00E98310E01530C0F4A3E21A9FF001EB551F
:1041DC00F94FE081AE2FE981EA1749F4F001EC5573
:1041EC00F94FE081AE2FE0912F08EA1709F002C0D9
:1041FC00E12F03C01F5FE6CFEFEF188122960895E1
:10420C000E946A7DED81EA93D8DF1E2F1F3FF1F0EB
:10421C00A3E21A9FF001ED55F94F9F01D9011296B7
:10422C00EC91EF77EC93EC81D901EC930E94027145
:10423C00EF5EFC4FBF01E081EF77DB01EC93EC818B
:10424C000E940271E15FFC4FA1E0A083E12F0E946C
:10425C00717DE4C40E94C96D0E94287161F4E091E3
:10426C004B0CEF5FE0934B0C0E94C96DED55F94F71
:10427C00A0914B0CA0830E94C96DED55F94FE081C4
:10428C00219608951A931FEFE091D40BF091D50B62
:10429C00A981BA81AE17BF073CF0E091D60BF09123
:1042AC00D70BEA17FB070CF412C00E942D710E9469
:1042BC0010181E2F103031F01F3F21F0E0912F0805
:1042CC00E11729F4E1E0E093590CE0E01FC0E0E0D5
:1042DC00E093590C1AC01A930E942D71D3DF1E2F34
:1042EC00103099F01F3F39F4E8EEF6E1FA93EA93B7
:1042FC00EB81FC8106C0E8EFF6E1FA93EA930E94A9
:10430C003271FA93EA930E947111E12F188123966E
:10431C000895E0916505E03009F00895E0912C06D0
:10432C00E03009F008950AC0E0916605E03009F02C
:10433C000895E0912D06E03009F00895E0E008952D
:10434C000E946A7DE0912606F0912706AC81BD8122
:10435C00EA27FB279F0110E0153090F4F901E1707A
:10436C0049F0A7E11A9FF001EF5CF94FDF01EC91E6
:10437C00EF5FEC93D9010E9435719F011F5FECCF69
:10438C00EC81FD81E0932606F09327060E94717D57
:10439C0045C428970E94687D3091260610E01530A0
:1043AC00B8F5A7E11A9FF001EB5BF94F0081E12F03
:1043BC00A1E00E948D7A2E2FE22FE32391F000389A
:1043CC0010F0003C08F001C00F5F003C31F4E22F0C
:1043DC00A0912306EA2BE0932306003808F400E8AA
:1043EC000FC0003408F40F5F003439F4EFEFE2270C
:1043FC00A0912306EA23E0932306003808F000E09E
:10440C00A7E11A9FF001EB5BF94F00831F5FC7CF49
:10441C00E0E0E0932C06E0E0F0E0E0931608F09387
:10442C001708E091590CE03021F0E0911A0CEA9356
:10443C00D6DDE0911D08EF5FE0931D08E091E30BE2
:10444C00A0911D08EA1751F4E091E30BF0E0A0E015
:10445C00B1E00E94A97BEA1BE0931D08A09119080A
:10446C00A13019F0A93009F096C0A091620BB0915F
:10447C00630BE4E1F0E00E943F7B309719F4E1E03C
:10448C00E0931F0846DFE03019F04EDFE07809F4C6
:10449C0062C04ADFEF775E2F5A930E94CF180E94BA
:1044AC001D6DED55F94F5081503011F40C94B12223
:1044BC0051DDE13031F4E0911A08EA9367DDE03028
:1044CC0009F449C00E943A710E94BD6FEC91EC71E5
:1044DC00EC3021F4E0911D08E07851F40E943F711A
:1044EC00EC91EA937CDD0E944471EC91EA9377DDC8
:1044FC000E943F71AC91A63070F5A3EEB6E00E941D
:10450C001D6D0E94CC6D0E94706E0E943F71EC91EB
:10451C00EA937FDD1E2F1130F0F00E9449710E944A
:10452C004C71CF010E9449710E94CC6D6D917C91B0
:10453C00E12F0E941C71EF5CF94F0E945171E60F44
:10454C00F71FDC01ED93FC93E12F0E941C71EF5CD3
:10455C00F94FA0E0A08310E01530E8F40E945471EC
:10456C0013965C915F3FA9F05A9374DE5E2F0E9404
:10457C005E710E9449710E944C71BF010E94497189
:10458C000E94CC6D0E946471AE81BF811296E0E0F6
:10459C00EC931F5FE1CFA0911908A23039F0A8303D
:1045AC0029F0A53019F0A73009F0EAC1E0E0E0935A
:1045BC00200800E0053010F00C94C624A3E20A9FFA
:1045CC00F001ED55F94FEA87FB87AA85BB85AC91C5
:1045DC00A03019F0A281A07809F0D0C1E091200898
:1045EC00EF5FE0932008AA85BB8513960E94867B1B
:1045FC00309771F0AA85BB8513960E9471710E9449
:10460C00777129F4AA85BB8513960E94E670B6C112
:10461C008BDEE03021F00E94777109F4AFC120E00D
:10462C0030E0333010F00C9471240E948171DF0162
:10463C000E94AA6C0E94A06DE887F987A181A270E4
:10464C0021F4A481B581109709F410C1E885F9858E
:10465C00A181A47011F40C949323A181A87021F46E
:10466C000E94A633E03009F457C00E948771EBE03A
:10467C00EC93A885B9850E949471A885B985139689
:10468C00EC91AC85BD851796EC93EC85FD85389641
:10469C000F01E885F985A181E1E0EA230E949B7175
:1046AC00ED93FC93A885B98514960E94867BAC8506
:1046BC00BD851296ED93FC930E949E71AC85BD85D1
:1046CC001496ED93FC93A02FEAE0EA9FF001E30F20
:1046DC00EF5F0E94A471E885F985A085B185E2E0C1
:1046EC00F0E00E94E27AA885B9851896ED93FC93C8
:1046FC000E949E71309739F4A885B9851896E8EE1A
:10470C00F3E0ED93FC93E885F985A181E8E0EA2BD1
:10471C00A885B9851196EC936EC0E885F985A181C1
:10472C00A17031F4A885B98514960E94717143C0AB
:10473C000E94AD716EDCE1501E2F0E9454711296D6
:10474C00EC91E03001F5AE81BF8153960E94706E02
:10475C00EE81FF81A189B289109751F003881488EA
:10476C00AE81BF8151960E94867BE015F1050CF05D
:10477C0009C00E94FD6C14DCE03011F00E94B27193
:10478C000E94BA710EC0E885F98534960E94C271F8
:10479C000E949B710E9481700E94CA7153960E9464
:1047AC00E670E885F985A581AA232AF4A885B98540
:1047BC0014960E94E670A885B985EC91EC71EC30EA
:1047CC0021F4E0911D08E078B1F4E885F985A48125
:1047DC00B5815E971CF4A181A07209F404C0E88530
:1047EC00F985A28106C00E94AD71F9DBE885F985D7
:1047FC00A381AA93F4DB0E949E71309791F0A88557
:10480C00B98518960E9471710E949E71309749F477
:10481C000E94FD6CC5DBE03011F00E94B2710E9469
:10482C00BA710E94AD7111DCE03001F10E94FD6C97
:10483C00B7DBE03049F00E94B271AA85BB85EC91E0
:10484C000E9402710E94256DAA85BB851296EC917F
:10485C00E058AA85BB851296EC93E3E0E09324061E
:10486C000E94AD71E4DBEF73E0932506A885B98552
:10487C0014960E94867B309761F52F5F323048F595
:10488C00A885B98516960E94867B309789F0E885B5
:10489C00F985A681B7810E94D171AA85BB85139633
:1048AC00ED93FC93A885B98516960E94E67011C00D
:1048BC000E948171DF01E32FEF5FF0E00E94A06D99
:1048CC00E887F987A181EDEFEA23A885B9851196D0
:1048DC00EC933F5FA6CE233011F00C94C4240E94BD
:1048EC00A633E03069F00E948771E8E0EC93AA856A
:1048FC00BB850E949471AA85BB85EC910E94A47122
:10490C000E94FD6C4DDBE03011F00E94B271AA8563
:10491C00BB85E0E0EC93EA85FB85A581ECE1EA231D
:10492C00E83061F50E94DE6DAE2FEA85FB85E38DE4
:10493C00EA1741F4EA85FB85E48DE150EA930E9485
:10494C00D0171CC00E94A633E030C1F00E948771C2
:10495C00E3E0EC93AC85BD85EFEFEC931896EA851C
:10496C00FB85E38D0E94D671AC85BD851296EA85D8
:10497C00FB85E48D0E94D6710E94DA710F5F1ACE0E
:10498C000E94E07149F4A0911908A23021F0A830DE
:10499C0011F0A53009F401C050C010E0153010F032
:1049AC000C9423250E94547113965C915F3F11F473
:1049BC000C9421250E945E71AE81BF81BD010E94C5
:1049CC006471EE81FF8138960E94C2710E94E6717B
:1049DC000E94CA710E94867BDF010E945E7DB4F446
:1049EC00EE81FF81A681B7810E945E7D7CF4AE8151
:1049FC00BF810D901C90AE81BF8116960E94867B64
:104A0C00D001AE1BBF0B0E945E7D0CF014C0AE81BA
:104A1C00BF81BD010D901C90EE81FF81A681B781F5
:104A2C00F001EA1BFB0BDB01ED93FC935A93E5E0E1
:104A3C00EA930E94F3421F5FB1CFE0911C08E03073
:104A4C0041F4E0911608F0911708E0931408F093E4
:104A5C0015080E946F7D2E9608950E946A7DA09184
:104A6C00C10BE091C20BE150EA9FF001EF5F1E2FEA
:104A7C002FE330E000911E08A091180CA13080F0BB
:104A8C00E091180CE150A0911E08AE1728F0E091AF
:104A9C00180CE1503E2F04C0E091180CE2502E2F60
:104AAC00EC81E03049F1EF3F51F4A0911E08A11BBD
:104ABC00A31720F0E0911E08E11B0E2F1DC0EE3F46
:104ACC0059F4E12FA0911E08AE0FA21720F4A0916B
:104ADC001E08EA0F0E2F10C0EC3F49F4A091180CE1
:104AEC00A13020F0E091180CE1500E2F05C0AC81E4
:104AFC00A1501A9FF0010E2FE0911E08E01751F003
:104B0C000A930E94CF18A0918A0BAD3209F4032F9F
:104B1C0000931E080E94CB46A0911908A83019F4E6
:104B2C000E94870F02C00E94000F0E94717D259683
:104B3C0008950E94687DFDD9E03111F40C94112682
:104B4C0020E030E040E050E010E0133060F50E94CF
:104B5C00EA710E94CC6D0E94867B309711F10E9405
:104B6C00ED710E9407712E2B3F2B0E94ED71EA9381
:104B7C006CDAE03029F0E3E0E0932406E0E04CC08E
:104B8C000E94F4710E9407712E2B3F2B0E94F4712E
:104B9C00EA935BDAE03029F0E3E0E0932406E0E00E
:104BAC003BC01F5FD2CF00E0053058F5A3E20A9F4F
:104BBC00F0010E94287119F110E0133000F50E94E9
:104BCC008171DF010E9432710E94FB71AE0FBF1F19
:104BDC001296EC910E9407714E2B5F2B0E948171F3
:104BEC00DF010E9432710E94FB71AE0FBF1F139642
:104BFC00EC910E9407714E2B5F2B1F5FDECF0F5F76
:104C0C00D3CFF901E423F523309729F0E1E0E093C9
:104C1C002406E0E001C0E1E00E946F7D2696089535
:104C2C001A93E0914F0CE03011F40C945D26E09156
:104C3C00E40BE13059F4A0914F0CA13311F4EFE0E7
:104C4C0001C0E0E0EA930E94505E31C0E23059F4BA
:104C5C00A0914F0CA13311F4E6E001C0E5E1EA9319
:104C6C000E94505E24C0E330B1F410E0173040F4E1
:104C7C000E943271E05CF64F0E9402721F5FF6CF09
:104C8C00A0914F0CA13311F4E1E301C0E0E3EA93EE
:104C9C000E94505E0CC00E940672E9E4EA930E94E6
:104CAC00A562E0914F0C0E940D720E94127288C492
:104CBC0022970E94687D30E0A0911908A23029F05B
:104CCC00A83019F0A53009F021C1A985A03410F045
:104CDC000C948B27E0912F08E03009F417C1E9857B
:104CEC000E94C16FE03131F4E1E3E0934F0C98DFA7
:104CFC00E1E00CC12FD9E03009F408C110E0153007
:104D0C00A0F4A3E21A9FF001DF010E94287141F088
:104D1C00FD01EB55F94FE081AE2FE985EA1709F05B
:104D2C0002C0E0E0F3C01F5FEACF03DFE03011F414
:104D3C000C948B2710E0A3E21A9FF001ED55F94F6C
:104D4C00EE83FF83AE81BF81EC91E03011F00C94C7
:104D5C00842713960E94E67000E0033010F00C9448
:104D6C005327A3E21A9FF001E855F94FDF010E9487
:104D7C00926C0E94A06DAF01DA0116960E94E6704B
:104D8C000E941772DA011296EC930E941E72DA01DD
:104D9C001396EC93A0919A0BEEEFEA23DA01EC93C5
:104DAC000E942572DA011196EC93C3D8E43139F0E4
:104DBC00FA01A181E2E0EA2BDA011196EC930A9355
:104DCC00E5D8E03011F40C943527FA01A281AA93AE
:104DDC0020D9E1502E2F2F3F81F0A7E12A9FF0011F
:104DEC00EF5CF94FA0E0A083A7E12A9FF001EE5BF6
:104DFC00F94FA0E0B0E0A083B1830E942D720E9415
:104E0C00CC6D0E94867BDA011496ED93FC930130F5
:104E1C0040F00E942D720E94CC6D0E94867B3097D0
:104E2C0009F00EC0AE81BF811596E02F0E946E6F07
:104E3C000E94FB71AE0FBF1F1196EC91E062EC93D8
:104E4C00AE81BF815A96EC91E062EC93023030F463
:104E5C000E943072DA0116960E94D67104C0DA01F3
:104E6C0014960E94E67065D8EC3019F4E0E0E093FB
:104E7C001D080E9437720E94DB6FDA011896ED93C1
:104E8C00FC93FA01A281A63030F0A181E4E0EA2B78
:104E9C00DA011196EC930F5F60CFA0911908A23044
:104EAC0011F0A53019F4A885AF3F08F007C0E091C8
:104EBC002F08EA93EA85EA930E94041AE885AE81EA
:104ECC00BF81EC93E0912F08AE81BF811196EC93DA
:104EDC00E985AE81BF811296EC93A885A43138F494
:104EEC00E8850E940271E15FFC4FA1E0A083AE81D6
:104EFC00BF811696EC91ED7FEC9331E01F5F303063
:104F0C0011F4153008F001C016CFE32F0E946F7D0D
:104F1C002A9608951A930A93A0911908A23011F0B9
:104F2C00A53021F40E943E720E948B6EA09119084C
:104F3C00A830C9F40E943E72E1E0EA930E942D472A
:104F4C00E091E20BE03069F4EA810E944972E08161
:104F5C00EF771E2FABE01A9FF001EA51FA4FA0E059
:104F6C00A083689420F8198108812396089564978A
:104F7C000E94C66CA23039F4E0912F08EA93EB8DB5
:104F8C00EA930E94041AA0911908A83011F00C940D
:104F9C0033280FEF20E0253050F4A7E12A9FF001D1
:104FAC00EE5CF94FE081AE2FEA8DEA1709F402C0EE
:104FBC002F5FF1CFA7E12A9FF001E15DF94FAF011F
:104FCC00DA0115960C910F3F11F40C9433280E94C2
:104FDC004F7210810E94BA700E945E7DECF4ACE2BC
:104FEC00BCE00E9471710E9455720E949170A08366
:104FFC00B1831A930E94B41EABE00A9FF001E252F7
:10500C00FA4F30810A93FE0137960E945B723A93F5
:10501C00FE0137960E945F720E946572F1F40E9445
:10502C004F72AFEFA083DA011396EFEFEC93DA0136
:10503C001596EC930E9455720E946B72E0E0F0E0C2
:10504C000E949F70E0E0E093290C1A930E94B41E1A
:10505C000A930E94ED10689420F80E946F7D6B9665
:10506C0008951A9310E01031B0F4A7E11A9FF001E3
:10507C00EC5BF94FE081EF73AE2FE981EA1729F46D
:10508C001A930E942B20E03009F403C0E1E0188150
:10509C00E0C01F5FE8CFE0E01881DBC01A93E0911D
:1050AC00520CF091530CFA93EA93E4EFF1E00E9466
:1050BC00AE70F9F00E94707210E01530D0F4A0912F
:1050CC00560CAF5FE5E00E943C7BE093560CEF5F23
:1050DC00EA93C7DFE03059F0E3E0E0932406E09177
:1050EC00560CF0E0EF5FFF4EE093250669C21F5FA0
:1050FC00E4CF66C21A93E0912306E0934E0CE8E7E6
:10510C00F0E0FA93EA93ECEDF0E0FA93EA930E9464
:10511C00FC4610E01530D8F4E12FEF5FEA93A1DFE5
:10512C00E03099F00E940F6CE12FEA5FF0E00E94F2
:10513C00DA6DE5E0F7E10E94786DA6EEBBE00E9427
:10514C0032710E94A06D0E94A86D1F5FE3CF38C220
:10515C00A5DFE0912406E13029F4EDE0F7E10E94AF
:10516C0077723CC0E23029F4EAE1F7E10E947772F1
:10517C0035C0E33051F4E5E0F7E1FA93EA93E091BE
:10518C002506F0E0E050F04F29C0E43019F4E2E2DB
:10519C00F7E11FC0E53031F4E0912506EA930E9457
:1051AC00541120C0E63019F4EAE2F7E112C0E730FE
:1051BC0029F4E0E3F7E10E94777210C0E83029F49B
:1051CC00ECE3F7E10E94777209C0E93059F4EBE4A3
:1051DC00F7E1FA93EA93E0912506F0E0FA93EA936B
:1051EC000E947111E0E0E09324060895A881B98132
:1051FC001196E1E0EC930E94BE70A881B9811296E1
:10520C00ED93FC930E94A41FA881B9811796EC938F
:10521C000E94DE6DA881B98118960E94D671E0912A
:10522C00C605A881B981EC93E091290CA881B981BC
:10523C001696EC93E091890BA881B9811A96EC93A0
:10524C00E091AC0BF091AD0BA881B9811496ED9364
:10525C00FC932296089564970E946A7DA091E20BBC
:10526C00A230E1F4EB8DEA930E94CF180E94A41FA8
:10527C00ACE2BCE00E94D671AAE2BCE0EB8D0E94CD
:10528C00D671E0912F08E093290C0E94C66F3097DD
:10529C0021F00E94C66F0E94A97014C0AA8DAF3F66
:1052AC0009F4CAC0EA8DEA930E94AD1EAB8DAF3FE4
:1052BC0029F40E94BE700E94CB6FEB8FEB8DEA93AA
:1052CC000E94CF180E94A41F0E2FA98DAF3F21F072
:1052DC000E94B01FE03009F001C0AEC00E94917076
:1052EC000E94926CAE17BF071CF023DCE13009F072
:1052FC00A3C0A091D10BA03021F4A091E20BA2305D
:10530C0011F50E94DE6DE13041F00E94A633E030D1
:10531C0021F00E94BC33E03009F002C00E947C7284
:10532C000E94DE6DE13021F40E94AC33E03009F4D0
:10533C0009C00E948872EE55F84FFA93EA9356DF33
:10534C000E948E7277C0EB8DEA93EA8DEA93B0DC03
:10535C001E2F113011F00C94202AA091D30BA130E8
:10536C0059F4E0912F08EA930E94BE70FA93EA93E5
:10537C00EFEFFFEF0E9494720E9491700E94926C6A
:10538C000E9481700E949F70689420F8A091E20B9B
:10539C00A03019F4A88DAF3F09F437C00E94987261
:1053AC00EE51FA4F0E949170A083B183E88D0E9458
:1053BC00816D3081E88DEA93FE0135960E945B7217
:1053CC00E88D0E94816DE081EA93FE0135960E9482
:1053DC005F720E949F1FE03131F00E949872EA5177
:1053EC00FA4FA1E005C00E949872EA51FA4FA2E070
:1053FC00A0830E949872EC51FA4FFF93EF930E9496
:10540C001768AF91BF91ED93FC930E94657219F4EC
:10541C00E0E0E093290CEA8DEA930E94B41EE0913F
:10542C002F08EA930E94C66F0E949D72FA93EA932A
:10543C000E94A21CE1E001C0E0E00E94717D6C962C
:10544C00089577DBE13041F40E94A633E03021F07F
:10545C000E94BC33E03009F007C00E94C66F0E9466
:10546C00A9700E947C7226C32EC30E946A7D0E9482
:10547C00A0721F3F11F40C94922AE0914F0CE03073
:10548C0011F00C94912A1A930E94CF18E5E0E09346
:10549C00240610932506A0911908A23031F40E941D
:1054AC00A9720E947121E03009F010C0A091500C3B
:1054BC00A13331F4E0912F08EA931A930E94041A55
:1054CC00E1E3E0934F0C0E94717DE2C2A0911908B8
:1054DC00A830A1F40E94C66F0E94AD720E2F0A93E1
:1054EC000E941E343E2F1A930A93EFEFEA933A93DD
:1054FC00B2DEE03019F00E94717DCAC2A091190889
:10550C00A53031F49EDFE03019F00E94717DC0C2ED
:10551C00E0E3E0934F0C06C0E0E3E0934F0CE4E0D3
:10552C00E09324060E94717DB3C2E09140090E9471
:10553C00B17208951A93E6E0EA930E94505E0E94BD
:10554C000672A0914009A83539F4E7E5F7E10E940D
:10555C00BD72E0E00E941272A0914009A33509F5DA
:10556C0010E0A0911908A83021F0A23011F0A5305C
:10557C0009F411E3E3E5EA930E94A5621A930E94F1
:10558C00A562E0E8EA930E94A562E0E8EA930E9433
:10559C00A562E0E80E940D72E0934F0CE0E00E94DF
:1055AC001272A0914009A93459F40E94C172E0937F
:1055BC0025060E94CB72EC91E093500C56DF30DB49
:1055CC00199108950E946A7DA0913F09A53411F0AC
:1055DC000C942F2B0E94D072E2E3F0E0E093490C84
:1055EC00F0934A0CA0914009A73741F4E4E4F9E0A8
:1055FC000E94D7720E94DC720E94B172A091400985
:10560C00A03310F0AA3308F023C020912708309162
:10561C002808E0E4F9E00E94D772E2E0EA930E94E5
:10562C004B620E2F0E94DC72E09325060E94DC7206
:10563C000E94E0720E94A0720A931A930E94041AAC
:10564C002093270830932808E2E5EA930E94505EE5
:10565C001CC0E091470CF091480CFA93EA93E0914E
:10566C00490CF0914A0C0E94AE7079F0E0E0E093A6
:10567C003A09E5E4EA930E94505E0E94D072E8EC8D
:10568C00F0E0E093490CF0934A0C0E94717D00C24B
:10569C000E94E5720E94EB720E940F6C0E940F6CCC
:1056AC000E94A446A0911B08A23021F4EFE5F7E17B
:1056BC000E94786DA0911B08A13021F4E6E6F7E179
:1056CC000E94786DE0911B08E03021F4EDE6F7E1E3
:1056DC000E94786D0E94F5720E94506C0E94A44644
:1056EC000E94F8720E94FD72FA93EA93E0915F05B2
:1056FC00F09160050E9403730895E1E003C0E0E0BF
:10570C0001C0E2E0E0931B08C3DF08950E949F1FD5
:10571C00EC3109F0D8C1E091990BE33631F4A0914A
:10572C001908A23009F4EBDF17C0E23631F4A0916E
:10573C001908A23009F4E5DF0FC0A091C505A2300D
:10574C0011F0A63021F4E091990BEA9386D9A0913F
:10575C00C505A43009F4D1DFADC10E94AE6D0E9425
:10576C000F6C0E94B26D0E940F6C0E940F6C0E9415
:10577C00A446E8E7F5E00E94786DE0911A080E94D3
:10578C000773E6E8F5E00E94786DE2E0E0930E0422
:10579C0008950E94F16FE0ECF0E00E94F86FE88150
:1057AC00E03009F406C0A0911A08AF5FE3E00E9454
:1057BC003C7BE0931A08E1E0E0934B0C0E945520EF
:1057CC006FC20E946A7D10E0103410F00C94342CDF
:1057DC000E943271ED55F94F30813F3FE9F11A9338
:1057EC000E94CF1800E00E940B730E94CC6D0E94A7
:1057FC00867B3B9794F00E940E730F010E940B73F3
:10580C000E94CC6D0E9414730E941A730E94BD6F8B
:10581C00EC91EE7FD001EC9301E00E941F730E948B
:10582C00CC6D0E94867B759794F00E940E730F01CD
:10583C000E941F730E94CC6D0E9414730E941A73F5
:10584C000E94BD6FEC91E160D001EC9301E001305E
:10585C0019F41A930E94EF181F5FB6CF0E94717D46
:10586C0017C11A930A9323FE03C00E9422733CD7DC
:10587C000E940343E030C1F1E0E00E94297310382C
:10588C0020F5113219F40E9422732ED71D3439F4ED
:10589C000E9430730E94BB63E3E0E09318081B3254
:1058AC0071F40E943573EAE2EA93E8E7F7E1FA93C0
:1058BC00EA93E0911A08E05DEA930E94BB631F3201
:1058CC0019F4E1E0EA93C9D848DF103868F00E9477
:1058DC003B731A930E94302119DFE03011F410321F
:1058EC0008F002C0EEE5F6E20E949A210E2F003875
:1058FC00C8F10F770034A8F5E0911F08E03031F0C3
:10590C000A930E94C211E0E0E0931F08E091570C4B
:10591C00E01739F10A930E94CF180E943F71AC91A5
:10592C00A83028F40E944471AC91A830A8F0E02F64
:10593C00EF5FE093A2060A930E9430210E943F7110
:10594C00EC91EA930E944471EC91EA93E091A206E7
:10595C00EA930E94351F03C0E0E0E093A206009397
:10596C00570C0EC0A091570CAF3F51F0E091A2061E
:10597C00E03019F0EA930E94521FEFEFE093570CBE
:10598C00099119910895A881A03310F0AA3308F059
:10599C001DC00E943F730E944473AAE0B0E00E94B5
:1059AC00E27ADF01E8810E944973EA0FFB1FE09362
:1059BC002508F0932608E2E0E0930E040E94F572AD
:1059CC000E94506C0E94B26D0E94F872A881A334A0
:1059DC0051F40E94EB720E94F5720E94506C0E946E
:1059EC00B26D0E94F8725CC11A930A93A0E023FC7A
:1059FC00A1E0A03019F0AA81A03009F016C0E894FB
:105A0C0023F8E7E0E09318080E94EB45A0913108D9
:105A1C00A03019F40E944C7309F407C0E7E0EA9334
:105A2C000E94517361D6E89424F824FE24C00E948D
:105A3C005473EAE5F0E00E945B7319F0AA81A1307F
:105A4C00C9F47ED6E030B1F00E9461730FEF1FEF06
:105A5C000E94A9720E944821E03021F4009127088D
:105A6C0010912808EB81EA93E0912F08EA931A939E
:105A7C000A933AD60BC00E945473ECE2F1E00E94F8
:105A8C005B7321F40E946873E093300819810881DC
:105A9C0024960895E091C70BF091C80B0E946C738B
:105AAC0011F4E2E00895E091C50BF091C60B0E9451
:105ABC006C7311F4E1E00895E091CB0BF091CC0BF9
:105ACC000E946C7311F4E0E00895EFEF0895E0E0AC
:105ADC00E0931B08A0911908A23021F40E94CB4638
:105AEC000E94000FA0911908A83009F45CD6A0916F
:105AFC001908A53009F443D10895E2E0EA930E9415
:105B0C00CF40E2E0E0930E04E881EA933CDFA88109
:105B1C00AF3721F4E0912B06E37009F403C0E2E007
:105B2C00E0931808A881A13239F0A33421F40E9423
:105B3C003F73109709F004C0A0911908A23009F026
:105B4C000FC0A0911B08A33009F4DBDDA0911B084A
:105B5C00A23009F4BCDFE0911B08E03009F4CFDD82
:105B6C00A881AD3311F00C94122E0E94EB45E091FC
:105B7C001B08E030A1F4E0912508F0912608FA9377
:105B8C00EA930E947121E03041F4E0912508F091F4
:105B9C0026080E94E0729BDF01C0B1DD3DC0E13000
:105BAC0069F478DFEF3F41F0E3E00E9470730E94EC
:105BBC0030730E94767301C08ADF2EC0E230F1F49C
:105BCC000E943F73A034E0E0BE07B4F4E0912508D6
:105BDC00EA930E947D73E2E0E0930E040E940F6C46
:105BEC000E940F6C0E94A4460E946B6D0E9455107F
:105BFC00E3E0E0931B0801C084DD0EC0E33061F4E8
:105C0C00E0912508EA930E94CF18E0912508EA93C9
:105C1C00EEEFEA934DD875DDA881AD3409F46DDD56
:105C2C00A881A43521F4A0911908A23009F001C073
:105C3C0066DDA881AB3221F4EEEFEA930E943325A6
:105C4C00A881AD3221F4EFEFEA930E943325A881AD
:105C5C00A73421F4E1E0EA930E943325A881AB3408
:105C6C0021F4ECEFEA930E9433251AC00E94CD2058
:105C7C000E94CB46E0E0E0931B08A881A13039F4E8
:105C8C000E944C7321F0A091CA0BA03009F402C001
:105C9C0036DD06C00E94000F0E94A9720E944821A6
:105CAC00219608951A930A930E9481730E947F1F74
:105CBC000E940343E03091F10E948A7378F10E94B4
:105CCC003B7324DDE03051F50E9492730E94062153
:105CDC00EF3F09F006C50E94A9720E947121E030C5
:105CEC0021F40E94B01FE13009F018C00E949F1FE0
:105CFC00E83119F40E94977309F001C0F2C40E94B4
:105D0C0092730E945E260E2F013021F4A091990B04
:105D1C00A03009F403C01A930E945411A0912E06CE
:105D2C00AF3F61F110912E06EFEFE0932E061A9320
:105D3C000E94CF180E94A9720E947121E03021F4B8
:105D4C000E94B01FE13009F019C00E949F1FE8317A
:105D5C0019F40E94977309F001C0C3C41A93EEEFB3
:105D6C00EA930E945E260E2F013021F4A091990B2C
:105D7C00A03009F403C01A930E945411B2C40E94BB
:105D8C00CD200E945520E89421F8E0E0E0931E0815
:105D9C000E949E730E94CB460E940F6C0E940F6C57
:105DAC000E94A446E09132060E94EF6DE09133060A
:105DBC000E94EF6D0E940F6C0E94736D0E94A446AE
:105DCC00E0913F060E94EF6DE0913906F0913A06A2
:105DDC000E94C56D08950E946A7D0E9481730E9485
:105DEC000343E03049F00E948A7330F00E943B7309
:105DFC008DDCE03009F425DBE091540CF091550C6E
:105E0C000E948F6E11F40C946B2F0E949E730E9453
:105E1C000F6C0E94666D0E94B26DE0913706F09196
:105E2C0038060E94C56DE0913B06F0913C060E943D
:105E3C00C56D00E0053010F00C946B2FA7E10A9FA4
:105E4C00F001E15DF94F9F01F901A381AF3FD9F159
:105E5C00D9011A960E94D16D7F936F93FF93EF93A4
:105E6C000E94A573AF91BF918F919F910E94A47ACC
:105E7C000E94E77ADF01CB010E94AA73D9011C961C
:105E8C00ED93FC93F90104841584D9011E960E94AC
:105E9C00867BE015F105B9F0F90104841584A6851B
:105EAC00B785F001EA1BFB0BE093AC0BF093AD0B49
:105EBC00C8DAE13041F4D9011C960E94867BD901E5
:105ECC001E96ED93FC930F5FB5CF0E94717D2AC493
:105EDC000E946A7D0E9481730E947F1F0E9403436F
:105EEC00E03011F40C9404300E9406430E2F0A93F8
:105EFC0004DE003820F0A091C605A03808F429C0B3
:105F0C000F770A930E94B1730E94AD721E2FA0915D
:105F1C00E20BA03011F41F3F09F416C030E035300D
:105F2C0098F4ABE03A9FF001E452FA4FE081E117AC
:105F3C0049F43A9FF001E252FA4FE081EF5FE093AF
:105F4C00C605232F3F5FEBCF0A930E9492732A93CF
:105F5C0054C0A091E20BA03021F4003810F00538A9
:105F6C0008F00AC00F770E944F721081EFEFEA938E
:105F7C000E9492730A936FD9A091E20BA03011F09A
:105F8C00003808F43BC00F770A930E94CF18BEDB91
:105F9C00E030A1F50E94B4730E940621EF3F19F086
:105FAC000E94717DBFC30E94B01FE13039F50E9481
:105FBC00A41FE03049F40E94B4730E945E26E030C6
:105FCC0011F00E94B9731AC00E949F1FE83141F46E
:105FDC000E94977321F00E94B4730E945E260EC03B
:105FEC00A0911E08E02F0E94456DAE0FBF1F1C91A3
:105FFC000A930E949273EFEFEA932DD9A0912E068B
:10600C00AF3FF9F000912E06EFEFE0932E060A93C6
:10601C000E94B1730E94AD721E2F0A931A93EEEF79
:10602C00EA93EFEFEA9317D91F3F41F4A0919D0B30
:10603C00A03021F4A091A00BA03009F002C00E9466
:10604C00B97320FE0AC0E89420F8E091E20BE0302E
:10605C0019F401D452D501C0B1D530E0353080F5FA
:10606C00ABE03A9FF001DF01EA51FA4FE081E030FA
:10607C0049F0AC51BA4F0E94BF73E8EEF3E00E94B6
:10608C00AE7099F4ABE03A9FF001EA51FA4FE0811F
:10609C00E23051F43A9FF001EC51FA4FDF010E94CB
:1060AC00867B0E948F6E09F409C0ABE03A9FF00129
:1060BC00EA51FA4FA0E0A083689420F83F5FCECF5E
:1060CC000E94717D2FC30E94C66CA33011F40C94F6
:1060DC002232E0913A08ED3411F00C944B31E091FE
:1060EC003B08EA3511F00C94003124FC83C0E0919C
:1060FC003C08E0532E2FE0913D08E0533E2FEEE399
:10610C00F8E00E94D7720E94CB72AC91AB3429F4A8
:10611C000E94C4730E94D7610E2F0E94CB72AC9167
:10612C00A43529F40E94C4730E94D761AF01E09199
:10613C00CD0BE31731F5E0E0E0934D0C0E94617359
:10614C004093270850932808A09130080A1759F05B
:10615C00E7E0E09318080093300820934C0CE0E043
:10616C00E0932F080DC0A0914C0C2A1721F0A091A0
:10617C002E08A03009F004C02093180820934C0C72
:10618C0035C0A0913008A03049F4A091CE0B0E94EC
:10619C00AA6CE255FF4FE491EA2309F40CC0E7E046
:1061AC00E093180820934C0CE0E0E0932F08E0916A
:1061BC003908E0934D0CE0913908A0914D0CEA1789
:1061CC00A9F44093270850932808009330080E94A4
:1061DC006173A0914C0C2A1721F0A0912E08A030CD
:1061EC0009F004C02093180820934C0C273011F4AC
:1061FC000E94D370E0913B08E93439F4E7E00E9447
:10620C0070730E946873E0932F08E0913B08E234AE
:10621C0039F4E4E00E9470730E946873E0932F08D5
:10622C00E0913B08E03519F4E1E0E0931808E091C7
:10623C003B08EC3449F4E4E0E0931808E0913C08A6
:10624C00E053EA930E941916E0913B08E334E9F419
:10625C00A0913C08A13320F0A0913C08A93308F090
:10626C0014C00E94C773E0912208EA930E941F1B7E
:10627C00E0913908EA93E4E8F7E1FA93EA930E9493
:10628C00FC6F0E94997B0E94AE63E0913A08E03566
:10629C0021F4A0911908A13009F003C00E943573B4
:1062AC005CDAE0913A08EF3459F4E0913B08EE34B3
:1062BC0039F4E0913908EA93E7E8F7E10E94CD73ED
:1062CC00E0913A08E33569F5E0913B08EF3349F585
:1062DC00A0913C08A03320F0A0913D08A03308F415
:1062EC0020C00E94C773E0913D08E0531E2FA0917F
:1062FC002208A63010F41A3008F013C0103011F434
:10630C000E94691AE0913908EA93EAE8F7E1FA93F6
:10631C00EA930E942F700E9412700E94997B0E9437
:10632C00AE63E0913A08E33411F00C94EA31E09159
:10633C003B08EF3311F00C94EA31E0913D08E03367
:10634C0019F4EFEFE0932308A0913C08A033F8F088
:10635C000E94C773A0912208A630C8F4E0912308CC
:10636C00EF5FE0932308E0912208EA93E091230881
:10637C00EA930E94E51AA0911E0CB0911F0C109785
:10638C0021F4A0912308A03408F001C0E7CFE091DC
:10639C002308EA930E94CF180E94D373EDE8F7E12B
:1063AC000E94BD720E94D26E0E94D8730E94DD734F
:1063BC000E94D76E0E94997B0E94DD730E94396FF8
:1063CC000E942F630E947E63E0913A08E434A1F5A9
:1063DC00E0913B08E43481F514E0E1E0E093390905
:1063EC00103538F40E943271E85CF74FE081E032EE
:1063FC0008F41AC00E943271E85CF74FE081E33276
:10640C0059F40E943271E75CF74FE081E053EA9354
:10641C000E94505E1F5F06C00E943271E85CF74F0D
:10642C000E9402721F5FDCCF0E94D373E0E9F7E198
:10643C000E94BD720E947E630E946F7D2696089515
:10644C001A930A930E94E07111F40C94A232E0E0CA
:10645C00E093590CE0911808EF770E2F0093180871
:10646C000E94CB460E94736DE4E0F0E0FA93EA934D
:10647C000E94A446013021F0A0911908A13009F026
:10648C000BC0EEE8F5E00E94786D9BD9E4EFF1E0EB
:10649C000E942C6C0E94CB46073049F40E94CD2000
:1064AC00E0E0E0931B080E94F5110E948028043064
:1064BC0031F4E3E9F7E10E94786D0E94B50D0830E4
:1064CC0019F40E94E3736FD1053019F40E94E37341
:1064DC0056DC013051F4E89423F8E0E0EA9359D902
:1064EC00009319083AD90E94000F093071F4E0E0CA
:1064FC00EA934FD9E0E0E0931E08E89423F80E9459
:10650C00000F0E94ED73E093590C023069F4E0E047
:10651C00E0931E08E0E0F0E00E94E072E89423F8BB
:10652C000E94ED73EA93A2DB033011F40E948140C8
:10653C00009319080E947F1FA0911908A73011F031
:10654C000C945033E091520CF091530C0E948F6ECE
:10655C0021F0A0911B08A03009F00AC00E947072B3
:10656C00E0914E0CA0912306EA1711F00E948028AE
:10657C000E940343E030E9F0E2E00E9429731A9391
:10658C0002DA1D3409F4B9D81D3399F40E94EB4595
:10659C0081DAEF3F41F0E3E0E09318080E9430739A
:1065AC000E94767306C0E7E8E0931808E0E0E093F9
:1065BC001B08A0912F08A03031F0E0912F08A0917A
:1065CC002E08EA1709F457C0E0912F08E150EA931E
:1065DC000E942419A091340CE1E0EA23E13021F46B
:1065EC00E0912B06EF7C09F429C0E0E0E0932E0843
:1065FC00E0914C0CE03019F0E09318081EC012E04A
:10660C00E0912B06EC7009F018E0E091C40BA0911E
:10661C002F08EA1781F0E0912B06E07439F011E0B5
:10662C00EAE2EA93E8E9F7E10E94CD73E0912B06E8
:10663C00E07809F019E0109318081DC00E94CB46B1
:10664C000E94F5110E94736DE4E0F0E0FA93EA9376
:10665C000E94A446EBE4EA930E944246E0912F0884
:10666C00EA930E947041EBE9F7E10E94786DE091AA
:10667C002F08E0932E08A0912F08A03021F4A091B0
:10668C002E08A03009F406C0E0E0E0932E08E7E8FD
:10669C00E0931808A0911908A33011F40E947E3ED3
:1066AC00A0911908A13009F4DCD8A0911908A230E6
:1066BC0009F4F8DAA0911908A83009F409DCA091C2
:1066CC001908A53009F487DBA0911908A93049F401
:1066DC00E0E0E0932008E0911908EA93E0E0EA9307
:1066EC0083D90991199108950E94F473E652F84FD9
:1066FC00A6E0A0830E94F473E752F84FAB81A0830D
:10670C000E94F473E152F84FAA81A0830E94F473A3
:10671C00E552F84FA881B981A083B1830E94DA7148
:10672C000E94FE50249608950E94FA73A881B981A4
:10673C00AC91A53020F0A881B981E0E0EC9389C040
:10674C00A0911308BB27E091120805C0A091110875
:10675C00BB27E0911008F0E031960E9481703596CD
:10676C00DF01E5E0F0E00E943F7B08951A93109161
:10677C001308E0911208E117A1F0ABE01A9FF001A9
:10678C00E652F84FE081E13011F0E23011F4E1E033
:10679C004DC0EDB7FEB7FA93EA931F93C5DF1F9177
:1067AC00E8CFE0E043C01A930E94CD20ECEDF5E079
:1067BC000E9446700E94F26C0E94A36810E0153093
:1067CC0068F40E94B470AFEFA083ABE01A9FF001A5
:1067DC00EE51FA4F0E946B721F5FF1CF10E0153033
:1067EC0048F4A7E11A9FF001EC5CF94FAFEFA083DE
:1067FC001F5FF5CFE0912B06E37019F00E944C73EC
:10680C0009F402C0689401C0E89421F8EFEFE0931A
:10681C002D08E091E20BE03029F41DD06ED1E89404
:10682C0020F804C00E94CB460E94870F199108954E
:10683C001A9310E0153058F40E94B470E081AE2F1A
:10684C00E981EA1711F4E12F03C01F5FF3CFEFEFDB
:10685C0018812296089522970E94687D00E00530E9
:10686C0058F40E940074A0E00E940674E152FA4FA2
:10687C00A0E0A0830F5FF3CF00E00530C0F50E94CD
:10688C004F72E081EF3F89F10E944F72E0810E94CC
:10689C00C370B9F00E945572DF010E94867B0E9482
:1068AC009170EA17FB0751F00E9455720E9491708B
:1068BC00A083B1830E940B74A1E0A0830E9400749A
:1068CC0012C0ABE00A9FF001EA51FA4FE081E030D0
:1068DC0061F40E944F72AFEFA0830E9455720E9428
:1068EC006B720E940B74A1E0A0830F5FC6CF0E9455
:1068FC009F1E1E2F1F3F11F0E1E001C0E0E0E0936E
:10690C00590C1F3F11F40C94DD3450E000E00530BD
:10691C0048F40E944F72E0811E1711F451E002C03E
:10692C000F5FF5CF5030E1F500E00530C8F50E945F
:10693C004F72E081EF3F91F50E944F7210830E94DD
:10694C0055720E949170A083B183ABE00A9FF00155
:10695C00E052FA4FA091290C0E940674EF51FA4FA5
:10696C00FF93EF930E94BE700E94CB6FAF91BF91CB
:10697C00EC930E940B74A1E0A0830E940074A1E030
:10698C000E940674EC51FA4FFF93EF930E94176824
:10699C00AF91BF91ED93FC9351E002C00F5FC5CF57
:1069AC00503029F01A930E94A61E1E2FAACF30E059
:1069BC00353010F00C942335A7E13A9FF001E15DDE
:1069CC00F94FEE83FF8350E000E0053048F550307E
:1069DC0029F5ABE00A9FF001EF51FA4F20812A9381
:1069EC000E94CF180E940074E081E13059F42A9380
:1069FC000E94C01FE13031F4A32FAF5FE0919D0BDB
:106A0C00EA1709F00BC0E22FAE81BF811396EC930D
:106A1C00E02FAE81BF811596EC9351E00F5FD5CF7F
:106A2C00503049F4AE81BF811396EFEFEC93AE81F9
:106A3C00BF811596EC933F5FBBCF0E946F7D0C948A
:106A4C00CB370E946A7DAC81BD81EBE4EC93EC8189
:106A5C00FD813196FA93EA930E941174E052FA4F39
:106A6C00E0810E946A6C00E00E941A74EC91E030A4
:106A7C0011F00F5FF9CF0E941A74E0E2EC930F5FF4
:106A8C000E9420740E94206D0E941174EE51FA4FE6
:106A9C00DF010E94D16D0E942574EE81ABE0EA9F6C
:106AAC00F001EF51FA4F10811A930E94CF1800E0B9
:106ABC000E941A74EC91E03011F00F5FF9CF0E9434
:106ACC001A74E8E7EC930F5F0E941A74E0E2EC93FF
:106ADC000F5F30E03A3060F40E942074EA0FFB1F25
:106AEC000F01AAE8BBE00E942C740F5F3F5FF2CF4E
:106AFC000E941A74EC930C94103864970E946A7D6F
:106B0C0000E010E0153040F40E94B470E081EF3FDB
:106B1C0009F40F5F1F5FF6CF053021F0A0912D080F
:106B2C00A03009F406C0E0E0E0932D08EA930E943F
:106B3C00A21010E0153088F5ABE01A9FF001E1527D
:106B4C00FA4FE081E03039F11A9FF001E352FA4F2D
:106B5C00E081E030B1F01A93FE0135960E945B7231
:106B6C00ABE01A9FF001EF51FA4F30813A930E943B
:106B7C00CF181A93FE013596FA93EA930E94FD10F2
:106B8C000AC01A930E94ED10ABE01A9FF001E1527B
:106B9C00FA4FA0E0A0831F5FCDCF053021F4A09168
:106BAC002D08A13009F406C0E1E0E0932D08EA932A
:106BBC000E94A2100E94717D689608950E94687DC3
:106BCC00A091E20BA23011F40C94AA3930E03431CC
:106BDC0068F40E9433740E943674DA011296E0E075
:106BEC00EC93DA01EFEFEC933F5FF1CF0E949F1E25
:106BFC000E2F0F3F11F0E1E001C0E0E0E093590CE3
:106C0C000F3FA1F10E94BE70FA93EA930E947F1885
:106C1C001E2F1F3F31F1A0911E08E12FEA1B3E2FC2
:106C2C003431F8F40E9433740E943674FA013296AF
:106C3C000F01E081AE2F0E943C74B0E0EA0FFB1F05
:106C4C00D001EC93FA01A281A43620F0DA0112965D
:106C5C00E3E6EC93DA01AC91AF3F19F4E02FDA01E3
:106C6C00EC930A930E94A61E0E2FCACF0E943215D7
:106C7C0030E0343110F00C94C9360E9433740E9409
:106C8C003674FA01A381AF3F11F40C94C7360E94FD
:106C9C0041740E94C16FE83139F40E944174EA9347
:106CAC000E94C617E03009F408C00E944174EA93B0
:106CBC000E94C617DA011296EC93A0919A0BA07859
:106CCC0039F4FA010280DA011196EC91E01509F41D
:106CDC0058C0DA0113962C91ADE02A9FF001EF5EBB
:106CEC00FC4F0F01DA011296EC91D001EC930E944B
:106CFC004174EA930E94E320EF3F29F0ADE02A9F14
:106D0C00F0010E94256DDA011296EC91E03089F0C9
:106D1C000E944674DF010E94406DEC93ADE02A9F07
:106D2C00F001E25FFC4FDF01E091980BEF70EC9308
:106D3C0013C00E94406DE03021F40E944674A0E024
:106D4C0003C00E944674A8E0A083ADE02A9FF00126
:106D5C00E25FFC4FA7E0A0830E944174EA930E947B
:106D6C00E320EF3F19F0ECE0E0930F04DA01129608
:106D7C00EC91DA011196EC932A93E1E0EA930E94EC
:106D8C002D473F5F76CF0C94AA39E7E0E0931808C3
:106D9C000E940818A8950E94661CA8950E94BB1E0C
:106DAC00A895EFEFE093B20BE093890BE093330CD3
:106DBC00E0932E0CE0932E060E944C74EC7F29F08D
:106DCC00A8E0B0E0E0E00E94C87B089524970E9400
:106DDC006A7D0E941E42E8EAF7E10E9446700E941A
:106DEC00AA420E944642E0912208E03061F0E3EBB7
:106DFC00F7E10E9446700E94AA42E09122080E948C
:106E0C0051740E9455740E9446420E94691A00E017
:106E1C000A30A0F40A930E94FE180E945F6FEFE004
:106E2C00EA930E948442E02FA3EAB6E00E945974D0
:106E3C000E9412700E945D740F5FEACF0E9458424C
:106E4C00ECEBF7E1FA93EA93EFE0EA930E94AA42A3
:106E5C000E949F6E0E945D740E945A420E9446429C
:106E6C0010E0103110F00C94C7370E94DE6DE11762
:106E7C00E1F5E2ECF7E10E9446700E94AA420E9402
:106E8C00616D0E945574E0E0E0931E08A0911E080D
:106E9C00A03448F5E0912208EA93E0911E08EA93A9
:106EAC000E94E51A0E94D26E3097B9F0E0911E084C
:106EBC00EA930E94CF180E94D26EFA93EA930E9432
:106ECC0063740E94AA420E94396FEAE0EA930E941E
:106EDC0084420E94D76E0E945D74E0911E08EF5FA1
:106EEC00E0931E08D3CF0E9468740E9432710E94F6
:106EFC00177011F00C94C537E2ECF7E10E94467064
:106F0C000E94AA420E94616D0E9455740E946C748A
:106F1C00E0E30E94237029F40E9428700E94D7613C
:106F2C009F0100240216030644F50E94C4730E94BC
:106F3C0001620E94426E0E94C4730E9474743A9360
:106F4C002A930E9463740E94AA420E947874EAE019
:106F5C00EA930E948442EC81FD816E817F810E94C4
:106F6C005D740E946C74E1E30E94237029F40E940A
:106F7C0028700E94D7619F01D4CF0E9468741F5F54
:106F8C0070CF0E941F420E94717D289608950E9426
:106F9C006A7DAD81BE812C910E947D740E94616DD1
:106FAC000E94926C0E94DA6DECE3EA930E944246D6
:106FBC00EC81EA930E9496462A93ED81EA930E9413
:106FCC001041EEE3EA930E9442460E94FD720E9439
:106FDC009D720E9403730E948274333409F431E26F
:106FEC00313320F0EC81E05DE31708F407C0E32FA8
:106FFC000E944973E255FF4FE4912E273D3311F067
:10700C00313209F401C0CACF3D3319F4AD81BE81D0
:10701C002C93E32F0E94717D279608950E94687D22
:10702C0020E0AF81B8855C910E947D740E94616DF7
:10703C000E94926C0E94DA6DE2E0EA930E949646FE
:10704C005A930E9470410E94FD720E949D720E9490
:10705C0003730E948274303310F03A3308F00EC080
:10706C00203009F450E021E0A52FEAE00E943C7B9F
:10707C00AAE0EA9FF001E30FE0535E2F3B3211F4DC
:10708C00533608F001C05F5F3D3211F4513008F403
:10709C0001C05150333429F4203009F431E250E06E
:1070AC0020E03D3319F4EE81E51708F005C0AF81FF
:1070BC00B8855C9130E020E03D3311F0313209F4B9
:1070CC0001C0B4CF3D3319F4AF81B8855C93D0C007
:1070DC000E94687D20E0AF81B8854D915C910E9443
:1070EC007D740E94616D0E94926C0E94DA6DAE817B
:1070FC00A23051F4E6E0EA930E949646FA010E940F
:10710C00D8730E944F4108C0E5E0EA930E9496466E
:10711C005A934A930E945A410E94FD720E949D729A
:10712C000E9403730E948274303310F03A3308F0DB
:10713C001EC0203011F440E050E021E04031E7E285
:10714C005E0734F0DA01E0E1F7E20E943F7BAF0129
:10715C00493BEBE05E0724F0DA010E944473AF0177
:10716C00DA010E9487740E948C74D097AD013B3277
:10717C0021F44033E5E75E070CF002C04F5F5F4F30
:10718C003D3221F40024041605060CF002C04150D7
:10719C005040333431F4203009F431E240E050E017
:1071AC0020E03D3311F0313209F401C09ACF3D3368
:1071BC0021F4AF81B8854D935C935AC00E94687DD1
:1071CC000E947D7420E050E04FEF0E94616D0E94A0
:1071DC00926C0E9491740E949474E885EA930E94C8
:1071EC006E46E52FE10FF0E00E949D720E94037342
:1071FC000E948274303310F03A3308F021C03053BF
:10720C00431729F04F3F09F05F5F20E005C0A22F24
:10721C00AF5FEA2FE3702E2FE52FAF81B8850E9468
:10722C0099740F01E32FA6ECB6E00E945974AE0FCF
:10723C00BF1FE22F0E949974E491D001EC93432F6D
:10724C003B3219F4EE815E1708F002C05F5F4FEF1E
:10725C003D3211F4513008F402C051504FEFEE8121
:10726C005E1720F4313211F03D3309F401C0ADCF7B
:10727C00E32F0E946F7D299608951A930A93A0918B
:10728C009A0BECEDEA231E2F00E00D3040F40E9427
:10729C009D740E94A174E11711F00F5FF6CF0E944C
:1072AC009D74EA0FFB1F0E94957B0E94786DE02F66
:1072BC003DC4AAE9BBE00E94C96DAE0FBF1FEC91A3
:1072CC00E17011F4E3E701C0E9E4EA930E9442465D
:1072DC00219608950E94687D0E947D740E94616DC4
:1072EC000E94926C0E949174C8DF5E2F0E94FD7206
:1072FC000E949D720E9403730E9482743D3211F0B1
:10730C00363311F4503009F401C051503B3211F0B6
:10731C00333311F45C3008F001C05F5FA0919A0B1D
:10732C00E1E0EA232E2FE52FA0E0B2E00E94597491
:10733C000E94A174E20FE0939A0B3D3311F03132AD
:10734C0009F401C0CBCFE32F0E946F7D26960895E0
:10735C000E946A7D0E947D740E94616D0E94926CF5
:10736C000E949174AAE9BBE0EC810E94BD6FEC9184
:10737C00E17019F4EFECF7E102C0E3EDF7E1FA93F9
:10738C00EA930E9459460E94FD720E949D720E94CF
:10739C0003730E948274303310F03A3308F00FC03C
:1073AC00AAE9BBE00E94E16F0F01AAE9BBE0EC8106
:1073BC000E94BD6FAC91E1E0EA27D001EC933D3324
:1073CC0011F0313209F401C0C7CFE32F0E94717D57
:1073DC00259608950E947A6CE1E0EA930E949F0E34
:1073EC000E940F6C0E940F6C0E94A4460E94396F81
:1073FC00EAE0EA93E3DEE13209F45FC40E940F6C29
:10740C000E940F6C0E94B26DE7EDF7E10E94786D5F
:10741C00E5E9FBE00E9446705BDEE13209F44DC405
:10742C000E940F6C0E940F6C0E94B26DEDEDF7E1A3
:10743C000E94786DE091970BEF5F0E2FEDB7FEB7C2
:10744C00FA93EA930F93EAE0EA93E8DD0F91E132C5
:10745C0009F433C400240216030624F4E02FE1508F
:10746C00E093970B0E940F6C0E940F6C0E94B26D00
:10747C00E6EEF7E10E94786DECEAFBE00E94A67460
:10748C0009F41BC40E940F6C0E940F6C0E94B26D19
:10749C00ECEEF7E10E94786DEEEAFBE00E94A67438
:1074AC0009F40BC40E940F6C0E940F6C0E94B26D09
:1074BC00E2EFF7E10E94786DE9E9FBE0FA93EA93D9
:1074CC00E3E60E94AF7409F4F8C30E940F6C0E94AB
:1074DC000F6C0E94B26DEBEFF7E10E94786DFADE53
:1074EC00E13209F4EAC310E0133010F00C94353B90
:1074FC000E940F6C0E940F6C0E94B26DE12F0E94D3
:10750C000773E1E0F8E10E94786D0E94B4740E9468
:10751C00A446ADE9BBE00E9432710E94206DE0E10F
:10752C000E94AF7409F4C9C3E9E0F0E00E94506C0A
:10753C000E94A446A0EABBE00E9432710E94206D1A
:10754C00E0E10E94AF7409F4B8C30E940F6C0E9472
:10755C000F6C0E94B26DE12F0E940773ECE0F8E112
:10756C000E94786D1A93F4DEE13209F4A6C30E94EE
:10757C00B4740E94B87451F40E94EA710E94C274EF
:10758C00E2E00E94C67409F498C309C00E94EA7133
:10759C000E94C274E0E00E94C67409F48EC30E947B
:1075AC000F6C0E940F6C0E94B26DE12F0E9407734A
:1075BC00EEE0F8E10E94786D0E94B4740E94A4463B
:1075CC00A9EABBE0EE27A10FBE1F2C913327EDB724
:1075DC00FEB73197FA93EA933F932F93E0E0EA9347
:1075EC0077DD2F913F91E13209F467C3A9EABBE043
:1075FC000E943271EA0FFB1F2083123070F50E943B
:10760C000F6C0E940F6C0E94B26DE12F0E940773E9
:10761C00E5E1F8E10E94786D0E94B4740E94A446E2
:10762C00A0EBBBE0EE27A10FBE1F2C913327EDB7CB
:10763C00FEB73197FA93EA933F932F93E0E0EA93E6
:10764C0047DD2F913F91E13209F437C3A0EBBBE04A
:10765C000E943271EA0FFB1F20831F5F45CF2DC3A1
:10766C000E946A7D10E01A930E947D730E94CB7475
:10767C000E940F6C0E94A4460E94EA6D0E94CF7477
:10768C000E946B6D0E94C66F0E94C56D0E940F6CAC
:10769C000E94736D0E94A4460E94D46F0E94D66D06
:1076AC00E7E0F0E0FA93EA930E94736D0E94A4461F
:1076BC00E091AE0BF091AF0B0E94A47A0E94D66DB4
:1076CC000E940F6C0E94666D0E94A446ECE1F8E1EA
:1076DC000E94786DE091970BEF5FEA930E947041E6
:1076EC00E7E0F0E0FA93EA930E94666D0E94A446EC
:1076FC00C4DD0E94B66DE091990BE03029F0E09169
:10770C00990BEA930E94704100E00330D8F50E9477
:10771C000F6CE02FED5FF0E00E94DA6D0E941772A3
:10772C00EA930E947041EBE2EA930E9442460E9467
:10773C001E72EA930E9470410E94B66D0E942572DF
:10774C0051F40E942D720E94CC6D0E94D16D0E944A
:10775C00D374E3E709C00E942D720E94CC6D0E9485
:10776C00867B0E94C56DE9E4EA930E9442460E9422
:10777C00B66D0E943772EA930E9476410E94D774CC
:10778C000F5FC3CF0E9406433E2F3B3211F41034DF
:10779C0008F001C01F5F3D3211F4113008F401C034
:1077AC0011503D3439F41A930E94CF1813DE1A93FA
:1077BC000E94EF18313209F056CF7FC20E946A7DC9
:1077CC0010E00E94CB46012F0E940F6C0E940F6CA0
:1077DC000E94A446E0E2F8E10E94786D31E03C3072
:1077EC0018F51038F8F40E940F6C0E94AA6C0E94D5
:1077FC00DA6D1A930E9424190E94EA6D0E94B66DEC
:10780C00A091340CE3E00E94DB74A091350CE7E00E
:10781C000E94DB74E0912B06EA93E8E0EA930E9465
:10782C00104113953F5FDBCF0E94B50D0E940643BC
:10783C003E2F3D34E9F50E94E572102F1038C0F54B
:10784C001A930E9424190E940F6C0E940F6C0E94C4
:10785C00B26DE4E3F8E10E94786D0E94EA6D0E943B
:10786C00CF740E94F16D0E94A446E7E3F8E10E94F8
:10787C00786DE4E3FCE0FA93EA93E3E00E94AF74E2
:10788C0009F41BC20E94F16D0E94B26DEDE3F8E1A8
:10789C000E94786DE5E3FCE0FA93EA93E7E00E943E
:1078AC00AF7409F40AC21A930E9458191F5FC6CF0D
:1078BC00313211F0103808F001C083CFFEC10E94A4
:1078CC007A6C0E94CB740E940F6C0E94A446E3E475
:1078DC00F8E10E94786D10E01530F0F41A930E94D4
:1078EC0066190E940F6C0E94B56E0E94EA6D0E9490
:1078FC00CF74E0912F0C0E94E074E091320C0E9446
:10790C00E074E091300C0E94E074E091310CEA9349
:10791C000E9476411F5FE0CF0E9406430E2F0D346C
:10792C00E9F50E94E57210E01530C0F51A930E943B
:10793C0066190E940F6C0E940F6C0E94B26DE6E5F6
:10794C00F8E10E94786D0E94EA6D0E94CF7430E0DD
:10795C003430F8F40E94F16D0E94B26D0E94AA6C52
:10796C000E94977AEA55F94F0E94957B0E94786D98
:10797C000E94AA6C0E94977AEA55F94F0E94E4740F
:10798C00FD013596E4910E94AF7409F496C13F5FF6
:10799C00DFCF1A930E9486191F5FC6CF8EC10E943B
:1079AC00EB6BE1E0EA930E949F0E00E0083210F0CE
:1079BC000C949C3D0E94810D0E940F6C0E940F6CD8
:1079CC000E94A4460E94926C0E94E7740E94957BD0
:1079DC0031960E94786D0E94B66D0E94926C0E9446
:1079EC00E7743496E491E038A9F40E94DE6D1E2F02
:1079FC00EDB7FEB7FA93EA931F93E0E1EA930EDB3F
:107A0C001F91E13209F492C0E12FA9E0B0E00E948D
:107A1C00C87B88C0E238A9F40E944B701E2FEDB7CA
:107A2C00FEB7FA93EA931F93E0E1EA93F7DA1F911A
:107A3C00E13209F47BC0E12FAAE0B0E00E94C87BE0
:107A4C0071C0E138E1F40E944C741E2FEDB7FEB703
:107A5C00FA93EA931F93E3E0EA93E0DA1F91E132A1
:107A6C0009F464C00E94810D0E944C74E11731F03E
:107A7C00E12FA8E0B0E00E94C87BFFCF53C0E030FC
:107A8C0069F40E94926C0E94E77432960E947C6D9D
:107A9C00E1E00E94AF7409F449C044C0E13069F4DC
:107AAC000E94926C0E94E7740E94E474FD0135966A
:107ABC00E4910E94AF74D1F135C0E23061F40E94C0
:107ACC00926C0E94E77432960E947C6DEFE00E94EB
:107ADC00C67461F127C0E33071F40E94926C0E946D
:107AEC00E7740E94E474FD013596E491EA934FDA51
:107AFC00E132E1F017C0E430A9F40E94926C0E94CC
:107B0C00E77432960E94957BE0935A0CF0935B0CD1
:107B1C000E949D720E94E7743596E491EA934EDBC5
:107B2C00E13221F00E940B180F5F40CF099119919F
:107B3C000895E8810E940773EAEDF7E10E94786DE1
:107B4C000C941C421A930E94E57210E0133010F052
:107B5C000C94013E0E940F6C0E940F6C0E94B26D3F
:107B6C001A93E7DFECE0F0E00E94506C0E94A44610
:107B7C001A939FDB0E94B4740E94B87451F40E9453
:107B8C00EA710E94C274E2E00E94C67409F4FFC25A
:107B9C0009C00E94EA710E94C274E0E00E94C6749F
:107BAC0009F4F5C2123028F50E940F6C0E940F6C7C
:107BBC000E94B26D1A93BDDFE9E5F8E10E94786D81
:107BCC00ECE0F0E00E94506C0E94A4460E94D77436
:107BDC00EAE0F0E00E94506C0E94A446A0EBBBE0EF
:107BEC000E9432710E94206DE3E60E94AF7409F48A
:107BFC00CEC21F5FABCFCBC20E946A7D10E01A933E
:107C0C000E947D730E94CB740E940F6C0E94A4464C
:107C1C000E94EA6D0E94CF740E946B6D21E000E01F
:107C2C00033080F5E3E0F0E00E94C16C0E94DA6D55
:107C3C000A937FDF0E94257249F40E942D720E94E4
:107C4C00CC6D0E94D16D0E94D37408C00E942D721D
:107C5C000E94CC6D0E94867B0E94C56D0A9329DB25
:107C6C002F5F023068F4E7E0F0E00E94C16C0E94E4
:107C7C00DA6D0E9430720E94EF6D0E94D7742F5FF4
:107C8C000F5FCECF0E9406433E2F3B3211F41034CF
:107C9C0008F001C01F5F3D3211F4113008F401C02F
:107CAC0011503D3439F41A930E94CF184BDF1A93BC
:107CBC000E94EF18313209F0A2CF0E94717D2496F8
:107CCC0008950E94E5720E940F6C0E940F6C0E9436
:107CDC00A446EFE5F8E10E94786DE1E0E09322081C
:107CEC00E2E2F8E0FA93EA93E5E0EA9397D9089593
:107CFC0022970E94687D0E9406430E2FE0911B087C
:107D0C00E03011F00C942F400132D1F4EAE4F6E0AB
:107D1C00A0913A0CB0913B0CEA17FB0761F4E7E039
:107D2C00E0931808EAE2EA93E8E6F8E10E9446706C
:107D3C000E94BB63A8C0E0E0E093C0050E94EC7415
:107D4C000D3331F4E091C005F0E00E94B06C049169
:107D5C000D3441F4EAE2EA93EBE6F8E10E94467056
:107D6C000E94BB63063449F4E2E7F6E0E0933A0C78
:107D7C00F0933B0CE0E0E093C005003311F00B32C4
:107D8C0029F4E091C005EF5FE093C0050D3229F4B2
:107D9C00E091C005E150E093C005013329F491DF77
:107DAC00ED3311F40E94F374033321F48ADFED33C5
:107DBC0009F40CD8063329F4E0E0E09322080E9481
:107DCC00EC36043329F4E0E0E09322080E94F374CB
:107DDC00A0912408A13010F40C94C53F023301F596
:107DEC0070DFED33E9F40E940075D1F4E0912208C4
:107DFC00EA930E941F1B30E0303190F40E94AA6C71
:107E0C000E94177059F4E32FE05DEA93EEE6F8E177
:107E1C000E941C70E0E3EA930E94DD633F5FECCFAD
:107E2C00053331F5E0E0E09322080E94007501F57E
:107E3C0011E01630E8F41A930E941F1B30E0303129
:107E4C00A8F40E94AA6C0E94177071F4E32FE05DF5
:107E5C00EA93EEE6F8E1FA93EA93E12FE05DEA9318
:107E6C00E0E3EA930E94DD633F5FE9CF1F5FE1CF60
:107E7C00013469F4EAE2EA93E1E7F8E10E94CD7398
:107E8C00E1E0E09318080E946F7D289608950A346B
:107E9C0009F4B2DE073311F00C94C53F0E94CB46B7
:107EAC00E0E0EA930E94E60DE1E0E0931C08E0E0DC
:107EBC00F0E0E0931408F0931508EFE2F6E00E946E
:107ECC004670E3E7F0E00E94F86F0E941768EE83BB
:107EDC00FF830E940975E8E2F0E00E94AE70B9F0F1
:107EEC000E9438120E941768EE83FF83A091190C30
:107EFC00A03021F00E94A633E03009F408C00E94A3
:107F0C00F473E652F84FAEE0A0830E94DA71E5E01C
:107F1C00F0E00E942C6C40E050E00E949A21E03886
:107F2C0068F00E949A21EF573E2F313010F031311A
:107F3C0008F004C0E32F0E940771AF015A934A93D3
:107F4C000E94591F40931408509315080091DB05AB
:107F5C00E0E0E093DB05013211F00B3209F401C0D3
:107F6C00B8CF0B3221F4E1E0EA930E94E60D013226
:107F7C0009F0A3CFE0E0E0931C08E093DB05A091AF
:107F8C002408A23011F00C942840093309F407DDC1
:107F9C00053409F494DC033611F40E94290D0833DE
:107FAC0009F45EDB023409F409DC0334B1F51091F9
:107FBC00390C0E94CB4600E0E091380CE11711F02F
:107FCC000C3008F01DC00E940F6C0E94926C0E9435
:107FDC00DA6D1A930E94AD1E1A937CD10E94B66D75
:107FEC00E091290C0E94E074E0912C0C0E94E0744A
:107FFC000E94BE700E94C56D0E94A4700395DCCFD8
:10800C000E94B50D0E9406430E2F013221F0E09123
:10801C00380CE11709F401C0CCCF043499F40E9458
:10802C00007581F4A091D30BA03021F4A091D10B59
:10803C00A03031F00E9451730E940F6C0E942E539D
:10804C000E94FB1CE0911B08E03011F40E943E0ED4
:10805C0049C0E130D1F4A0912108AB3010F40132C9
:10806C0009F405C00E94C9150E94B50D0DC0E0E0D1
:10807C00E0931E080E940E750E94CD73E0E00E94F2
:10808C001375E2E0E0931B082DC0E23059F5013284
:10809C0069F4E0E0E0931B080E94CB46EAE2EA9325
:1080AC00EBE6F8E10E94CD730E943E0E0B3211F00C
:1080BC000D3359F40E940E75FA93EA93E1E3EA93B7
:1080CC000E94BB63E1E00E9413750D3259F40E94CB
:1080DC000E75FA93EA93E2E3EA930E94BB63E2E043
:1080EC000E941375A0911808A33009F404CE0E94C5
:1080FC006F7D0C9475451A93E3E0E09319080E9488
:10810C00CB460E940F6C0E940F6C0E94A446E7E7BE
:10811C00F8E10E94786D0E940F6C0E94736D0E94B2
:10812C00A446E3E1F6E00E944670E0E1F0E00E9434
:10813C00F86F10E0E091C90B1E1700F50E94DE6D80
:10814C00E117D1F0E12FE05DEA93EFE7F8E1FA9364
:10815C00EA93E0E3EA93E0E00E94237049F40E9482
:10816C003271ED5EF94FA1E0A083E12FE05D01C01B
:10817C00EEE2EA930E9442461F5FDCCF0E94EC7451
:10818C00E0E0E093C005E0931B080E943E0E1991BD
:10819C000895E881E03021F4E4EFF6E00E941875D0
:1081AC00A881A13021F4EEEEF6E00E941875A881AA
:1081BC00A23021F4EAEFF6E00E941875A881A330F2
:1081CC0021F4E8E0F7E00E941875A881A43021F4AE
:1081DC00EEE0F7E00E94187529C11A930A93E0E0CB
:1081EC00E0937D05E0937E0510E0143190F400E0FF
:1081FC00033068F4A3E01A9FF001EC57FA4FDF014B
:10820C00EE27A00FBE1FE0E2EC930F5FF1CF1F5FD4
:10821C00ECCFECC31A9311E0E981E11780F00E94D6
:10822C003271E255FF4FE491AA81EA2319F0E12F54
:10823C00E05D01C0E0E2EA931FD51F5FEDCF30C5D2
:10824C001A9311E0E981E11778F00E943271E2553E
:10825C00FF4FE491AA81EA2311F0E1E301C0E0E3CE
:10826C00EA930AD51F5FEECF1BC52A97A0911B0C72
:10827C00A13038F0EA85FB856C857D850E94D3742E
:10828C0007C00E941D750E9421750E941D75FCD4AB
:10829C0026C12A970E941D750E942A750E9433756B
:1082AC000E941D75F1D41BC12A970E941D750E9456
:1082BC0046750E944D75E8D41FC12A970E941D7502
:1082CC00EDE9F8E10E9452750E94D8730E944D7539
:1082DC00DBD412C12A970E941D75E0EAF8E105C0B3
:1082EC002A970E941D75E4EAF8E1FA93EA93EE8569
:1082FC000E946A6C0E941D75C7D42B9608950E942B
:10830C006A7D10E0E1E3E0933809E89431F8EA93F0
:10831C000E946363E8EAF8E10E94BD7200E0E0911C
:10832C0082050E17E0F40E94926CEC57FA4FE08134
:10833C00E03258F4E3E2EA930E94A5620E94926C48
:10834C00EC57FA4FE081E05D05C00E94926CEC574F
:10835C00FA4FE081EA930E94A5620F5FE0CF0E9482
:10836C0057759F010E943B153A932A93E8ECF0E075
:10837C00FA93EA930E9423680E2FA0E031FCA1E04F
:10838C00A03011F4003009F001C0ECCF31FE09C06F
:10839C00E0E0E0938205E89431F8E1E00E94717D21
:1083AC00F2C41F5F123008F4ADCFE0E0E093820519
:1083BC000E94717DE8C4E0918105E03021F4E881F0
:1083CC00EA930E94505EA0918105A13069F4A0E06F
:1083DC009299A1E0A13021F4A8950E94E06EF7CF0C
:1083EC00E881EA930E94F060A0918105A230F1F43B
:1083FC00E0918205F0E0EC57FA4FA881A083E09160
:10840C008205EF5FE0938205E0918305EF5FE093D7
:10841C008305A03218F4EF5FE0938305A0918305E8
:10842C00A83320F06CDFE0E0E093830521960895FB
:10843C0008950E9468740E94687422D0EBE1EA935C
:10844C00BADFE9E6EA93B7DFA0918105A13061F4C8
:10845C00E8ECF0E00E944B6EE0919A00E069E0934A
:10846C009A00E9E1E0939900A0918105A23021F4F2
:10847C0046DFE0E0E0938305E0E0E09381050895BA
:10848C00EDE0EA9398DFEAE0EA9395DF08951A931A
:10849C0010E0E9811E1728F4EA81EA938CDF1F5F54
:1084AC00F8CFFEC3EDE201C0EDE3EA93E8E2EA9314
:1084BC00EEDFE6DF08952A97A0911B0CA13038F06F
:1084CC000E941D750E942A750E94337504C00E947B
:1084DC001D750E942175FE010E9446700FD02E96CC
:1084EC0008952A970E941D750E9446750E945B751F
:1084FC00FE010E94467002D02C9608951A930A939E
:10850C0010E0EA81E03011F408E201C00A81AB818D
:10851C00BC81EE27A10FBE1FAC91A03011F010173B
:10852C0008F007C0AB81BC810E9460750E94657524
:10853C00EECFEA81E03039F0EA811E1720F4E0E258
:10854C000E946575F9CF27C01A930A9310E0EA814F
:10855C00E03011F408E201C00A81E12FAB81BC814B
:10856C000E949974E491E03011F0101708F009C0E2
:10857C00E12FAB81BC810E949974E4910E946575D6
:10858C00ECCFEA81E03039F0EA811E1720F4E0E20A
:10859C000E946575F9CF1981088125960895E0919F
:1085AC00C405A091C305EA17B1F00E946A750E9438
:1085BC00CC6DEC91E093C6050E946A750E944C71DB
:1085CC00E181E093C505A091C4050E947075E0930C
:1085DC00C405E1E00895E0E008950E947575A98155
:1085EC00A0830E9475753196A881A083A091C305C4
:1085FC000E947075E093C305C2C0E091DB0508953D
:10860C001A93E091DB05E03059F40E943B150E946F
:10861C00E07121F4A091DB05A03009F001C0F5CF89
:10862C001091DB05E0E0E093DB050E94E07109F0BE
:10863C0011E2E12FD9C30E946A7D0E9417688F0155
:10864C000E943B15EC81FD81E00FF11FFF93EF932E
:10865C000E941768AF91BF91AE1BBF0B9D01002408
:10866C00021603061CF40E94E07109F001C0E8CF69
:10867C00E0E00E94717D269608951A93E9810E948C
:10868C0049720E947B75E05FFC4F108117FF05C09B
:10869C00E12F0E948275A0E0A08316FF05C0E12F98
:1086AC000E948975A0E0A083E981ADE0EA9FF0010A
:1086BC00E05FFC4F0E947B75E15FFC4FA0E0A08364
:1086CC0018815DC00E946A7D30E0EE81ADE0EA9FCA
:1086DC00F001E05FFC4F108116FF17C0E12FEF7324
:1086EC000E2F0E94907511F03A3008F009C00E94CC
:1086FC009875DF010E94AA6C0E949E753F5FF1CFB6
:10870C000E9498750E948C74EC9317FF17C0E12F90
:10871C00EF730E2F0E94907511F0343108F009C0E0
:10872C000E94A475DF010E94AA6C0E949E753F5F97
:10873C00F1CF0E94A4750E948C74EC930E94717D01
:10874C0042C2E881F9810E947C6DEA81FB813296FC
:10875C000E947C6DEC81FD8134960E947C6DEE81D3
:10876C00FF8136960E947C6DE885F9853896E491F8
:10877C00EA93E985FA8539960E948F6C02D022968D
:10878C000895A0970E94687DEDA5FEA5A9A9BAA998
:10879C00EA0FFB1FAF01E5E0F3E0EE83FF8310E08F
:1087AC001431C0F5AE81BF81AC91A03049F1EE819E
:1087BC00FF81A381B481EFA5F8A9EA17FB0701F5A6
:1087CC00EE81FF81A181B281E9A9FAA9AE17BF0799
:1087DC00BCF0EE81FF81A181B2814A175B0784F066
:1087EC000E94AA75AE0FBF1FE9A9FAA9AE17BF0761
:1087FC003CF00E94AA75AE0FBF1F4A175B070CF422
:10880C0002C01A933ADFEE81FF813D96EE83FF831F
:10881C001F5FC6CFE5E0F3E0EE83FF8310E0143179
:10882C0010F00C94BC44AE81BF81EC91E03011F09F
:10883C000C94B544EAA5EC93E9A9FAA9AE81BF81E1
:10884C001196ED93FC93EFA5F8A9AE81BF81139619
:10885C00ED93FC93EDA5FEA5AE81BF811596ED932E
:10886C00FC93EBA5AE81BF811796EC93E0910904C4
:10887C00A0910F04EA27AE81BF811896EC93E0918A
:10888C001004AE81BF811996EC93E0911104AE8176
:10889C00BF811A96EC93AE81BF811B960E942D6D01
:1088AC001C96E0E0EC93E887E8A5F9A5309741F039
:1088BC000E94B5750E94BA75E4E1EA930E940269C0
:1088CC00EEA1FFA1309751F00E94B575E8A5F9A56E
:1088DC00FA93EA93E4E1EA930E94EE68E0E0EC8F0D
:1088EC000E94B5750E94D9683E2F3B30C8F000E05D
:1088FC000E94A475E081E03011F0053008F002C050
:10890C000F5FF6CF0E94A475E081E03049F40E941D
:10891C00A4750E94BF75E058AE81BF811B96EC9385
:10892C00E0E0EA8B3130C8F000E00E949875E081FD
:10893C00E03011F0043108F002C00F5FF6CF0E9456
:10894C009875E081E03049F40E9498750E94BF75DB
:10895C00E05CAE81BF811B96EC93E12F08C0EE81E9
:10896C00FF813D96EE83FF831F5F59CFEFEF0E948F
:10897C006F7DE39608951A930A930E94CA753097F7
:10898C00A9F1E0916205E03061F50E94CA7504908E
:10899C0000926205E0916205E03031F4E0E0F0E035
:1089AC000E941875E0E01AC00E94CF750E94CA752B
:1089BC000E94957BF595E7958F01D801E0E0F1E0F9
:1089CC000E940D7BE0938700D801E0E0F1E00E946B
:1089DC003F7BE09386000E94CF75E0E4E0938B0030
:1089EC0005C0E0916205E150E0936205099119918F
:1089FC0008950E946A7D00E025E033E010E0143118
:108A0C00B8F5D901EC91E03079F111960E94867B92
:108A1C000E94D77524F5D90113960E94867BAC81F0
:108A2C00BD81EA17FB07DCF4F90101801280D90142
:108A3C0015960E94867BE00DF11DAE81BF81AE17AD
:108A4C00BF076CF4F90103801480D9011796EC91DF
:108A5C000E94E671AC81BD81AE17BF070CF004C05B
:108A6C00E12FEF5F0E2F04C0235F3F4F1F5FC7CF77
:108A7C00003049F0E0916305E01721F0A091630507
:108A8C00A03009F401C022C0A0916405A53079F48E
:108A9C000A93E1E0EA93A1DD009363050093650579
:108AAC00D901EC91E0936605E3E0E0936105A091B8
:108ABC006405AE3119F4E4E0E0936105A091610521
:108ACC00A33018F0E5E0E093680507C0E0E0E09320
:108ADC006405E09361050E94DC750E94717D289607
:108AEC000895E0916305E03091F0A0916405A932FE
:108AFC0020F4EA93E2E0EA9370DDA0916405AD33D3
:108B0C0030F0E0916305EA93E4E0EA9366DDE0E09F
:108B1C00E0936105E09364050E94DC75E0E0E0936E
:108B2C006305E0936705089530D157DB0895EA811A
:108B3C00E0937F05E881E0938005E0910A04E06111
:108B4C00E0930A0420C10E94687DA0917F05A431A6
:108B5C0020F4A0918005A33008F033C0E0917F058C
:108B6C00F0E0ACE0B0E00E94E27A8F01E091800589
:108B7C00F0E0A4E1B0E00E94E27A9F010E94E2756D
:108B8C00ECE0F0E00E94E775F0E00E94957A0E941C
:108B9C00356CEE81E030A9F0E0917F05A3E0EA9F0F
:108BAC00F001EC57FA4FDF01E09180050E94BD6F98
:108BBC004C9155270E94E2754A93EFE0EA930E948C
:108BCC00624D0E946F7D27960895E0910A04E07132
:108BDC0041F0E2E0EA93B7DFE0910A04EF7EE09324
:108BEC000A0408950E94EC75AF3EE0E0BE0744F421
:108BFC00A0910203B0910303AF33E1E0BE070CF088
:108C0C0039C00E94F1750E94CF6F0E94624DA091F5
:108C1C005D05B0915E05549734F4A0915F05B09159
:108C2C00600513970CF012C0E0915D05F0915E05A4
:108C3C00A3E0B0E00E94BA7AEC57FA4FA0915F051E
:108C4C00B0916005EA0FFB1FA981A083E0910D0490
:108C5C00ACE0EA9FF0010E94EC750E9499740E94AE
:108C6C00FE75E0915D05F0915E053196E0935D0532
:108C7C00F0935E050C94A74AE881EA93E091100406
:108C8C00EA93B0DF0C94764A1A9310E00E940376B4
:108C9C00E03031F00E940376EA93EEDF1F5FF6CFEF
:108CAC001881239608950E9406760E940B76E03078
:108CBC0021F00832E0E01E070CF007C00E940B7692
:108CCC00EA93DADF0F5F1F4FF0CF198108815BC089
:108CDC000E940676F801AB81BC810E94127621F0CD
:108CEC00EA810E9417760CF009C0F801AB81BC81B7
:108CFC000E941C76C1DF0F5F1F4FECCF19810881DA
:108D0C000EC30E946A7D0E94EC750E9421763197F9
:108D1C008F010E9426760E94E2750E942E7633C047
:108D2C000E946A7DAC810E9435760E2F11270E941D
:108D3C0026760E94E2750E942E76F1C2EA81FB81B2
:108D4C00E0935D05F0935E05E881F981E0935F05A2
:108D5C00F0936005AA81BB81ECE0F0E00E94E27A1E
:108D6C000E94FE75A881B981E4E1F0E00E94E27AEC
:108D7C0006C0EA81FB810E94FE75E881F981E093CF
:108D8C000203F0930303249608950E943D76143158
:108D9C0020F41A9372DC1F5FFACF0E940F6C0E94B2
:108DAC000F6C0E94306CEFE3F1E00E94356C10E028
:108DBC00153048F4A5E11A9FF001E051FB4FA0E0FB
:108DCC00A0831F5FF5CF10E0143148F4ABE01A9F7D
:108DDC00F001EC5EFB4FA0E0A0831F5FF5CFE091AC
:108DEC000A04EF7EE0930A04199108950E943D76DF
:108DFC00143100F5ADE01A9FF001BF01E85FFC4FA4
:108E0C00DF010E94867B0F01DF01EB81FC81AE1735
:108E1C00BF075CF0E981FA81E015F10534F0FB0144
:108E2C00E05FFC4FE081E03009F402C01A9325DCCE
:108E3C001F5FDECF0E940F6C0E9445760E94306C43
:108E4C00A985BA850E944A760E94356C67C2A297A2
:108E5C000E94687DE9A50E9449728F01D8011B967A
:108E6C00EC91E03009F415C2D8011B96EC91E9A302
:108E7C00E07859F0FE013696FA93EA93EBA10E9442
:108E8C008275FA93EA930E94C368E9A1E07459F0E1
:108E9C00FE013696FA93EA93EBA10E948975FA9338
:108EAC00EA930E94C368FE013696FA93EA930E94F5
:108EBC00D968E8A3E0910D04EB8FE0910E04EA8FE2
:108ECC000E94996ED80111962D913C91D801139660
:108EDC004D915C91D80115960E94867BEEA3FFA361
:108EEC00D8011796EC91F0E0ECA3FDA3D8011896ED
:108EFC00EC91EC8FE0910E04A0E10E94EF6BEAA3E1
:108F0C00FBA30E944F760E94BA750E94BA75ECA121
:108F1C00EA930E94BA4BD8011996EC91EC8FE03091
:108F2C0011F4E8E0EC8F0E944F760E9454765A932D
:108F3C004A930E945B760E945F760E9466760E943E
:108F4C0069760E944F763A932A930E946976EEA135
:108F5C00FFA10E9470765A934A930E9454760E9405
:108F6C006976A8A5A130B1F43A932A93FA01319607
:108F7C000E946676FA013196FA93EA930E945B7628
:108F8C00F90131960E947576F9013196FA93EA93BC
:108F9C000E946976A8A5A230F1F40E945F76319701
:108FAC000E946676EAA5FBA5E40FF51F3197FA93AC
:108FBC00EA930E945B76EEA1FFA1E20FF31F3197BB
:108FCC000E947576EAA5FBA5E20FF31F3197FA9381
:108FDC00EA930E946976E8A5E03011F40C941F49DD
:108FEC00D8011996EC91EC8FE0910D04ACE00E9445
:108FFC007A760E940D7BED8FA8A1EA1710F40C94E1
:10900C004E48E1E0E0930E04E03021F0ECA1FDA12C
:10901C00B5970CF402C00E948076AAA1BBA1ECA16A
:10902C00FDA1EA1BFB0BDF010E943571EAA3FBA338
:10903C00ABA1AA231AF4E0E0EAA3EBA3A8A10E9437
:10904C003576AEA1BFA1F0E00E948876EE8FA8A580
:10905C00A13021F40E948B760E948E76A8A5A230B6
:10906C0031F40E948B760E9470760E949A76E0E032
:10907C00E9A30E94A076AE0FBF1FEC91E03039F04F
:10908C000E94A0760E941C760E94A576F2CFD1C0D9
:10909C00E1E0E0930E04E03031F0ECA1FDA1E73407
:1090AC00A0E0FA070CF402C00E948076E8A1EF8FD2
:1090BC00EAA1FBA1EE0FFF1FACA1BDA1AE1BBF0B24
:1090CC00E3E0F0E00E940D7BEAA3FBA3ABA1AA2393
:1090DC0022F4E1E0F0E0EAA3FBA3EF8DE150EF8F87
:1090EC00EF8DF0E0DE011696AE0FBF1FAC91A032F3
:1090FC0019F0AF8DA13008F404C0EF8DE150EF8F63
:10910C00EFCFAF8D0E943576AE2FEEA1FFA1B0E070
:10911C00EA17FB0714F3EF8DE03011F4ED8DEF8FB0
:10912C00AF8DECE00E947A760E948876EE8FA8A52F
:10913C00A13021F40E948B760E948E76A8A5A230D5
:10914C0031F40E948B760E9470760E949A76E0E051
:10915C00E9A30E94A0760E94127621F0EF8DA9A1BE
:10916C00AE1708F007C00E94A0760E941C760E94E1
:10917C00A576EFCFAF8DE8A1EA1BAE2FED8DEA17E8
:10918C0068F0AF8DE8A1EA1BACE0EA9FF001A0917A
:10919C000D040E947A760E94887601C0E0E0EE8F82
:1091AC00A8A5A130A1F40E948B76E20FF31F319693
:1091BC000E94E775AFE00E94EF6BE40FF51FDF0133
:1091CC00ECA1FDA10E944C7131960E94476EA8A59E
:1091DC00A23089F40E948B76E20FF31F0E94E77590
:1091EC00AFE00E94EF6BE40FF51FDF01ECA1FDA1D6
:1091FC000E94C274BEDD0E94A076AE0FBF1FAC9160
:10920C00A03219F4E9A1EF5FE9A30E94A0760E94B5
:10921C00127639F0AF8DE9A1EA1BAE2FED8DEA176E
:10922C0008F407C00E94A0760E941C760E94A576C6
:10923C00ECCFD8011C96EC91E03029F10E94996E8C
:10924C000E944F7696DDF801A485A43698F4EFE0E1
:10925C00E0931004F801A485AA3028F0A485AA9301
:10926C000E94704106C0D8011C96EC91E05DEA9317
:10927C0003DD09C0ECE0E0931004E2E5EA93FCDCCA
:10928C00EDE4EA93F9DCEB8DE0930D04EA8DE093C9
:10929C000E040E946F7DAA9608951A9310E0E8942C
:1092AC0027F8143170F40E94766EE03011F00E94B1
:1092BC007D6E1F5FA895E12FE37011F40E943215AB
:1092CC00F0CFEFE0E09310040E9432150C94FD4DAA
:1092DC001A9310E01431F8F40E94826EB1F0A85F7A
:1092EC00BC4F0E94867BDF01EB81FC81EA17FB07F8
:1092FC0064F4F001E85FFC4FDF010E94867BDF0124
:10930C00E981FA81AE17BF070CF002C00E947D6E96
:10931C001F5FA895DFCFEFE0E0931004188125962E
:10932C0008951A9310E0143190F40E94826E31F07B
:10933C00FD01E15FFC4FE081E17009F406C01A9376
:10934C00E0910A04E170EA9382DD1F5FECCF0C948C
:10935C00FD4D2C970E94687DAD89BE890E943571A8
:10936C000E94AD76EB8BFC8BED89FE890E94B27668
:10937C00EB89FC89E017F107FCF00E94E5762E2FB3
:10938C0033270E9409770E9410770E9417770E945A
:10939C001C770E940977F801A98DBA8D0E94206D67
:1093AC000E941777F8010E942677EA8DEA930E94B3
:1093BC001D4C0F5F1F4FDCCF48C02C970E94687D5F
:1093CC00AD89BE89E4E0F0E00E940D7B0E94AD7691
:1093DC00EB8BFC8BED89FE89EE0FFF1F0E94B276A2
:1093EC00EB89FC89E017F10784F10E94E576AE2F3A
:1093FC00ED89FE89B0E0EA0FFB1F9F010E940977FF
:10940C000E941077E98DFA8DEE0FFF1F0E942677D0
:10941C000E941C77ED89FE89EE0FFF1FA98DBA8D76
:10942C00AE1BBF0BBA93AA93F801A98DBA8D0E94FB
:10943C00206D0E941777F8010E942677EA8DEA9337
:10944C000E941D4C0F5F1F4FCBCF0E946F7D6B9600
:10945C000895EA81F0E0EBBBF5BBF7E1F093650012
:10946C001F98E6E1E0936500F09365001F9AE88190
:10947C00F981EBBBF5BB1F98FFE1F0936500EEE1C2
:10948C00E0936500F09365001F9A0C94704EE2E235
:10949C00EBBBE0E0E5BBE7E1E09365001F98E6E19C
:1094AC00E0936500E7E1E093650008951F9A089545
:1094BC00A0910403A23021F4E881A8E4B3E10BC02D
:1094CC00A0910403A43021F4E881A8E4B3E103C023
:1094DC00E881A8E2B3E1F0E00E944C710E94957B18
:1094EC0021960895E0910403E23011F4EEE40AC0F1
:1094FC00E43039F4E0E2EA93A981BA810E94217642
:10950C0004C0E0E2EA93E981FA81FA93EA930E94BB
:10951C002F4A17C0E0910403E23011F4EFE40AC0C3
:10952C00E43039F4E1E2EA93A981BA810E942A7706
:10953C0004C0E1E2EA93E981FA81FA93EA930E948A
:10954C002F4A22960895E0910403E230B9F4E4E442
:10955C00EA930E942F77AE0FBF1FFD01FE2FE0E0B4
:10956C00AF81B8850E94206D0E942F4AE5E4EA93F2
:10957C000E9445760E942F4AE6E453C0E33089F4FA
:10958C00E7E3EA93FF81E0E00F010E942F77EA0FF7
:10959C00FB1F0E9434770E9445760E942F4AE6E317
:1095AC0040C0E43049F5E7E3EA93AF81B8850E9407
:1095BC002176DF01EB81FC81AE1BBF0BFD01FE2F81
:1095CC00E0E00F01AF81B8850E9421760E943477CC
:1095DC00AD81BE810E942A77DF01E981FA81AE1B41
:1095EC00BF0BBA93AA930E942F4AE6E3EA93AD818C
:1095FC00BE810E942A771CC0E0E5EA930E94947415
:10960C000E942F4AE1E5EA930E942F770E94206D79
:10961C000E942F4AE2E5EA930E9445760E942F4A67
:10962C00E3E5EA93E981FA81AD81BE81EA0FFB1F84
:10963C00FA93EA930E942F4A28960895E091040326
:10964C00E33029F4E3E0EA93E0E1F1E00BC0E4302D
:10965C0029F4E3E0EA93E0E2F1E004C0E3E0EA930A
:10966C00E0E3F0E1FA93EA930E942F4A0895E09127
:10967C000403E33029F4E3E0EA93E1E2F1E00BC008
:10968C00E43029F4E3E0EA93E1E1F1E004C0E3E043
:10969C00EA93E8E3F0E1FA93EA930E942F4A0895E3
:1096AC001A930A93EFE10E943D77EBE10E943D771C
:1096BC00EFE10E943D77E8EFFFEFE0935C0CF09355
:1096CC005D0CE491EF3F39F0E0915C0CF0915D0C96
:1096DC00049000920403E6ECF3E18F01A0910403E3
:1096EC00A23019F4E8EAF3E18F01A0910403A4304D
:1096FC0019F4E8E6F3E18F01F801E491ED3F39F458
:10970C00F80131960E947C6D0E94677A19C0EE3F79
:10971C0071F4F80131960E94957BDF01E09104030E
:10972C00F0E0EA17FB0711F00D5F1F4F09C0F801BD
:10973C00E491EA93F80131960E947C6D0E942F4AC5
:10974C000D5F1F4FF801E491EF3FB1F60E94086CDA
:10975C00E1E0E0930E04E0930D04E4E1E0931304E4
:10976C006DDF0991199108950E944177AE85AA2366
:10977C0062F0AD85BE85A03FE0E0BE0734F4AB855A
:10978C00BC85AF33E1E0BE070CF050C00E944977B6
:10979C00AE0FBF1FA03FE0E0BE0734F0AD85BE8525
:1097AC000E942176E987FA87EF81F885AB85BC8525
:1097BC00AE0FBF1FA034E1E0BE0734F0AB85BC8513
:1097CC000E942A77EF83F8870E94876D0E94876D2D
:1097DC000E94876D0E94876DB6DE0E94876D0E9485
:1097EC004E77498554DE0BBB15BB2EE13FE100E003
:1097FC0010E0EF81F885E017F10764F050E04517B1
:10980C0030F020936500309365005F5FF8CF0F5FF9
:10981C001F4FEFCF4BDE0E940F6C0E940F6C0E940B
:10982C00306CEFE3F1E0FA93EA938DDEC9C00E944D
:10983C0041770E944977EA17FB0741F0EF81F885E1
:10984C00AB85BC85EA17FB0709F03EC00E94567732
:10985C001CF00E945D7784F42D853E85ED85FE8598
:10986C00E987FA872D873E872B853C85EB85FC8520
:10987C00EF83F8872B873C870E94876D0E944E7779
:10988C000E944977EA17FB0749F4F1DEEB85FC856A
:10989C00ED87FE87EF81F885E987FA87F8DD0BBB4A
:1098AC0015BB2EE13FE10D851E85E985FA85E01794
:1098BC00F1073CF020936500309365000F5F1F4F5C
:1098CC00F4CFF4DDBBDE7CC000930B0410930C04CE
:1098DC000E9464770E946B77FF93EF930E946F77DF
:1098EC000E946B77AF91BF91EA17FB0780F10E9442
:1098FC005D77B4F420E030E00E947277E217F30752
:10990C0074F00E9464770E9479770E9472770E94AB
:10991C007E770E94877758D02F5F3F4FEDCF16C0D0
:10992C0020E030E00E946F77E217F3077CF00E9492
:10993C0064770E9479770E946F770E947E77F90195
:10994C000E948E7741D02F5F3F4FECCF39C00E94E1
:10995C005677DCF420E030E00E949277E217F307B0
:10996C009CF00E946F770E9479770E949277D001C9
:10997C000E940D7BAF010E948777FA010E948E77BF
:10998C0023D02F5F3F4FE8CF1BC020E030E00E9478
:10999C006477E217F307A4F00E946F770E9479773F
:1099AC000E946477D0010E940D7BAF01F9010E94E7
:1099BC008E77FA010E948E7707D02F5F3F4FE7CF4B
:1099CC000E946F7D2F960895EA81FB81FA93EA93AA
:1099DC0089DD0E9499779EDDE2E2EA93E0910B0427
:1099EC00F0910C04FA93EA930E942F4A249608955E
:1099FC000E94687D00910D0410E0E0910E041E178A
:109A0C0010F00C94614DE885F985FA93EA9382DDA8
:109A1C002C853D854A855B85022E032A11F40C9416
:109A2C00594D37FF36C05A934A935CDDE2E2EBBBEB
:109A3C00E0E0E5BBE7E1E09365001F98F6E1F09309
:109A4C006500E0936500EE81EBBBEF81E5BBEFE1D8
:109A5C00FEE1E0936500F0936500E093650001FF83
:109A6C0004C0F0936500E093650036FF11C0F093DD
:109A7C006500E093650001FF06C0F0936500E0937C
:109A8C0065004F5F5F4F220F331F4F5F5F4FEDCF6E
:109A9C001F9A220F331F01FF02C04F5F5F4F4F5FB2
:109AAC005F4F0C94124DE885F9853196E887F9875C
:109ABC001F5F0C94034D38C022970E94687DE88587
:109ACC00EA930E945E4AEE83FF83E985A8E1EA9F50
:109ADC00F001E85DF84F8F0130E0383028F5F801DF
:109AEC00E4915E2F0F5F1F4FF801E4914E2F407FE2
:109AFC000E949E770E94A377EA87FB87F801E49186
:109B0C004E2F440F440F440F440F0F5F1F4FF801AB
:109B1C00E4915E2F0F5F1F4F0E949E770E94A377E8
:109B2C00EA87FB873F5FD9CF0E946F7D2E96089501
:109B3C0024970E94687DEA85EA930E945E4AEE8330
:109B4C00FF8300E010E0EB850E941776C4F5EF85EB
:109B5C00F889E887F98720E030E0EC850E94B0773F
:109B6C001CF5E989FA89449155273196E98BFA8BD2
:109B7C005A934A930E94FD6CE989FA89FA93EA9305
:109B8C00EC85FD85FA93EA930E94FE4CE0910D045E
:109B9C00EE0FEE0FEE0FA885B9850E949974E88739
:109BAC00F9872F5F3F4FD9CFE0910E04AD85BE856D
:109BBC000E949974ED87FE870F5F1F4FC4CF0E94E0
:109BCC006F7D639608951A93EFEF0E940D72E093E8
:109BDC00390910E00E943271E05CF54FE081EF3FF3
:109BEC0031F00E9432710E94B5771F5FF3CF19914B
:109BFC0008951A930A930091CF0BAA81A53411F4FE
:109C0C00E0E066C0AA81A23539F4A0913508A130F4
:109C1C0019F40E94B87709F405C00E94531CE0E0C7
:109C2C00E0933508AA81AB3411F0A33599F4E02FF9
:109C3C00E470E43011F414E001C013E0E02FE270A2
:109C4C00E23009F41C5FE02FE170E13009F41F5F92
:109C5C00E12F3EC0AA81A13511F0A13799F4E02F74
:109C6C00E470E43011F417E001C016E0E02FE2706C
:109C7C00E23009F41C5FE02FE170E13009F41F5F62
:109C8C00E12F26C0AA81A33421F0A13411F0A23413
:109C9C0041F413E0E02FE170E13009F41F5FE12F94
:109CAC0017C0AA81A73741F417E0E02FE170E1302B
:109CBC0009F41F5FE12F0CC0AA81A03441F415E018
:109CCC00E02FE170E13009F41F5FE12F01C0EFEFED
:109CDC00198108812396089524970E94687D20910C
:109CEC00CF0BA0914009A53411F00C943C4FE0E04F
:109CFC00E09335080E940672E0E0E0935D0BE09182
:109D0C00D30BE03089F5E0911008A0911108EA1707
:109D1C0039F00E94BE77ED55F84FE081E13009F043
:109D2C0023C0E7E7EA930E94A5620E94BE77E8553C
:109D3C00F84F0E945171FA93EA930E94C477EC5544
:109D4C00F84FDF010E94BF730E94C477E755F84FAC
:109D5C000E94C977E2E0E09335080E94BE77ED558A
:109D6C00F84FA2E0A0832FDFE0913508E03011F02E
:109D7C000C943C4F0E94B87711F40C94164F0E942F
:109D8C00481CE1E0E0933508E22FE870E83081F4FC
:109D9C000E94CE77E8EEF3E00E940D7BDF010E947B
:109DAC005E7D14F4E1E301C0E0E3EA930E94A56256
:109DBC00E22FE074E03411F413E001C012E0E09102
:109DCC00240C0E9451741A930E940263E22FE470D7
:109DDC00E43049F40E94CE77E0E1F7E20E943F7B49
:109DEC00AF0114E006C00E94CE770E944473AF010D
:109DFC0013E0E22FE071E03111F4415050405A93DE
:109E0C004A931A930E940263E22FE072E03211F43B
:109E1C0014E001C013E0E091270CF091280C17C05E
:109E2C0018E0E22FE470E43009F41F5FE22FE870D1
:109E3C00E83009F41F5FE22FE072E03209F41F5F93
:109E4C00E22FE074E03409F41F5FE0E0F0E0FA93F5
:109E5C00EA931A930E940263E22FE170E13029F435
:109E6C00E0915D0BEA930E94A562ADDEA0914009E2
:109E7C00A73729F4E2E0E0933508E03009F473C029
:109E8C000E9406720E94D3770E94C1721E2F0E94FC
:109E9C00DC72AF01E1E0EA930E944B620E2FE0917D
:109EAC001008A0911108EA1739F00E94BE77ED5501
:109EBC00F84FE081E23009F053C00E94BE77EC55B8
:109ECC00F84FDF010E94867B4E175F0711F00C9450
:109EDC00B24F0E94BE77E655F84F008011800E9469
:109EEC00DE6D0E949B71EA17FB0769F10E94BE7739
:109EFC00E655F84FDF010E94867B0E94D9770E94BD
:109F0C00BE77E655F84FDF010E94867BEC59F44F83
:109F1C00E0810E94E1770E94E8770E94616D0E94C7
:109F2C00EB77EFEAF8E10E94BD72003029F05A930A
:109F3C004A930E94D86202C00E94F1770E94F57782
:109F4C000E947E6309C0003039F00E94F97720F43A
:109F5C000E94B4730E945E26E1E1F8E00E94007852
:109F6C00E0E0E0933508A0914009A33421F40E946D
:109F7C00A633E03009F40BC00E9406720E94D3771E
:109F8C000E9451730E940F6C63D30E94FB1CA09122
:109F9C004009A13411F0A23421F40E9406720E94EF
:109FAC00D377A0914009A03421F40E94A633E0306D
:109FBC0009F420C00E94C172E887F987E2E0EA93B5
:109FCC000E944B621E2F0E9404780E9421180E944E
:109FDC00F4730E940A78E152F84F10830E94F473D4
:109FEC00E652F84FA7E0A0830E94DA710E94067235
:109FFC000E94D377A0914009AB3439F0A33529F0F6
:10A00C00A13519F0A13709F076C00E94A633E030D3
:10A01C0011F40C947B500E9406720E941178E1E4BA
:10A02C00F9E00E94D772E22FE270E23029F4E4E00A
:10A03C00EA930E944B6202C0E1E0F0E0E887F98706
:10A04C00A0914009A13511F0A13721F40E94DC72D6
:10A05C001E2F02C01091E50BE22FE470E43011F4D6
:10A06C00E4E001C0E3E0EA930E944B62AF01A091EF
:10A07C004009A33511F0A13731F4E885F9850E9428
:10A08C00817AE887F9870E94F97720F0A091D30BA9
:10A09C00A13011F51A935A934A93EB85FC85FA93E8
:10A0AC00EA930E941A1D0E946B77EE83FF83AE81A8
:10A0BC00BF810E945E7D84F40E940672E6E6EA93FC
:10A0CC000E94A562EE81FF813197EE83FF83AE8102
:10A0DC00BF810E945E7D94F31A935A934A93EB8549
:10A0EC00FC850E9494726FDD06C00E9451730E9421
:10A0FC000F6C0E941A1D0E946F7D2A9608950E9473
:10A10C001578E89422F80E94D373E2E7EA930E9450
:10A11C00A562E0913B08EA930E94A562EFE0EA9306
:10A12C000E94A562A0913808AA3219F41A9365D33B
:10A13C001AC0A0913B080E943271EC59F44FE08197
:10A14C00EA1721F4E0913B08E03349F40E94AD6C2E
:10A15C00AC59B44FE0913B08EC931A934ED322FCCC
:10A16C0002C00E947E63C0C20E941578E0913B0839
:10A17C00E053AE2F0E943271EB58F44FE081EA1796
:10A18C0041F51A933AD3A0913608A23019F40E94E3
:10A19C001D7809F402C00E942378A0913608A330E0
:10A1AC0019F40E941D7809F402C00E942378E0E0A3
:10A1BC00E0933608E093600C0E943271EB58F44F38
:10A1CC00BF01E081EF5FAE2FEAE00E943C7BDB0138
:10A1DC00EC938AC2E881E03019F40E94F17706C052
:10A1EC00E881E8500E9451740E94D862219608952B
:10A1FC000E94687D25FC28C20E941D7811F40C94E5
:10A20C007E520E942678E752F84F9F01D901119691
:10A21C00EC91E43071F50E942C780E942F780E940A
:10A22C003678F901A681A03021F4A281B381109770
:10A23C0009F007C0E2EBF8E10E94BD720E94F577CD
:10A24C0015C00E94E8770E943A780E94EB77E5EB04
:10A25C00F8E10E94BD720E943E780E944478F90198
:10A26C00A085B185BA93AA930E94D8620E944A78BD
:10A27C00EBC1E730C9F40E942C780E942F780E9421
:10A28C003678E8EBF8E10E94BD720E943E780E949D
:10A29C00EB77EBEBF8E10E94BD720E943A780E94DA
:10A2AC00D8620E944A78D0C1E93089F40E942C7897
:10A2BC000E942F780E943678EEEBF8E10E94BD7276
:10A2CC000E9451780E94EB770E944A78BDC1E6301B
:10A2DC0029F5EAE2EA930E946363E1ECF8E10E945B
:10A2EC00BD72D901EC910E945478E091CD0B0E9483
:10A2FC005478EBE4EA930E94A5620E943A780E949B
:10A30C00D862E4E5EA930E94A5620E943E780E941E
:10A31C00D8620E947E630E94237896C1E530C9F40E
:10A32C000E94A5730E94D977D901EC910E94E17724
:10A33C000E94E8770E943A780E94EB77EFEAF8E106
:10A34C000E94BD720E943E780E94D8620E944A7898
:10A35C007BC1E83039F50E942C780E942F780E943E
:10A36C003678E4ECF8E10E94BD72F901A681AA935B
:10A37C000E94B173309719F00E94C66F04C0D901C6
:10A38C001696EC91F0E0FA93EA930E94D8620E9440
:10A39C00F5770E947E63D9011196E0E0EC930E9460
:10A3AC00237852C1E130C9F5A0911908A53029F4E0
:10A3BC00E091CD0BE65F1E2F01C011E0E12F0E9452
:10A3CC0058780E9432710E945D780E9460780E94D9
:10A3DC00E8770E943A780E94EB77E7ECF8E10E946C
:10A3EC00BD720E943E780E944478D9011796EC9178
:10A3FC000E9451740E94D862A0911908A53041F4B2
:10A40C000E946478A481B581BA93AA930E943A639E
:10A41C000E9457750E946A7817C1E330B1F40E940C
:10A42C00A573F0960E9475780E94A5730E945D78C2
:10A43C000E946078EAECF8E10E94BD720E943E78BE
:10A44C000E9479780E946A78FFC0EB3069F50E940F
:10A45C007C780E947F780E946078EDECF8E10E9495
:10A46C00BD72F901A681AA93B5DE0E946478A7811A
:10A47C00AA93B0DE0E946478A085B185BA93AA93A2
:10A48C000E9444780E943E780E944478F901A4818D
:10A49C00B581BA93AA930E9444780E9451780E9485
:10A4AC0079780E946A78D0C0EC3089F40E947C786C
:10A4BC000E947F780E946078E0EDF8E10E94BD7206
:10A4CC000E9451780E9479780E946A78BDC0EE3063
:10A4DC0079F40E947C780E947F780E946078E3ED8A
:10A4EC00F8E10E94BD720E9457750E946A78ACC058
:10A4FC000E94B87761F0A0913608A03041F4A09189
:10A50C00D20BA13021F40E94DE6DE13009F426C09B
:10A51C00A091850BA03059F0E091870BF091880B3E
:10A52C00FA93EA93E8EEF3E00E945B73B9F4E1E38B
:10A53C000E947578E091760BE05D0E94E1770E94B5
:10A54C00DE6DEA930ED1E09336080E945775E093C6
:10A55C005E0CF0935F0CE0E0E093850BA091360865
:10A56C00A03059F0E0915E0CF0915F0CFA93EA93F5
:10A57C00E4E6F0E00E945B7309F025C0A091360878
:10A58C00A23019F40E941D7809F402C00E942378AD
:10A59C00A0913608A33019F40E941D7809F410C05C
:10A5AC00A091600CA33030F00E942378E0E0E0939F
:10A5BC00600C06C00E942678E652F84FA8E0A083F3
:10A5CC00E0E0E0933608A091860BA130E9F5E0912C
:10A5DC00390CA091380CEA1791F1EAE20E947578D7
:10A5EC00E091740BE05D0E94E177E091390CEA9305
:10A5FC000E94AD1E0E94E877E091290C0E945174D4
:10A60C000E94EB77E6EDF8E10E94BD720E94BE70ED
:10A61C00FA93EA930E9444780E943C740E948378D7
:10A62C000E947E63E091390CEA930E94F21CE09147
:10A63C00390CEA930E94C11CE093390C05C0E0E090
:10A64C00E093860B689420F80E946F7D26960895FF
:10A65C001A930A930E94A633E030D9F00E94F47347
:10A66C00E752F84F8F01EC81FD81D8011296ED93E2
:10A67C00FC93EA81FB81D8011896ED93FC93EE8153
:10A68C00D8011696EC93D8011196E4E0EC930E9455
:10A69C00DA711981088127960895E091420BEA93AB
:10A6AC000E94A562E091430BEA930E94A562089573
:10A6BC00F4DF0E9499770E9486780E9486780E9427
:10A6CC00EB7799C01A930E94D7611E2F103021F09E
:10A6DC00E12FE150E093400BE0DFE091400BEF5FA6
:10A6EC000E9451740E94EB77199108950E946A7D23
:10A6FC0031E00E948D7828F00E94CB72AC91A4338B
:10A70C0008F02AC030E00E94CB72EC91E270E69522
:10A71C001E2F0E94CB72EC91E1700E2FA0915A0B60
:10A72C001A1729F4E1E0EA27E0935A0B31E0A091E3
:10A73C005B0B0A1729F0E1E0EA27E0935B0B31E0B1
:10A74C00E0915B0BEE0FE05DA0915A0BEA0FEA93E0
:10A75C000E94A5620E94C473E32F0E94717D24960F
:10A76C0008951A9310E00E94B87711F40C94FD53DD
:10A77C000E94481CEAEDF8E10E94BD72E091240CA5
:10A78C000E9451740E94EB77EDEDF8E10E94BD72CE
:10A79C00E091270CF091280C0E9483780E94CE77D0
:10A7AC00A031E7E2BE074CF4E0EEF8E10E94BD7286
:10A7BC00E091250CF091260C13C0E3EEF8E10E9419
:10A7CC00BD72E9810E94DB6F0E94CE77EA0FFB1FFE
:10A7DC000E947C70E091250CF091260CE051F74220
:10A7EC00FA93EA930E94D8620E94F57711E00E94D6
:10A7FC009178E12F18812296089524970E94687D04
:10A80C000E9491780E948061E13010F40C94D9562A
:10A81C00E091420BEB3441F4E091430BE33219F439
:10A82C000E94D7611E2FBCC2E435A9F4E091430B02
:10A83C00E33221F40E94D761EE83FF83E091430B56
:10A84C00EF3441F40E94D7611E2F1A930E94947426
:10A85C000E942118A5C2E23411F00C947655E091B7
:10A86C00430BE13251F4AA85AF3F29F40E94517396
:10A87C000E940F6CEDDE0E94FB1CE091430BE13457
:10A88C00E1F40E94D7611E2F113071F4A0913608AB
:10A89C00A13019F40E94B87709F402C00E94531C2D
:10A8AC00E0E0E093850B09C0E1E0E093850B0E94AA
:10A8BC001768E093870BF093880BE091430BE5341A
:10A8CC00A9F4E6EEF8E10E94BD720E94301CF397E9
:10A8DC003CF00E94D7610E947C700E94987801C065
:10A8EC00E0E3EA930E94A5620E94F577E091430BA6
:10A8FC00E634D9F40E94A47819F40E94D761AF0110
:10A90C00E885F9850E94CB6F0E2F003420F0A091C2
:10A91C00D30BA13021F40E94B0780E941A1DAA8595
:10A92C00AF3F19F40E94B07893DEE091430BE2350F
:10A93C0011F00C9433550E94A47819F40E94D7613D
:10A94C00AF0130E0A091D30BA03021F40E94DE6D5A
:10A95C00E13009F027C00E94AC33E03011F10E94C5
:10A96C008872EC55F84FA885B985A083B1830E94F5
:10A97C008872E655F84FDF01EA850E94D6710E9475
:10A98C008872E855F84F10830E948872E755F84F8B
:10A99C0040830E948872ED55F84FA1E0A0830E947D
:10A9AC008E7259C00E94A633E23010F40C943155CB
:10A9BC000E9404780E94271E3E2F3F3F29F00E94E0
:10A9CC009170A417B5070CF412C00E943C74E41BE0
:10A9DC00F50B0E949F700E94657219F4E0E0E09301
:10A9EC00290C3A930E94B41E689420F803C0E0E04E
:10A9FC00E887E9870E94F473E752F84FDF01EA8594
:10AA0C00F0E0EC59F44FE081EC930E94F4730E9457
:10AA1C000A78EF51F84FDF01EA850E94D6710E9447
:10AA2C00F473E152F84F10830E94F473E652F84F1E
:10AA3C00A5E0A0830E94DA71E885F985309759F07A
:10AA4C000E940478FA010E94817A0E9494720E94FA
:10AA5C00B0780E94A21C689422F8E091430BE33575
:10AA6C00F1F50E94D761E887F9870E942678DF010B
:10AA7C00E652F84FE081E23081F4FD01EF51F84FDE
:10AA8C00008011800E94DE6D0E949B71EA17FB070B
:10AA9C0021F4A0913608A23009F01FC00E9426783C
:10AAAC00E552F84FDF010E94867BDF01E885F985CE
:10AABC00EA17FB0779F40E942678DF01ED51F84F75
:10AACC00E081EA93FD01E752F84FE081EA930E949E
:10AADC005E2603C0E7E0E0932406689422F860C188
:10AAEC00E43411F00C94DF55E091430BE33559F449
:10AAFC00E9EEF8E10E94BD720E94755E0E945478E6
:10AB0C00E1E0E0933909E091430BE03511F00C944E
:10AB1C00DE550E94B478E03011F40C94DE5520E040
:10AB2C000E94B87840F00E94CB72AC91A23219F01E
:10AB3C000E94BC7809F43CC0E22FE03061F40E9422
:10AB4C00CB72AC91A33211F421E004C00E94C07806
:10AB5C000E94505E2AC0E13051F40E94CB72AC913D
:10AB6C00A43211F422E001C020E010E01EC0E2305B
:10AB7C0011F0E330D1F40E94C0780E94EF67EF3FF0
:10AB8C0099F0E12FE295E07FEF930E94C0780E944C
:10AB9C00EF67AF91EA0F1E2F2F5F243021F41A9329
:10ABAC000E94505E20E001C020E00E94C473B8CF28
:10ABBC00F7C0E33411F00C944956E091430BE534A3
:10ABCC00B9F4E6EEF8E10E94BD720E94301CF397D6
:10ABDC004CF00E94D761E05FF84D0E947C700E949F
:10ABEC00987801C0E0E3EA930E94A5620E94F57791
:10ABFC00E091430BE634A9F441E050E00E94D761A8
:10AC0C000E2F0E94C478E13019F40E94D761AF0175
:10AC1C001A930E94926CE05FF84D0E9475760E9428
:10AC2C001A1DE091430BE335A1F40E94C8780E94F1
:10AC3C00C16FE83141F4E091890BEA930E94D0177F
:10AC4C00689420F806C0E885EA93EFEFEA930E9437
:10AC5C005E26E091430BE134A9F4ECEEF8E10E949E
:10AC6C00BD720E94C878EA930E94CF180E949F255B
:10AC7C00E03011F0E1E301C0E0E3EA930E94A56249
:10AC8C000E94F5778DC0E63511F00C94AE56E0912C
:10AC9C00430BE33411F00C94AD560E94D7611E2F78
:10ACAC00113010F40C94AD56A0911908A13091F507
:10ACBC000E94C478E03021F0A091A2061A1709F086
:10ACCC0028C011500E94D761AF011A930E94302105
:10ACDC003E2F0E940B730E944C710F010E940B734C
:10ACEC000E94CC6D0E94CF780E94C478E03071F045
:10ACFC000E94D761AF010E941F730E944C710F011B
:10AD0C000E941F730E94CC6D0E94CF781A930E94F0
:10AD1C00C2111DC01630D8F41150A12FEAE00E94C8
:10AD2C00EC7AA3E2EA9FF001E855F94FBF01A12F9D
:10AD3C00EAE00E943C7BF0E0BB01AAE0B0E00E949C
:10AD4C00BA7ADB01AE0FBF1F14960E94E67028C0C2
:10AD5C00E93431F5E091430BE03551F40E94D761B1
:10AD6C001E2FE0E0EA931A930E94A218E0932E069D
:10AD7C00E091430BEC34A1F40E949B61E093280614
:10AD8C000E94C478E03021F00E949B61E093290678
:10AD9C000E94C478E03021F00E949B61E0932A0667
:10ADAC000E943C612FCD0E946F7D2B960895A0913F
:10ADBC00580BA03521F4A091590BA03408F005C014
:10ADCC00E091590BEA930E94EF18A091580BA33510
:10ADDC0021F4A091590BAA3008F005C0E091590B51
:10ADEC00EA930E941A19A091580BAB3421F4A0914C
:10ADFC00590BA03808F005C0E091590BEA930E945A
:10AE0C005819A091580BA63521F4A091590BA031DB
:10AE1C0008F005C0E091590BEA930E948619A091A5
:10AE2C00580BA43511F40E940B189CD60895E3EA34
:10AE3C00F6E0FA93EA93E091420BEA93E0E8F0E053
:10AE4C000E94F86F08950E94D778A0E0A083E0914B
:10AE5C00400BE093590BE091420BE093580B089593
:10AE6C000E94687D0E948061E13010F40C94305A8D
:10AE7C00E091580BA091420BEA1709F098DFE09192
:10AE8C00420BE33239F5E091430BEC3431F4CFDF74
:10AE9C00E4E0E09318080E94DD78E091430BE43580
:10AEAC00C1F4C5DFE091630CE03029F0EF77A9E045
:10AEBC00B0E00E94C87BE091640CE03029F0EF77A1
:10AECC00AAE0B0E00E94C87B0E94DD78E7E0E09346
:10AEDC00180802C0EB34E1F5E091430BE13211F4B8
:10AEEC00A6DF35C0E53211F462DF31C0E33299F4EC
:10AEFC000E94E37821F00E94EE780E9424190E94AF
:10AF0C00D778E081EB3429F4E0E0E093340CE09363
:10AF1C00350C99DF1CC0E134D1F40E94D7619F013C
:10AF2C002093340C0E94F47891F00E94D7619F0119
:10AF3C00A091340CF901E270F070EA2BE093340C20
:10AF4C000E94F47821F00E94D761E093350C7FC207
:10AF5C00E33581F5E091430BE13211F468DF29C050
:10AF6C00E33299F40E94E37821F00E94EE780E947B
:10AF7C00FE180E94D778E081E33529F4E091400B6C
:10AF8C00EA930E94431B5FDF14C0EE3491F40E94DD
:10AF9C00747410E01A3068F4A3EBBBE0EE27A10F39
:10AFAC00BE1F0E943271EC5BF44FE081EC931F5F8B
:10AFBC00F1CF4DC2E63511F00C942C58E091430BB7
:10AFCC00E13211F434DF41C0E33299F40E94E378AA
:10AFDC0021F00E94EE780E9466190E94D778E081D9
:10AFEC00E63529F4E091400BEA930E9499192BDF86
:10AFFC002CC0E63531F40E94D7619F012093300CB0
:10B00C0024C0E53471F40E94D7619F0120932F0C6A
:10B01C000E94F47829F00E94D7619F012093320C92
:10B02C0014C0E43591F440E050E00E94D7619F01D8
:10B03C00022E032A11F042E050E00E94F47819F03D
:10B04C000E94D761AF014093310C01C2E43511F07D
:10B05C000C94E658E091430BE33231F40E94D76133
:10B06C003197E093400BABC0E03511F00C94E558F0
:10B07C0010E00E94B87850F00E94CB72AC91AD33C6
:10B08C0029F00E94BC7811F01E3008F005C00E9417
:10B09C0032710E94FA78EDCF0E9432710E940379CE
:10B0AC00EDE30E94087911F00C94E558E4E5E09387
:10B0BC00580B10E00E945A703496E491EF3F11F453
:10B0CC000C94E5580E9478740E945A700E947C6D12
:10B0DC000E94B168E03011F00C94E3580E945A7051
:10B0EC003496E491E03851F40E94D761E058FF4F58
:10B0FC00E093630CE0E8E093640C5FC0E23839F451
:10B10C000E94D761E058FF4FE093640C56C0E138C1
:10B11C0039F40E94D761A8E0B0E00E94C87B4DC012
:10B12C00E03011F0E13051F40E945070FF93EF9336
:10B13C000E94D761AF91BF91EC933FC0E23059F4BC
:10B14C000E945070FF93EF930E94D761AF91BF9113
:10B15C00ED93FC9332C0E33051F40E945070FF9396
:10B16C00EF930E94B661AF91BF91EC9326C0E4308F
:10B17C0021F50E945A703596E491EA930E948562FB
:10B18C000E945070E093610CF093620C00E00E94FE
:10B19C005A703596E4910E1780F40E94926CEC5B19
:10B1AC00F44FE081A091610CB091620CEC93A1E69C
:10B1BC00BCE00E94706E0F5FEACF1F5F7BCF47C170
:10B1CC00E03511F00C942D5AE091430BE33299F4D5
:10B1DC000E94E37821F00E94EE780E94CF180E9422
:10B1EC00D778E081E03529F4E091400BEA930E9496
:10B1FC00581B29DE2CC1E13211F419DE28C1E134CF
:10B20C00D1F40E94D7611E2F00E00D3098F40E94FB
:10B21C009D74EA0FFB1F3396E491E11749F40E94E9
:10B22C009D740E94A174A0919A0BEA2BE0939A0B47
:10B23C000F5FEBCF0CC1E63559F5E0E0E093410B25
:10B24C00ADE9BBE00E940D79FF93EF930E94D761AB
:10B25C00AF91BF91EC93EBE2EA930E944C61E0302A
:10B26C0059F0A0EABBE00E940D79FF93EF930E9486
:10B27C00D761AF91BF91EC930E941079A091410BD3
:10B28C00A33018F40E94F47809F401C0D9CFDFC0C0
:10B29C00ED34D1F4E0E0E093410BA9EABBE00E946D
:10B2AC000D79FF93EF930E94D761AF91BF91EC930F
:10B2BC000E941079A091410BA33018F40E94F478ED
:10B2CC0009F401C0EACFC3C0E735D1F4E0E0E09364
:10B2DC00410BA0EBBBE00E940D79FF93EF930E9412
:10B2EC00D761AF91BF91EC930E941079A091410B63
:10B2FC00A23018F40E94F47809F401C0EACFA7C078
:10B30C00E434C9F5E0E0E093410B0E94D7619F0162
:10B31C00E2E0EA930E945961AF01E3E70E940879E9
:10B32C0059F40E941679BF01D9010E94D171E40F22
:10B33C00F51FDB01ED93FC93E9E40E94087979F4A5
:10B34C000E94167920833183AAE9BBE00E940D7913
:10B35C000F010E941D79EC91E160D001EC930E94E9
:10B36C001079A091410BA33018F40E94F47809F4E1
:10B37C0001C0CBCF6CC0EE3499F40E94747410E011
:10B38C001A3068F4AAE8BBE0EE27A10FBE1F0E949A
:10B39C003271EC5BF44FE081EC931F5FF1CF57C03F
:10B3AC00E33449F40E94B4780E94D761E093950B82
:10B3BC00F093960B4CC0E33589F40E94D7619F0142
:10B3CC0000240216030624F42B30E0E03E070CF0B8
:10B3DC0004C0F9013197E093970B39C0E53529F496
:10B3EC000E94D761E093990B32C0EF3491F40E9424
:10B3FC00D7611E2FECE2EA930E944C61E12FE2959B
:10B40C00E07FEF930E94D761AF91EA0FE093980B26
:10B41C001EC0E035E1F4E0E0E093410BACEABBE0A8
:10B42C000E9423790E944C71FF93EF930E946562F6
:10B43C00AF91BF91ED93FC930E941079A091410BB9
:10B44C00A23018F40E94F47809F401C0E7CF0E94EE
:10B45C003C6108CDE0E0E093430A0E946F7D2696A4
:10B46C0008950E946A7D0E948061E13010F40C9472
:10B47C00E95CE091420BE332A9F4E091430BE03537
:10B48C0019F4EFEEF8E109C0E83419F4E0E1F9E160
:10B49C0004C0E33531F4EBE2F9E1FA93EA930E944C
:10B4AC00B6628EC2E43511F00C94F45AE091430B61
:10B4BC00E43229F4E8E2F0E00E9427798EC0E3320E
:10B4CC0011F400D98AC0E03511F00C94F35AE5D888
:10B4DC00A091400BA83210F00C94F35A0E942B79D7
:10B4EC000E947C6D0E94B662EDE3EA930E94A56215
:10B4FC000E942B793496E491E03839F40E94DE6D89
:10B50C000E9451740E94D86268C0E23839F40E94DB
:10B51C004B700E9451740E94D8625FC0E13839F4BC
:10B52C000E944C740E9451740E94D86256C0E03044
:10B53C0011F0E13051F40E942B7932960E94957BE8
:10B54C000E9451710E942F7948C0E23059F40E9438
:10B55C002B7932960E94957BDF010E94BF730E946B
:10B56C00D8623BC0E33051F40E942B7932960E9492
:10B57C00957BE081EA930E94E6622FC0E43069F586
:10B58C000E942B7932960E94957BE093610CF0938C
:10B59C00620C10E00E942B793596E4911E1790F402
:10B5AC000E943271EC5BF44F0F01A091610CB091D1
:10B5BC00620CEC91D001EC93A1E6BCE00E94706EA1
:10B5CC001F5FE8CF0E942B793596E491F0E00E9442
:10B5DC0003790E9478740E942F63F2C1E33579F5E8
:10B5EC00E091400BEA930E94FE18E091430BE43289
:10B5FC0029F4EAE0F0E00E94277920C0E33211F44C
:10B60C0061D81CC0EE34D1F448D810E01A3068F47C
:10B61C000E943271EC5BF44F0F01A3EBBBE00E9474
:10B62C006075D001EC931F5FF1CFE0E0E0934E0B1F
:10B63C000E9478740E942F630E94F577C1C1E63591
:10B64C00D9F5E091400BEA930E946619E091430B07
:10B65C00E43229F4E5E0F0E00E9427792CC0E332D3
:10B66C0011F430D828C0E53451F417D8E0912F0CE0
:10B67C000E9451740E943379E091320C19C0E63566
:10B68C0029F40E945353E091300C12C0E43599F424
:10B69C000E945353E091310CE03011F0E1E301C012
:10B6AC00E0E3EA930E94A5620E943979E091310CA3
:10B6BC00F0E00E94837884C1E03511F00C94B35C07
:10B6CC00E091400BEA930E94CF18E091430BE432D7
:10B6DC0029F4E0E4F0E00E9427793EC1E33219F44A
:10B6EC000E94685339C1E13411F00C94BF5B0E9485
:10B6FC00535312E0A0919A0BECEDEA233E2F00E09D
:10B70C000D3078F40E949D740E94A174E31739F4F3
:10B71C000E949D74EA0FFB1F3396149102C00F5FB9
:10B72C00EFCF0E94616D0E94EB77E091980BE030B7
:10B73C0089F0E6E4F9E10E94BD720E94406D0E941E
:10B74C0051740E943379E091980BEF700E94517400
:10B75C000E94EB77E091990BE03051F0E9E4F9E1CC
:10B76C000E94BD72E091990B0E9451740E94EB777C
:10B77C00F3C0E43479F50E943D79A091410BA330DC
:10B78C0040F5E091410BE03011F00E9439790E94B4
:10B79C001D79EC91E17061F4A3EABBE00E9423797E
:10B7AC000E94CC6D0E94BF730E943A63E3E70BC00A
:10B7BC00A3EABBE00E9423790E94CC6D0E94BF7368
:10B7CC000E94D862E9E4EA930E94A5620E94107973
:10B7DC00D4CFBEC0ED34C9F40E943D79A091410B89
:10B7EC00A33090F4E091410BE03011F00E943979D4
:10B7FC00A9EABBE00E944379EC910E9451740E942B
:10B80C00D8620E941079EACFA3C0E735C9F40E9430
:10B81C003D79A091410BA23090F4E091410BE030C6
:10B82C0011F00E943979A0EBBBE00E944379EC91B6
:10B83C000E9451740E94D8620E941079EACF88C08D
:10B84C00E63531F50E943D79A091410BA330F8F417
:10B85C00E091410BE03011F00E943979ADE9BBE089
:10B86C000E944379EC910E9451740E94D862EBE2E1
:10B87C00EA930E94A562A0EABBE00E944379EC9196
:10B88C000E9451740E94D8620E941079DDCF60C072
:10B89C00EE34D1F40E94535310E01A3068F40E9435
:10B8AC003271EC5BF44F0F01AAE8BBE00E946075AB
:10B8BC00D001EC931F5FF1CFE0E0E0934E0B0E94C0
:10B8CC0078740E942F6344C0E33499F40E9453535C
:10B8DC000E947874E1E5F9E1FA93EA930E94C66F4D
:10B8EC000E94D8730E945B750E9478740E942F632B
:10B8FC002FC0E035A9F40E945353E091AC0BF091AA
:10B90C00AD0BFA93EA930E9452630E943979E0914D
:10B91C00AE0BF091AF0BFA93EA930E94526318C0EE
:10B92C00E33531F40E945353E091970BEF5F0DC058
:10B93C00EF3491F40E9453530E94406D0E94517455
:10B94C000E943379E091980BEF70F0E00E942F7910
:10B95C00EBE3EA930E94A56233C0EB3489F5E091E6
:10B96C00400BEA930E942419E091430BE43229F432
:10B97C00E0E8F0E00E94277923C0E33219F40E943A
:10B98C0068531EC0E134E1F40E945353A091340C6F
:10B99C00E1E0EA230E9451740E943379A091340CA7
:10B9AC00E3E0EA230E9451740E943379E091350C54
:10B9BC000E9451740E94D862E4E5F9E10E94BD72C4
:10B9CC000E943C6150CD0E9491780E94717D24961A
:10B9DC0008951A930E940672E0E4F9E00E94D7726F
:10B9EC000E9491780E944779E181E43471F40E94BD
:10B9FC00477902800E94DE6DE05DE01529F00E941F
:10BA0C004779E281EA3209F401C057C00E944C79AF
:10BA1C000E944779E1810E9450790E944779E28126
:10BA2C000E9450790E94CB721C910E9447793396E8
:10BA3C000E94D772E12FE23131F40E945679E6E090
:10BA4C00EC930EDA3AC0E13131F40E945679E2E11E
:10BA5C00EC9307DD32C0EF30A9F40E945679EEE08A
:10BA6C00EC930E947C53E13039F4A0913508A0305E
:10BA7C0019F00E94B87709F402C00E94531C0E946E
:10BA8C005C791BC0EE30C9F40E945679EFE0EC9360
:10BA9C000E947C53E13089F4A0913508A03019F054
:10BAAC000E94B87709F402C00E94531CE0E0E093B6
:10BABC003508EFEFEA930E94035463C21A930E9475
:10BACC00D3730E942870EAE7EA930E94A5620E9451
:10BADC00CB7211971C91E12FE23131F4E6E0EA933D
:10BAEC000E94A562BDD937C0E13131F4E2E1EA939D
:10BAFC000E94A562B6DC2FC0EF3099F40E946078EA
:10BB0C000E947C53E13039F4A0913508A03019F033
:10BB1C000E94B87709F402C00E94531C0E945C7901
:10BB2C001AC0EE30C1F4EFE0EA930E94A5620E94C5
:10BB3C007C53E13081F4A0913508A03019F00E94BB
:10BB4C00B87709F402C00E94531CE0E0E09335087A
:10BB5C00EA930E940354A0913808AA3211F00E9473
:10BB6C007E630FC2EFEFE093580BE093590B0895EF
:10BB7C00AC81A03310F0AA3308F006C00E946379A0
:10BB8C00E0530E946B7999C4AC81A13410F0A734B6
:10BB9C0008F006C00E946379E7530E946B798DC44C
:10BBAC00A881B981E0E0EC9388C4AA93EA93FA9354
:10BBBC00EFB7EA931A930A931BB10CB1E0919D0C69
:10BBCC00F0E0E559F34F0083A0919D0CAF5FA0937B
:10BBDC009D0CA23319F4E0E0E0939D0C09911991AE
:10BBEC00F3C21A93E0919E0CA0919D0CEA17D1F32D
:10BBFC00F0E0E559F34F1081A0919E0CAF5FA0933C
:10BC0C009E0CA23319F4E0E0E0939E0CB9C1A09114
:10BC1C009D0CAE5CE0919E0CAE1BE2E30E943C7B63
:10BC2C0008950A921A92FA926A937A938A939A9343
:10BC3C00AA93BA93EA93FA93EFB7EA930E947079B6
:10BC4C0049F0A0913909A03021F00E94F50CE130A7
:10BC5C0009F401C011C0E091040DF0E0E156F34F7E
:10BC6C00E081ECB9A091040DAF5FA093040DA43654
:10BC7C0019F4E0E0E093040DE991EFBFF991E9913B
:10BC8C00B991A9919991899179916991F9901990AA
:10BC9C00099018951A930E94707959F45D9B09C00C
:10BCAC00A0913909A13021F40E94F50CE03009F083
:10BCBC0013C01091030D0E943271E156F34FA9810C
:10BCCC00A0831F5F143609F410E0E091040DE11716
:10BCDC00E1F31093030D02C0E981ECB9A1C20E94FB
:10BCEC00707921F40E94F50CE13009F001C019C300
:10BCFC0050C10E946A7D8BDFE03011F40C947D5FA3
:10BD0C0070DF1E2FA091680CA53618F0E0E0E093D0
:10BD1C003A0930913A09E0913A09E03011F00C946B
:10BD2C00E45EA091E40BA13021F0A091E40BA230D1
:10BD3C0031F4E12FEF77E0934009EBE4CEC01A35F4
:10BD4C0021F4E1E0E0933A09CAC0123049F4E4E18D
:10BD5C00E0933A09E0E0E0933B09E0933D09BFC072
:10BD6C00A091E40BA33069F4173729F01A3310F4BF
:10BD7C00103308F402C0E7E001C0E0E0E0933C09B6
:10BD8C0005C01A930E94FF4DE0933C09A0913C0919
:10BD9C00AF3F99F010934009E1E0E0933B09109319
:10BDAC003D09E0913C09E03011F4E5E404C0EAE01F
:10BDBC00E0933A09E0E0E0933F0991C0E13069F487
:10BDCC00103039F4E2E0E0933A09E0E0E0933F0907
:10BDDC0003C0E0E0E0933A0982C0E23059F41093DA
:10BDEC003C0910933D09E0E0E0933B09E3E0E0936C
:10BDFC003A0975C0E330F1F40E9476790E947C799F
:10BE0C00EA0F0E948679A9F4E0913D09E03071F4C3
:10BE1C00E4E0E0933A09E0913B090E946E6F0E94C6
:10BE2C008F790E947679A0E0A08303C0E0E0E093D4
:10BE3C003A0955C0E43049F41D3019F4EAE5E093B1
:10BE4C003F09E0E0E0933A094AC0EA3079F40E94F5
:10BE5C0076790E947C79EA270E94867931F4E0E0B9
:10BE6C00E0933A09E5E4E0933F0939C0E431B9F4D1
:10BE7C000E9476791083E12FA0913D09EA27E09387
:10BE8C003D09E0913B09EF5FE0933B09E0E0E09373
:10BE9C00670C133019F4E5E1E0933A0920C0E53161
:10BEAC0011F0E63159F41A93E7E6FCE0FA93EA93C1
:10BEBC00EAE3F9E0FA93EA935BDE11C0E73179F437
:10BECC00E0E0E0933A09173131F4E091670CA0916E
:10BEDC003D09EA1709F003C0E3E4E0933F09A091A0
:10BEEC003A093A1719F0E0E0E093680C04CF0E948D
:10BEFC00717D44C4AA93BA93EA93FA93EFB7EA9389
:10BF0C001A930A9310919B0000919C00E12FEC7105
:10BF1C00A9F4E091CD0DF091CE0DEB5FF24F0083C3
:10BF2C00ADECBDE00E94706EE83CA0E0FA0731F485
:10BF3C00E0E0F0E0E093CD0DF093CE0D0991199176
:10BF4C00E991EFBFF991E991B991A99118951A93DB
:10BF5C000E9494790E949979D9F30E949479EB5FAD
:10BF6C00F24F1081AFECBDE00E94706EE83CA0E097
:10BF7C00FA0731F4E0E0F0E0E093CF0DF093D00D50
:10BF8C00E12F199108950E9494790E94997909F0F2
:10BF9C00C8C1E0E008950E946A7DF5DFE03021F031
:10BFAC00A091660CA03009F0E5C0D1DF1E2FA09146
:10BFBC00D90DA53618F0E0E0E093D30D3091D30DF8
:10BFCC00E091D30DE03059F4113019F4E4E0E09332
:10BFDC00D30D1A3519F4EAE0E093D30DC3C0E43065
:10BFEC00C1F4E0E0E093D30D1A3229F00E94DE6D2B
:10BFFC00E05DE11769F4109338081093D40DE5E077
:10C00C00E093D30DE0E0E093660CE1E0E093D60D15
:10C01C00A9C0E530A9F4E0E0E093D30D0E94DE6DF9
:10C02C00E05DE11761F00E94A0790E94A979E0918E
:10C03C00D60DEF5FE093D60DE6E0E093D30D92C002
:10C04C00E63091F4E091D60D0E94A9790E94A07976
:10C05C00EF5FE093D60DE0E0E093D70D133019F4C9
:10C06C00E7E0E093D30D7EC0E73011F0E83059F4EF
:10C07C001A93E7EDFDE0FA93EA93E3EDFDE0FA9312
:10C08C00EA9376DD6FC0E93081F4E0E0E093D30D04
:10C09C00173131F4E091D70DA091D40DEA1709F0C6
:10C0AC0003C0E4E5E093660C5DC0EA3041F4103067
:10C0BC0011F4EBE001C0E0E0E093D30D53C0EB30A2
:10C0CC0071F4E0E0E093D60D1093D50D1093D40DE0
:10C0DC00ECE0E093D30DE0E0E093660C43C0EC3071
:10C0EC00A1F5E091D60DF0E0E05CF64F10830E94D4
:10C0FC00A079EF5FE093D60DE091D50DE150E09380
:10C10C00D50DA091D50DA03021F4A091D40DA03067
:10C11C0009F00EC0EDE0E093D30DE091D60D0E9436
:10C12C006E6F0E948F79E091D60DF0E00E948F79AE
:10C13C00A091D50DA03021F4A091D40DA03009F41C
:10C14C0003C0E0E0E093D30D0DC0ED3059F4E0E016
:10C15C00E093D30D1D3031F4EAE5E093660CEFEF7C
:10C16C00E093650CE091D30DE31719F0E0E0E09358
:10C17C00D90D13CF0E94717D01C3AA93EA93FA9350
:10C18C00EFB7EA93E091DB0EA091DA0EEA1791F08B
:10C19C00E0913708E03019F0E89426F80AC00E94C4
:10C1AC00AE79F0E0E030A1E0FA0719F4E0E0E093BA
:10C1BC00DB0E03C0E89425F826F8E091650CE0301E
:10C1CC0019F0E0E0E093D30DE991EFBFF991E9911B
:10C1DC00A99118951A93E091DB0EA091DA0EEA174B
:10C1EC0021F4E0919B00E072C1F4E091DA0EF0E0F2
:10C1FC00E652F24FA981A0831091DA0E1F5F0E94C4
:10C20C00AD6CA030E1E0BE0709F410E0E091DB0E6C
:10C21C00E117E1F31093DA0E03C0E981E0939C007F
:10C22C00188122960895E0E0E093DB0EA091DA0EDF
:10C23C00A13020F00E94AE79689426F80895AA9354
:10C24C00BA93EA93EFB7EA93E091650CE03041F4CE
:10C25C00E0E0E093DB0E0E94DE6DEF5FE0933708C9
:10C26C00E991EFBFE991B991A99118950E94B8781D
:10C27C0018F00E94BC7809F403C00E94C473F6CF76
:10C28C000E94BC7811F40E94C47308950E94CB7272
:10C29C00AC91E881EA1729F40E94C4733197E1E06C
:10C2AC005DC1E0E05BC10E946A7D00E010E0EEE25F
:10C2BC000E940879E9F420E030E0EC810E94B0772C
:10C2CC00BCF4D8010E9487748F010E948D7818F0FD
:10C2DC000E94BC7908F009C00E94CB72EC910E94BC
:10C2EC0049730E0F1F1F0E94C4732F5F3F4FE5CF82
:10C2FC00F801E1C00E94B87828F00E944779E181EA
:10C30C00E03208F410C00E94CB72EC91E093420B27
:10C31C000E94C4730E94CB72EC91E093430B0E9479
:10C32C00C473E1E008950C9451660E9406760E9455
:10C33C00C0780E94EF67EF3F89F0F8010E94957A70
:10C34C00FF93EF930E94C0780E94EF67AF91BF916B
:10C35C000E9499748F010E94C473E9CFF8011EC02A
:10C36C001A930A9310E00E94CB720C910B3311F0CC
:10C37C00003208F412C0013310F0093308F007C082
:10C38C00E02F0E944973E255FF4FE4911E2B0E944F
:10C39C00C4730E94CB720C91E9CFE12F09911991D2
:10C3AC0008950E946A7D00E010E00E94CB72AC916F
:10C3BC00AD3221F40E94C47331E001C030E00E9420
:10C3CC008D7818F00E94BC7908F009C0D8010E9441
:10C3DC0087740E94C0798F010E94C473F0CF3030F3
:10C3EC0021F4F8010E94717DC9C1F8010E94817A83
:10C3FC000E94717DC3C124971A93E0E0E983EA831C
:10C40C00EB83EC830E94CB72AC91AD3221F40E9491
:10C41C00C47311E001C010E00E948D7818F00E94E6
:10C42C00BC7908F022C0A981BA818B819C81EAE099
:10C43C00F0E060E070E00E94E77A7F936F93FF93E7
:10C44C00EF930E94CB72EC91E053AF91BF918F911F
:10C45C009F91FF27662777270E94777AE983FA83D3
:10C46C006B837C830E94C473D7CF103031F4E98185
:10C47C00FA816B817C81188120C0E981FA816B8102
:10C48C007C810E94857A188118C00E946A7D20E008
:10C49C0030E000E010E0EC810E9417765CF4D901EA
:10C4AC000E9487740E94C0799F010E94C4730F5F21
:10C4BC001F4FF1CFF9010E94717D259608950E94BE
:10C4CC006A7D6FDF8F0120E030E0EEE20E94087998
:10C4DC0011F467DF9F01112322F4F9010E94817A84
:10C4EC009F01A0911B0CA13030F0D8010E94D1719A
:10C4FC00E20FF31F8F01F8010E94717D3FC11A9367
:10C50C0010E00E94B478E030A1F00E94B87858F0A6
:10C51C000E94CB72AC91A23231F00E94BC7819F01F
:10C52C00E9811E1708F005C00E9432710E94FA784A
:10C53C00ECCF0E9432710E9403790C94AD66E881B5
:10C54C000E945079E881A0915C0BEA0FE0935C0BA0
:10C55C00E881A0915D0BEA27E0935D0B219608958D
:10C56C001A9310E0E12FA981BA810E949974E49189
:10C57C00E03049F0E12FA981BA810E949974E491CD
:10C58C000E94C679EFCF0BC01A9310E00E9403767D
:10C59C00E03029F00E9403760E94C679F7CF18810B
:10C5AC002396089564970E941D750E94CB79E88D9F
:10C5BC00F98D0E94D8730E944D75E6DF669608953A
:10C5CC001A93ECE3EA93BBDF11E0193080F40E947C
:10C5DC003271E255FF4FE491A981EA2319F0E12F62
:10C5EC00E05D01C0E0E2EA93AADF1F5FEECFEEE36D
:10C5FC00EA93A5DF0C94AD6664971A930E94D079E8
:10C60C000E94CB79EA8DFB8D0E94D8730E945B75DA
:10C61C000E94D0790E94D9681E2FED891E1720F434
:10C62C000E94F1771F5FF9CF0E94D079ADDF18819E
:10C63C000EC064970E941D750E94CB79E88DF98D10
:10C64C006A8D7B8D0E9425740E941D759DDF6896F6
:10C65C000895E2E2EA9373DF0E94997795DFE2E2B4
:10C66C00EA936DDF0C94AE66A881B981E4E6F0E044
:10C67C000E940D7B0E942F79EEE2EA9360DFA88185
:10C68C00B981E4E6F0E00E943F7BFA93EA93E2E0A2
:10C69C00EA93B2DF0C94AE66A0911B0CA13020F093
:10C6AC000E949977E1DF07C00E9499777BDFE2E671
:10C6BC00F9E10E94BD720C94AE6625FE06C0E5E061
:10C6CC00F0E00E944B6EA895F8CFEAEDFDE0E09308
:10C6DC005E0BF0935F0BE1E00E940D72E0935C0B3C
:10C6EC000E94D5790E94DE6D0E9454780C941A69D0
:10C6FC001A930A93E091650CE03011F00C942068C9
:10C70C00E3E0EA931CDFE0915C0BE295EF70EA93B7
:10C71C000E9406681E2FE0915C0BEF70EA930E945A
:10C72C0006680E2F1A930BDF0A9309DFE7E1EA93F1
:10C73C0006DFEAEDFDE0A0915E0BB0915F0B0E946D
:10C74C00A97BEA1BE093DA0E689425F80C94206818
:10C75C00EE81EA93B2DFEC81FD810E94BD720E94F2
:10C76C00D97967DFC5DF0C944169EB81EA93A5DFCA
:10C77C000E942D71F5DE0E94D579BADF24960895BA
:10C78C00ED81EA939ADFEB81FC810E94BD72EA8114
:10C79C00EA93D5DEE981E03011F0EA93D0DEE8814E
:10C7AC00E03011F00E94D579A3DF269608950E94FF
:10C7BC00687D10E0E6E6F9E1A885B985EA17FB0784
:10C7CC0019F444E150E002C048EC50E0EA85E093F3
:10C7DC003809E89431F8EA93E985FA85FA93EA93F3
:10C7EC00EA85EA93EA85EA93E0E0EA93C9DF0E94DE
:10C7FC0017689F010E943B150E944F760E94236888
:10C80C000E2F31FC02C0003009F001C0F3CF31FE15
:10C81C0004C0E89431F8E1E004C01F5F1230B0F2BC
:10C82C00E0E00E946F7D2B9608951A930A93E09195
:10C83C00400AE03011F40C942068E0E0E0933909F0
:10C84C00E2E0EA9327DA10E003E00E9432710E94E2
:10C85C00E07961F00E9432710E94B5770E943271CA
:10C86C00E05CF54FE0810E271F5FEFCFE3E0EA932A
:10C87C0011DAE02FE295EF700E94E579E02FEF706E
:10C88C000E94E579E7E1EA9305DA0C9420681A93A3
:10C89C000A93E091400AE03011F40C9420680E9455
:10C8AC004B70E03021F0E091420AEA3209F405C005
:10C8BC000E944B70E05DE093420AE0E0E09339099E
:10C8CC00EAE5EA93E7D9E0E0EA93E4D910E00E94C4
:10C8DC0032710E94E07911F01F5FF9CF1F5F012FB9
:10C8EC000A93D8D910E00E9432710E94E07961F06D
:10C8FC000E9432710E94B5770E943271E05CF54F54
:10C90C00E0810E0F1F5FEFCFE02FE195EA93C2D9C4
:10C91C00EDE0EA93BFD90C9420681A930A93F8942B
:10C92C00E0E0E0933708E091DB0EE093DA0E7894C8
:10C93C00E091400AE03011F40C942068EAE5EA93A7
:10C94C0049DCE0E0EA9346DC10E00E9432710E9480
:10C95C00E07911F01F5FF9CF1F5F012F0A933ADCCA
:10C96C0010E00E9432710E94E07979F00E943271DD
:10C97C00E05CF54FE081EA932DDC0E943271E05CC3
:10C98C00F54FE0810E0F1F5FECCFE02FE195EA939E
:10C99C0021DCEDE0EA931EDC0C942068E881EA933C
:10C9AC008CDEEAE5EA93CBDDE0914009EA93C7DD42
:10C9BC000E94CB72EC91E03031F00E94C078BFDD68
:10C9CC000E94C473F5CF94DE0C941A691A930E94DA
:10C9DC000672E0913B08EA93B2DDE4E4EA93AFDD42
:10C9EC00E0913908EA93ABDD14E00E943271E85C07
:10C9FC00F74FE081E43040F00E943271E85CF74F71
:10CA0C00E0810E94C679F1CFE0E0EA9398DD3FDF48
:10CA1C003DC11A930A936DD9E0913F09E03011F4AE
:10CA2C000C948C65A0913F09AA3541F4A0913B0967
:10CA3C00A33020F0E0914109E43409F04BC00E948E
:10CA4C004B70E03021F0E0914209EA32C1F40E94CF
:10CA5C00DE6DE05DA0914209EA1721F0E0914209F8
:10CA6C00EA3221F40E94EF5C12DF08C0E3E4F9E043
:10CA7C000E94D772E09142090E94EB792BC00E9470
:10CA8C004B70E05DA0914209EA1721F50E94DE6D22
:10CA9C001E2FE0914309ED3421F4E0914409E33277
:10CAAC0009F007C0E5E4F9E00E94D7727ADC1E2F8A
:10CABC00DDDB0E94DE6DE11729F0E12FE05D0E94C5
:10CACC00EB7908C00E94DE6DE05DE09342090E94A4
:10CADC00EF5CDDDEA0913F09A53449F4A091E40B95
:10CAEC00A33019F40E94E82A02C00E94724EA09151
:10CAFC003F09A33411F40E94A02AA0913F09AB3442
:10CB0C0011F40E949B2AE0E0E0933F09A091E40B12
:10CB1C00A33011F40E94E82AE0E00C9420683BDA80
:10CB2C00A091660CA43529F4A0E025FCA1E0A0306E
:10CB3C0009F03AC0E0913A08E03581F4E0913B0805
:10CB4C00EA93E6E0EA930E94F342A0913B08A038F6
:10CB5C0020F0E0913B08E093650523C0E03721F419
:10CB6C00E0E0E09365051DC0EA3519F40E94645DB0
:10CB7C0018C0EA3711F42ADF14C0E23519F40E9408
:10CB8C0085500FC0E23719F40E94BA500AC00E94B7
:10CB9C006930E0913908A0913809EA1711F46894CA
:10CBAC0031F8E0E0E093660CA091660CAA3531F404
:10CBBC000E94EF5CB2DEE0E0E093660C6CC0A091EA
:10CBCC00690CA13050F0E091690CE150E093690CD4
:10CBDC00E03019F4E1E0E0936A0CA0E025FCA1E060
:10CBEC00A13049F4A0E026FCA1E0A03021F4A091F2
:10CBFC003708A03009F001C016DBE0913708E030AF
:10CC0C0019F0E150E09337080895E091D90DEF5FEA
:10CC1C00E093D90DE091680CEF5FE093680CE09124
:10CC2C00650CE03019F0E150E093650C0895A0918B
:10CC3C00E40BA13021F0A091E40BA23029F4E3E045
:10CC4C00E0939000E8E3E9B90895E0E00E94CF6B2F
:10CC5C00E1B3E360E1BB85E38A95F1F7E1B3EC7FE7
:10CC6C00E1BBE4E4E09374000E94E66B08951A9330
:10CC7C0014EAE4EA0E94F27941F40E94F779183040
:10CC8C0011F0103111F4E0E001C0E2E019910895C7
:10CC9C00E4E9E0937400E0E008951A93E981E1601F
:10CCAC000E94FC7931F40E94F779103411F4E0E021
:10CCBC004EC04CC01A93E9810E94FC7931F40E9459
:10CCCC00F779183111F4E0E042C040C01A93E981C1
:10CCDC000E94FC7931F40E94F779183211F4E0E0EB
:10CCEC0036C034C01A93E981E03011F0E4EC01C095
:10CCFC00E4E80E94F27979F40E94F779E0917300EC
:10CD0C00AA81BB81EC93103511F0183521F4E0E0C9
:10CD1C0018810C94976BE1E018810C94976B1A9323
:10CD2C00E981E093740010E0E0917400E07811F474
:10CD3C00163908F005C08BE18A95F1F71F5FF4CF27
:10CD4C00E0917400E07811F0E0E001C0E1E01881BE
:10CD5C00229608950E946A7D3D810C8120E087DF38
:10CD6C00E03011F5EE810E94FB6EF1F43A93AEDFE8
:10CD7C00E030D1F40E94007AB9F479DFE030A1F40C
:10CD8C00EE810E94DD6B81F4EDB7FEB7FA93EA9366
:10CD9C001F930E94E26B1F91E03031F479DFE12F99
:10CDAC000E94717D0C94416950DFD9CF0E946A7D3D
:10CDBC0030E00E811D815BDFE03099F4EF810E9441
:10CDCC00FB6E79F40E94007A61F41A937FDFE030F5
:10CDDC0041F4EC81EA937ADFE03019F459DFE0E0BA
:10CDEC0002C033DFE8CF0E94717D28960895229708
:10CDFC000E94687D50E02B853A85A89538DFE0309D
:10CE0C0011F00C945F67EE850E94FB6E11F00C9490
:10CE1C005F672A935BDFE03011F00C945F673A9305
:10CE2C0055DFE03011F00C945F6721DFE03011F03A
:10CE3C000C945F67EE850E94DD6BD9F5E0E0EE8324
:10CE4C00EF83EC85FD8531970E94D77549F4EDB7DA
:10CE5C00FEB7FA93EA931F930E94E26B1F9109C0ED
:10CE6C00EDB7FEB7FA93EA931F93E1E0EA933ADF4A
:10CE7C001F910E2FEE81FF81A885B985EA0FFB1F4C
:10CE8C001083EE81FF813196EE83FF83003039F4FD
:10CE9C00EC85FD85AE81BF81AE17BF0708F001C0E0
:10CEAC00D0CFEC85FD850E94D77519F4F1DEE0E05A
:10CEBC0002C0CBDEA3CF0E946F7D2F96089568979A
:10CECC000E94687D20E0E0E0EC8FED8F31E0A895CA
:10CEDC00E9A1FAA1662777270E943F7CEA87FB87A6
:10CEEC006C877D87EE8D0E94057AEE83FF836887C1
:10CEFC007987AA85BB858C859D850E94157DEA8BDB
:10CF0C00FB8B6C8B7D8B0E94997BFE017296FA9346
:10CF1C00EA930E94996BEE8BFF8B688F798F0E943E
:10CF2C000B7A0E94067CAF010E940B7AAE8DBB2758
:10CF3C00882799270E94A07B0E941E7ADE015A96B0
:10CF4C000E94067CED93FC930AA119A190DEE030BF
:10CF5C00D1F5EDA10E94FB6EB1F50E94007A99F516
:10CF6C001A93B4DEE03079F5303051F14F5F5F4FFA
:10CF7C00EC8DFD8D3196EC8FFD8FAC8DBD8D1197A9
:10CF8C00EBA1FCA1EA17FB0711F430E018C0EC8D03
:10CF9C00FD8D3197AF8DB8A10E941C7697DEEE8D7A
:10CFAC00DA01F0E0EA17FB0751F472DEEA8DFB8D33
:10CFBC00A9A1BAA1EA0FFB1FE9A3FAA389CFD4CF89
:10CFCC0067DEE0E002C041DEC1CF0E946F7DA69615
:10CFDC000895A881A03310F0AA3308F004C0E881AA
:10CFEC00E0530C941A69A881A13410F0A73408F00E
:10CFFC0004C0E881E7530C941A69EFEF0C941A699A
:10D00C00A881AA3020F4E881E05D0C941A69A8810B
:10D01C00AA3020F0E881E95C0C941A69E8E50C94DC
:10D02C001A691A930A93F8940091620B1091630B8E
:10D03C007894F8010991199108951A930A93F1DFE4
:10D04C008F01EA81FB81AC81BD81EA0FFB1FE01BE4
:10D05C00F10BDF010E945E7D2CF4E0E01981088168
:10D06C000C94C56BE1E0198108810C94C56BECE95B
:10D07C00F4E1FA93EA93EAEBF0E0FA93EA93E5E051
:10D08C00F0E0FA93EA93E4E0EA93E6E2EA93EEE066
:10D09C00EA930E949E4DE4E3F5E1FA93EA93EAEAFF
:10D0AC00F0E00E94237AE8E0EA93E0E2EA93E1E020
:10D0BC00EA930E949E4DE4E3F6E1FA93EA93E2EDE3
:10D0CC00F0E00E944B6CFA93EA93E2E0EA93E2E11F
:10D0DC00EA93E1E0EA930E949E4D0E940F6C0E943D
:10D0EC005C6EEFEAF0E00E94237AE3E0EA930E94A0
:10D0FC00BA4BEAE0F0E0FA93EA93E4E3F0E00E9442
:10D10C00476EE0E0E0931004EAE6F9E10E94786DE6
:10D11C00EFE0E093100408950895998188810096BA
:10D12C0041F0BD81AC81FB81EA8105900D920197A4
:10D13C00E1F7FD81EC810C94C56BB981A881109647
:10D14C0031F0FC81EB816A8161931197E9F7EB81F6
:10D15C00FC8125960895E991F991A991B9911D90B9
:10D16C000590011421F40020D1F7EE270895101832
:10D17C00E1F3E1E008F4E2500895E991F991A99105
:10D18C00B991CD0161916D936623E1F7FC0108958E
:10D19C00E991F991A991B991CD0105900D920020D9
:10D1AC00E1F7FC010895A991B991EE27FF276D9144
:10D1BC00662311F03196FBCF0895AA27BB27E9917E
:10D1CC00F9910590002011F01196FBCFFD01089507
:10D1DC007991E991F991A991B991CD01772351F008
:10D1EC007A9561916D936623C9F7772319F07A9537
:10D1FC006D93FBCFFC0108956991E991F991A99187
:10D20C00B991CD01662351F06A9505900D920020DD
:10D21C00C9F7662319F06A950D92FBCFFC010895AE
:10D22C005D9BFECFE881ECB9219608951A930A9381
:10D23C00AC81BD810E94867B3097C1F0AA81BB81F5
:10D24C000E94867B8F01309749F00230E0E01E0788
:10D25C0060F0F80131978F01ED93FC93AC81BD81A7
:10D26C000E94706E3197AE81A08303C0EE81EA9369
:10D27C00D7DF19810881279608952C970E94687D25
:10D28C0010E0E88DF98D3196E88FF98F3197E491A4
:10D29C002E2FE03011F40C94016BE12FE03039F4B7
:10D2AC00253211F411E002C00E942A7AA3C1E130A8
:10D2BC00C1F4253219F40E942A7A9BC112E0E0E0F5
:10D2CC00E98B00E02D3211F401E094C12B3219F4FA
:10D2DC00EBE2E98B8FC1203219F4E0E2E98B8AC1D1
:10D2EC0002C0E23039F450E013E0203311F400684E
:10D2FC0081C102C0E330A1F4203310F02A3308F0CE
:10D30C0009C0A52FEAE0EA9FF0015E2FE22FE0535F
:10D31C005E0F70C140E02E3211F414E06BC110C0EE
:10D32C00E430A1F4203310F02A3308F009C0A42F04
:10D33C00EAE0EA9FF0014E2FE22FE0534E0F5AC164
:10D34C002C3619F4026015E055C104C0E53011F01B
:10D35C000C94006BE22FE33649F40E94357AEE8987
:10D36C00FF89A481AA930E943B7A43C1E33741F41D
:10D37C000E94357A0E94457A0E94D9681E2F0AC0F5
:10D38C00E037A1F40E94357A0E94457A0E94E36846
:10D39C001E2F08600F77403011F0411708F001C0C4
:10D3AC00142F40E0E0E0E88B30E076C0E43611F07A
:10D3BC00E93611F4046002C0E537A1F4EAE0E88B29
:10D3CC0001FF08C0E0E0FAEC6AE97BE30E94286EFA
:10D3DC001AE023C0E0E1F7E260E070E00E94286E02
:10D3EC0015E01BC0E83511F4086004C0E83711F0F3
:10D3FC000C94FF6AE0E1E88B01FF08C0E0E0F0E08C
:10D40C0060E070E10E94286E18E007C0E0E0F0E1F7
:10D41C0060E070E00E94286E14E0403011F00F774D
:10D42C0001C041E001FF08C00E94357AAE89BF8976
:10D43C0014960E948A7B13C002FF08C00E94357AA2
:10D44C00AE89BF8914960E94D16D09C00E94357AAD
:10D45C00AE89BF8914960E94867B66277727EC8756
:10D46C00FD876E877F8702FF16C0AF85AA2362F403
:10D47C00EC85FD856E857F850E94857AEC87FD871E
:10D48C006E877F87EDE2E98BE989E03019F01F5F49
:10D49C004F5F01C00B7F342F00FD14C0151710F423
:10D4AC00351708F00FC007FF08C002FF04C00B7F40
:10D4BC002989115001C020E301C020E20E942A7A80
:10D4CC005150ECCF1417B0F4006102FF0AC00B7F6F
:10D4DC00E989EA930E943B7A503009F0515011507F
:10D4EC004150E0E3EA930E943B7A503009F05150EE
:10D4FC004150E8CF312FE889E030D1F43030B9F029
:10D50C0003FF08C0EE81FF813196EE83FF833197D4
:10D51C00E49105C0AE81BF81ED91AE83BF83EA93E8
:10D52C000E943B7A503009F051503150E7CF57C030
:10D53C000E944D7A0E94127B2E2F2A3030F003FF6E
:10D54C0002C0295C01C0295A01C0205D04FD25C020
:10D55C00213360F4A885B9858A859B85A130E0E0EC
:10D56C00BE07E0E08E07E0E09E0709F40BC043170E
:10D57C0040F4531710F000FF01C014C020E207FF65
:10D58C000CC020E3006102FF08C00B7FE989EA931D
:10D59C000E943B7A503009F051500E942A7A503048
:10D5AC0009F0515031500E944D7A0E944D7BEC870E
:10D5BC00FD876E877F87E889A885B9858A859B85D5
:10D5CC00FF27662777270E94127B0E94286EE8852A
:10D5DC00F9856A857B850E945A7D09F0A9CF00FFE9
:10D5EC0008C0503031F05150E0E2EA930E943B7A8F
:10D5FC00F8CF10E046CE0E946F7D6A960895FF9298
:10D60C00F82E22971A930A93DE010E94737A8D01E9
:10D61C00DE0116960E94737A0E94867BEA83FB8356
:10D62C00DE0114960E94737A0E94BF731A930A93B8
:10D63C00FE0136960E94506C20DEAA81BB81E0E090
:10D64C00EC93198108812496FF900895A991B991C2
:10D65C00EE27002460E8E894162E169407941E2AF0
:10D66C001EF0A015B10518F0A019B109E62BB7FBF7
:10D67C00AA0FBB1F669580F708957B816A81F9819B
:10D68C00E88177FB770F67FD7160972F9E5781F0CC
:10D69C0078F0983190F4AA27BB27882708948795AF
:10D6AC00B795A7959A95D1F7EA23FB23682305C074
:10D6BC00E8947727EE27FF2766276F77769508F48F
:10D6CC00606877F9A991B99189919991EA17FB074B
:10D6DC006807790797FB08950E94D9790E94567ABA
:10D6EC0019F40E945D7A1DC0E6F7A881B9818A8180
:10D6FC009B81E0E0F0E060E87FE30E941E7A11C0BD
:10D70C000E94D9790E94567A19F40E945D7A09C058
:10D71C00E6F30E945D7AA0E0B0E080E89FE30E940F
:10D72C00797C249608950E94627A0E945A7D39F47D
:10D73C00A881B9810E94FC6F0E94907B20C0AA81B5
:10D74C00BB818C819D810E94627D34F40E94627A3F
:10D75C000E94997BC1DF05C00E94627A0E94997B6E
:10D76C00CFDFA881B9810E94907BA881B9810E94EA
:10D77C008A7BAA81BB818C819D810E941E7A269610
:10D78C000895E991F99130971AF4E095F095319656
:10D79C000895E0937100E0E0E0937400E2B3E3607D
:10D7AC00E2BB089588EC90E00197F1F70895EA93B5
:10D7BC000E945366E0300895E0E0EA930C9478669A
:10D7CC0080E991E00197F1F708951A930A930C946C
:10D7DC00CB46EA9FF001F0E00895FA93EA93A02F6C
:10D7EC00B0E00895ECE3F0E00E94E27A0895ECE3F7
:10D7FC00F0E0FA93EA930895EAE3F3E0FA93EA93FC
:10D80C000C94A743E0E0E0930F04EFE0E0931004E6
:10D81C000895E0E0F0E0FA93EA930895FA93EA931E
:10D82C00E8E2F0E0FA93EA93E0E0EA930C94BA4B66
:10D83C00E0915905F0915A05FA93EA930895E09115
:10D84C005B05F0915C05FA93EA930895FA93EA93D9
:10D85C000C942143EFEEF0E0FA93EA930895FA93D7
:10D86C00EA93E0E0EA930C94BA4BFA93EA930C94A3
:10D87C00A743E12FA0E4B2E0F0E00E94997AEA0F0E
:10D88C00FB1F0895A12FB0E0ADCFFA93EA93E2E32A
:10D89C00F0E00895FA93EA93BCCFE0911004E09382
:10D8AC000F0408950E948C0D0C945349E32FF0E063
:10D8BC00E05BFD4FE4910895EA930E94A20DFE01F6
:10D8CC003696FA93EA930895FF27662777270E94E6
:10D8DC00997B84E00E94056B28960895FE01719651
:10D8EC00FA93EA930C94C7430E946A7D0C94CB463E
:10D8FC00E8E0F0E0FA93EA930895E4E0F0E0FA93BC
:10D90C00EA930895FA93EA93E8E3F0E0FA93EA9342
:10D91C0008950E94957BBECFE02FF0E00895A09172
:10D92C003A0CB0913B0CBD01A3E0B0E00E94BA7A76
:10D93C00E60FF71FE491E0300895E091C005EE0F7B
:10D94C00EE0FEF5F3E2F0895E32FF0E00895A12F27
:10D95C00B0E00895A0913A0CB0913B0CBD01A3E04E
:10D96C00B0E00E94BA7AE60FF71F08950E94977AEA
:10D97C00E05AFD4F0895FA93EA93E22FF0E00895F0
:10D98C000E94687DA09119080895E091C20BF0E007
:10D99C000895AFE3B1E00E940D7B089530911E080D
:10D9AC00E1E0E0930D04E2E0E0930E043A930E9470
:10D9BC00CF18E091980BE295EF70E0930F04E09193
:10D9CC00980BEF70E09310040895FA93EA93E52F07
:10D9DC00F0E0FA93EA930895E7E3F0E0FA93EA9320
:10D9EC000895E22FE450F0E0FA93EA930895EA8563
:10D9FC00FB85FA93EA930895E32FE058EA9309CF55
:10DA0C00EAE8FBE0FA93EA930C94C7433A930E943A
:10DA1C00CF18A0918A0BAD320895E091980BE29546
:10DA2C00EF70E0930F04E091980BEF700895E52FE1
:10DA3C00F0E00895EA0FFB1FFA93EA930895EF5E66
:10DA4C00FC4FBF01E081E058DB01EC930895E0E06E
:10DA5C00EC93AE81BF810895E3E0F0E0FA93EA9392
:10DA6C000895E52FE450F0E0FA93EA930895E55019
:10DA7C00F0E00895E091980BE295EF700895EA1BA1
:10DA8C00A2E5B7E0F0E00E94997A0895F0E0EE0F7D
:10DA9C00FF1FEA5CFD4F0895A4E3B2E0F0E0EE0F47
:10DAAC00FF1FEA0FFB1F0895FA93EA93E12FF0E0B2
:10DABC00FA93EA930895E12FF0E0FA93EA9308952C
:10DACC00E2E0F0E0FA93EA930895EAE8FBE0FA93D7
:10DADC00EA93EAE0EA930C946E46E1E0F0E0FA9304
:10DAEC00EA930895FA93EA930C9459460E94957B15
:10DAFC00FA93EA930895ABE0EA9FF001E252FA4FF1
:10DB0C000895ED85FE85FA93EA9308951A930A9386
:10DB1C003CCF1A930A93E0E0EA930E94BA4BDDCF14
:10DB2C00E1E0E0933C0C0E941768E0933D0CF0930D
:10DB3C003E0C0895BD01AAE0B0E00E94BA7AE60F4F
:10DB4C00F71F0895FA93EA93EAE0EA930C946E4671
:10DB5C00E1E0E0930E045DCE0E94A4460C9487464F
:10DB6C00E0E2EA930C944246A3E2B7E0E881F0E0ED
:10DB7C00EE0FFF1FAE0FBF1F0E94867B0895FA9316
:10DB8C00EA930C945A41E881F0E00895EE0FFF1FE0
:10DB9C00AE0FBF1F08950E94867B0E94A47A089541
:10DBAC000E94997B0C943B41FA93EA930C94A44603
:10DBBC00A9E0B0E00E94B47B0895A7E11A9FF001A0
:10DBCC00EF5CF94FE0810895E12FEF5FEA930C943D
:10DBDC007041F0E0D4CFE8E0F0E05CCEEA93E6E010
:10DBEC00EA930E94264184CEE0916D05F0916E057A
:10DBFC000895E0916905F0916A050895AE0FBF1F75
:10DC0C00E3E0F0E00E940D7B0895FA93EA931A93F7
:10DC1C000A930C94C912FA93EA933A932A930C94AC
:10DC2C00C912A0917105B09172050895A091730568
:10DC3C00B091740508950E94A97BEA1BFB0B0E940E
:10DC4C00A47A0895E887F9876A877B870895A88561
:10DC5C00B9858A859B85EFEEF0E060E070E0089571
:10DC6C000E94B07BDF01F001EA1BFB0B08950E94C0
:10DC7C00A47A0E94377B0895EC83FD836E837F83A7
:10DC8C000895FA93EA930C94BF46FA93EA930C9492
:10DC9C00677AA9E01A9FF001E058FC4F0895379677
:10DCAC000E94957BDF010E94867B0895E2E3F0E001
:10DCBC00FA93EA9308950A921A92FA926A937A93D3
:10DCCC008A939A93AA93BA93EA93FA93EFB7EA9347
:10DCDC001A930895ED91FD913196FE93EE9308956C
:10DCEC00ADE01A9FF001EB5FFC4FE08108951A93B1
:10DCFC00E1E0EA930C942D47ADE01A9FF001DF01AF
:10DD0C00EB5FFC4FE081E0300895E2E0EA930C9485
:10DD1C002D47FA93EA93E4E6F0E0FA93EA930E9433
:10DD2C002368E0300895E1E0E0930D04E0930E04E5
:10DD3C000895E0912908F0912A0860912B087091C0
:10DD4C002C080895E0912108E150A3EAB6E0F0E038
:10DD5C000E94997AAE0FBF1F0E948A7B0895E12F13
:10DD6C00EF5FF0E021CFE0912208EA93E0911E08EA
:10DD7C00EA930E94E51AA0911E0CB0911F0C10970B
:10DD8C000895A091200CB091210C8091220C9091BF
:10DD9C00230C0E94627D0895E0911E0CF0911F0CE3
:10DDAC000895E091200CF091210C6091220C70915F
:10DDBC00230C0895E2E3F0E068CF1A93E0EAEA93CB
:10DDCC00EA81F0E0E054F14FFA93EA930E94B066D6
:10DDDC001E2F0895E0EAEA93EA81F0E0E054F14F57
:10DDEC00FA93EA931A930C94DC66EA930E946066A9
:10DDFC00E0300895E0EAEA93EEE5F0E0FA93EA9376
:10DE0C00E0E0FFE0FA93EA93EEEBFBE00895FA937F
:10DE1C00EA93E0E2EA930C946567E0EAEA93E9811D
:10DE2C00FA81E050FE4EFA93EA930895EA81F0E00D
:10DE3C00A8E2B0E00E94E27A0895E0EAEA9340CECC
:10DE4C00FA93EA930C94FD66FA93EA930C94B066F9
:10DE5C00E0EAEA93E8E2F0E0FA93EA931A930A9381
:10DE6C00EAE8FBE00895EAE8FBE0FA93EA93089508
:10DE7C00EDE2EA93EAE0F0E0FA93EA930E94A368F9
:10DE8C00E0E00895EA81F0E0ABE0B0E00E94E27AD5
:10DE9C00E050F24F8F01AA81AA300895E0EAEA938C
:10DEAC00EBE0F0E0FA93EA931A930A93E2EBFBE0CF
:10DEBC000895E3EBFBE0FA93EA930895EA81F0E02E
:10DECC00EE0FFF1FE050F04F8F01AA81A03808958C
:10DEDC00E150F0E00895EA81F0E00E94997AE05870
:10DEEC00F14F8F01AA81A5300895EFE2FCE0FA937F
:10DEFC00EA93E0E0EA9301CDECE1FCE0FA93EA93DB
:10DF0C00E0E0EA93F5CC0E94997A0E94957ADF01C1
:10DF1C00EA85F0E0AE0FBF1FE8E0F0E00E94E27A85
:10DF2C00E050FA4E8F01E0EAEA93E2CC1A930A939E
:10DF3C00ECE1FCE085CFAE81BF81888599850E949C
:10DF4C00777AEE83FF8368877987089540931E0C58
:10DF5C0050931F0CEE81FF8168857985E093200C2E
:10DF6C00F093210C6093220C7093230C0895F0E035
:10DF7C00AE0FBF1F0895EA930E94CF180C949F1FF9
:10DF8C00E091950BF091960B0895FA93EA930C940B
:10DF9C006E18ED81EA93ED81EA930895E091AC0B54
:10DFAC00F091AD0B0E94A47A0895F0E0A4E6B0E0E5
:10DFBC000E94E27A0895EC81F0E0EA0FFB1F0895CD
:10DFCC00E0912708F09128080895E093270CF0932E
:10DFDC00280C0C94361CE3EAF6E0FA93EA93E0E0A2
:10DFEC00EA930895FA93EA930C94A368E0E0F0E0C6
:10DFFC0060E070E00895E0932908F0932A0860939C
:10E00C002B0870932C080895E091970BA3EAB6E0C7
:10E01C00F0E00E94997A0895AE0FBF1F0E948A7B90
:10E02C000895ED5EF94FE081E1300895FA93EA939B
:10E03C00E0912208E05DEA930895EA930E94DD6383
:10E04C00E1300895ECE3F8E0E093600BF093610BA2
:10E05C000895E12FA3EAB6E0F0E00E94997A0895C2
:10E06C000E949368A881AF5FEAE00E94EC7AE05DC1
:10E07C000895A881AF5FEAE00E943C7BE05D0895C3
:10E08C00FA93EA93E0E0EA930895AAE0B0E00E94E4
:10E09C00B47B0895E12FF0E00E94977AE854FF4F8B
:10E0AC0032960E94957B0895E12FF0E00E94977ABA
:10E0BC00E854FF4F08953696E491D901EC930895F6
:10E0CC00E0EAEA93E5E0F0E0FA93EA930895EA9344
:10E0DC000E94271CFA93EA93E4E2FCE00895FA9379
:10E0EC00EA93EFEFEA93E5E0F0E07CCFE093250CC8
:10E0FC00F093260C08950E94A97BEA1BFB0B089554
:10E10C00A0912A0CB0912B0C0895E0E0E093380C10
:10E11C00E093390C0895A0912C0CB0912D0C08951E
:10E12C00E0912C0CF0912D0CAC81BD81EA0FFB1F02
:10E13C000895E0932C0CF0932D0C08951A930E94E3
:10E14C00C11C1E2F0895E0932A0CF0932B0C0895FC
:10E15C00FA93EA930E942368E0300895ABE01A9F8B
:10E16C00F001E452FA4F08951A930E94AD1ED3CFDA
:10E17C00E0912A0CF0912B0C0895EA930E94AD1EAD
:10E18C000E944A1EE0300895EB81EA930E94E81C3D
:10E19C00FA93EA93E9E2FCE00895E0E0E0934D0C99
:10E1AC00E0934C0C08951A930A93E0911208ABE09B
:10E1BC00EA9FF001E752F84F8F01D80111960895AC
:10E1CC00E0E0F0E0ED93FC930895EA81D801EC9344
:10E1DC00E2E1F8E0FA93EA930E949A3319810881FC
:10E1EC000895E12FACE8B0E0F0E0EE0FFF1FEA0F6E
:10E1FC00FB1F0E94957B0895E150ADE0EA9FF00172
:10E20C000895ACE8B0E0F0E0EE0FFF1FEA0FFB1F43
:10E21C000E94957B0895A0911608B0911708EA2BDF
:10E22C00FB2BE0931608F09317080895E150A7E133
:10E23C00EA9FF0010895A7E10A9FF001E15DF94F13
:10E24C00AF010895ED55F94FE081E0300895E98173
:10E25C00FA81FA93EA930895E12FF0E00895E2E051
:10E26C00F0E00E940D7B0895AAE9BBE0E0911A084A
:10E27C000895ADE9BBE0E0911A0879CEA0EABBE0C5
:10E28C00E0911A0874CEA3E2B7E0D1CBEE0FFF1FDA
:10E29C00EA0FFB1F0895E081F0E00895A7E11A9FB3
:10E2AC00F001E15DF94FEE83FF83AE81BF810895EC
:10E2BC00EE81FF81A481AA930C94F51F0D901C9004
:10E2CC00AE81BF811296EC91F0E0E00DF11DDB0107
:10E2DC00ED93FC930895ED91FD913197FE93EE93A0
:10E2EC0008950E949A21EF770E2EAA85BB8512966F
:10E2FC00EC91E0150895A3E20A9FF001E855F94F5F
:10E30C000895E0911208ABE0EA9FF001E752F84F54
:10E31C00EC87FD87AC85BD85119608951296EC911E
:10E32C00AC85BD851696EC930895D001F0E0089568
:10E33C00A885B98518960E94867B0895AC85BD8505
:10E34C00EC93E2E1F8E0FA93EA930C949A33E885C3
:10E35C00F985A281AA930895AA85BB85EC91EA93CD
:10E36C00E3E0EA930C94F342AA85BB85E0E0EC93DE
:10E37C00E2E0E09324060895BF0100801180AE8195
:10E38C00BF811296EC910895DB01ED93FC93AE8165
:10E39C00BF8112965CCBE4E6F0E00E94E27A08952D
:10E3AC00F0E0ED93FC930895E2E1F8E0FA93EA9340
:10E3BC000C949A33E0911908A0911808EA17089563
:10E3CC00F0E0E00DF11D0895A3EABBE045CFADE907
:10E3DC00BBE0EE27A10FBE1FEC910895A0EABBE0B5
:10E3EC00EE27A10FBE1FEC910895BD01AAE0B0E08D
:10E3FC000E94BA7ADB010895E081EA930C94505E96
:10E40C00E0E4FAE0E0935E0BF0935F0B0895EA937F
:10E41C000E94A562E0E00895EA930E94A5620C9424
:10E42C001B64ADE9BBE0EE27A00FBE1FEC91089575
:10E43C00A0EABBE0EE27A00FBE1FEC910895AAE95D
:10E44C00BBE0EE27A00FBE1FEC91E1700895A3EA8C
:10E45C00BBE062CAA0EBBBE0EE27A00FBE1FEC91A5
:10E46C000895A9EABBE0EE27A00FBE1FEC9108951A
:10E47C00EA81ADE0EA9FF001E15FFC4FA0E0A083F0
:10E48C00EA81EA930895ADE0EA9FF001EB5FFC4F5F
:10E49C000895ABE00A9FF001E452FA4F0895ABE007
:10E4AC000A9FF001EE51FA4F0895FA93EA930C94F7
:10E4BC002735FA93EA930E9468433A9326CCE0916D
:10E4CC002C0CF0912D0C30970895AFEFBFEFA0837B
:10E4DC00B18308950E941768E093520CF093530C8B
:10E4EC000895FA93EA93E0E0F0E80895E0911208B9
:10E4FC00ABE0EA9FF001E752F84FFA93EA930E94DF
:10E50C00FC2852CFE0911008ABE0EA9FF00108958F
:10E51C00E0E1F8E0FA93EA930C949A33FA93EA93D5
:10E52C000C942E53E88DABE0EA9FF0010895FA931A
:10E53C00EA93F2C9E0E1EA93E0912506EA930E949E
:10E54C00A2181E2F08953CDDFA93EA930895FA93CE
:10E55C00EA930C94781EE0932506E0E0E0934F0CD0
:10E56C00E1E3E093500C0E943B2A0C941626FA939C
:10E57C00EA930C94B662E1E4F9E0E093600BF0935B
:10E58C00610BE3E0EA930C944B62A091600BB091A9
:10E59C00610B08950E941768E093470CF093480CA8
:10E5AC000895E093600BF093610B0895E3E0EA9318
:10E5BC000C944B62E0932708F093280808950E946E
:10E5CC00CB46E0E0EA930C949F0EE0E0F0E0E093A1
:10E5DC002508F0932608E2E0E0930E040895E091FC
:10E5EC00130445CAE0912508F0912608C8CAE091A9
:10E5FC005D05F0915E0531970895FA93EA930C94BA
:10E60C009D45EF5CEA930C944246A3EEB6E09CC9A0
:10E61C00A3EABBE0E0911A08F0E038CE0E94867BBA
:10E62C00D001ED93FC9320CEF0E0EA0FFB1F0F011D
:10E63C001BCEA3E2B7E088C9E7E0E0931808EA93A1
:10E64C00E0E0EA93E6C8EA930E94CF400E940643BA
:10E65C001E2F0895EAE2EA93E5E7F7E111CD0E9457
:10E66C00E72BE1E0EA930C94CF2B1F771A930C94D1
:10E67C00CF18A0912508B09126080895E8EEF3E094
:10E68C000E943F7B0895E053F0E00895A0E024FC45
:10E69C00A1E0A0300895E0E0EA93BBC8E091330814
:10E6AC00F0913408FA93EA930895FA93EA930E944E
:10E6BC002368E13008950E941768E0933308F093C3
:10E6CC0034080895E0E0E0934C0C0895D2DFEA178B
:10E6DC00FB070895E0931808E0E0E09330080895F4
:10E6EC000E94BB630E94502DE093240808950E9461
:10E6FC00CF180C94CB46E0911908EA93E0E0EA932A
:10E70C000E94FA2C0C94AE280E9406431E2F1A93DA
:10E71C000E94832D103808951A93E091C605EA9350
:10E72C000895E091890BEA930E94DA17E03008957E
:10E73C000E941768E093540CF093550C0895D9017E
:10E74C0018960E94867B0895E4E6F0E060E070E0A5
:10E75C000E94377B08950E94CF1812CC0A93E09147
:10E76C00C605EA930895E0912F08EA930A930C9456
:10E77C00041A0E94867BFA93EA930895A0E6BBE004
:10E78C00A9CAE0913C08E053E09322080895FA935B
:10E79C00EA93E0E3EA930C94BB63E0913908EA93C3
:10E7AC000C9463630E94A47A0E94997B08950E9442
:10E7BC001F63EBE3EA930C94A562E89423F8E0E082
:10E7CC00F0E0F8DE0A93E1E0EA930C94FA2C0A9359
:10E7DC00E1E0EA930E94FA2CE1E00895E09112083E
:10E7EC00ABE0EA9FF0010895A881B981EC91EF5F4D
:10E7FC00EC930895ABE00A9FF001E352FA4F0895B1
:10E80C00A083ABE00A9FF0010895ABE00A9FF001F2
:10E81C00E152FA4F0895E5EAF7E1FA93EA93EA85B3
:10E82C00ABE0EA9FF0010895AC81BD81EE27A00F0B
:10E83C00BE1F0895E02FAC81BD81F0E008950E94C9
:10E84C00997B84E00E94056B28960895EE27A30F10
:10E85C00BE1FEC91D001EC930895A2E5B7E074C80B
:10E86C000E94997AEA0FFB1FAF010895E0912C0CDE
:10E87C00F0912D0C0895E32FA0911E08EA0F089536
:10E88C00ADE02A9FF001E35FFC4F0895A8E0B0E0F3
:10E89C000E94B47B0895F0E0FA93EA9308950E94E5
:10E8AC0077420C944642F0E00E94997A08950E94B7
:10E8BC00997B0E9461420C9446420E947742E9EC9B
:10E8CC00F7E1DECB0E9446420C94464220E030E059
:10E8DC00E12FE05DEA93ECECF7E1A8CBEAE0EA93F8
:10E8EC000C948562E4E4FBE0FA93EA9308951091AA
:10E8FC005D0500915F0508950E9406433E2F0C9420
:10E90C00EB45EAE0F0E00E94E27A0895DF01EE27A1
:10E91C00A30FBE1F0895FA93EA931EC9EF81F885E1
:10E92C00FA93EA930895F0E0EA0FFB1F0895E02FA5
:10E93C00A0E0B2E0B8CFEA0FFB1F3296E491089545
:10E94C00FA93EA93E0911B0CEA930E946E38E13241
:10E95C000895EA930E941438E1320895E6E0F0E05D
:10E96C000C94506C0E94A446AAE9BBE0EE27A10FC0
:10E97C00BE1FEC91E1700895EE0FFF1F0C94206DFB
:10E98C00EA930E946E38E13208950E94B50D0C9402
:10E99C000F6CEAE3EA930C9442460E94997B0C9428
:10E9AC004F41E3E7EA930C944246EA23EA930E9430
:10E9BC007641D6C8EA930E947641D2C8DF013296DE
:10E9CC0095C80E94977AE854FF4F0895EAE4F6E060
:10E9DC00E0933A0CF0933B0C08950E94691AE0E026
:10E9EC00E09321080E94C9150E94B50DE1E0E09367
:10E9FC001B0808950E94CB460E9455100E940643A6
:10EA0C000E2F0D330895EE81FF81FA93EA9308954A
:10EA1C00EAE2EA93E4E7F8E10895EA930E94191612
:10EA2C000C94B50DE093C105F093C2050895FE0159
:10EA3C00FA93EA930895ECE8F8E1FA93EA93EE85F9
:10EA4C00FF8568897989FBCEE0E9F8E1FA93EA93CE
:10EA5C00AE85BF858889998977CE0E94997BAA89D2
:10EA6C00BB898C899D89E4E6F0E060E070E00E944F
:10EA7C00517B0E94997B88E00E94056B2C9608952F
:10EA8C00E9E9F8E1FA93EA93EE85FF858BCE84E011
:10EA9C000E94056B2896CBCFFA93EA93EE85FF85FF
:10EAAC0008950E947E630C94176884E00E94056BA5
:10EABC0028960895EE27A10FBE1FEC910895EA93B6
:10EACC000E94E1411F5F0895E091C405A7ECB5E0F9
:10EADC00F0E00895AF5FEAE00E943C7B0895E0917E
:10EAEC00C305A7ECB5E0F0E0D1CBA0E0A083E981B1
:10EAFC00ADE0EA9FF0010895EF73A5E1EA9FF00104
:10EB0C00E051FB4F0895EF73ABE0EA9FF001EC5E30
:10EB1C00FB4F0895AC81BD81EE27A30FBE1FAC91B6
:10EB2C00A0300895ABE00A9FF001EC5EFB4F089516
:10EB3C00EA0FFB1F0F01AC81BD8188CEA5E10A9FB6
:10EB4C00F001E051FB4F0895EE81FF8101801280AE
:10EB5C00AE81BF8115960E94867BD0010895FE017F
:10EB6C003896FA93EA930895EAA5FBA5FA93EA93EB
:10EB7C000895FA93EA93FE013A96FA93EA930E9467
:10EB8C00C36830E0E02F0895E091C105F091C20513
:10EB9C000895A1ECB5E0ED91FD913296FE93EE93C4
:10EBAC000895AE81BF81EA17FB070895E0E0E0937A
:10EBBC006505E093660508951A930A933A932A9390
:10EBCC000895FA93EA93E0910E040895A09100033E
:10EBDC00B09101030895E0910003F0910103FA93C1
:10EBEC00EA93E0910203F0910303FA93EA930895F8
:10EBFC00E0930003F09301030895A981BA815ACFE1
:10EC0C001A930A9300E010E00895F801AA81BB81E1
:10EC1C00EA0FFB1FE4910895AE0FBF1FAC91A0301B
:10EC2C000895D801F0E0AE17BF070895AE0FBF1FCF
:10EC3C00EC91EA930895EFEEF0E0EA1BFB0B0895DC
:10EC4C00A0910E04E4E1EA9FF0012E2F3327C3CFED
:10EC5C00E0E0EA930E94BA4B0E94717D0895ECE0CB
:10EC6C00EA9FF001A0910D04EA9FF00108951A9318
:10EC7C00E1E0E0930E04E0930D0410E00895ED81C3
:10EC8C00FE81FA93EA930895EF81F885EA1BFB0B5A
:10EC9C0008953A932A935A934A930895EAA5FBA5AB
:10ECAC00E20FF31FFA93EA930895ECA1EA930C9404
:10ECBC001D4C3A932A93EEA1FFA1E40FF51F089582
:10ECCC00FA93EA93EBCFEAA5FBA5E40FF51FFA93B1
:10ECDC00EA93EBCFE20FF31FFA93EA930895FA93BA
:10ECEC00EA935A934A930895EA9FF001AEA1BFA10B
:10ECFC00F0E00895E2E0E0930E04E0E2F0E0EAA335
:10ED0C00FBA30895AE1BBF0BAACAEE8DF0E00895CD
:10ED1C00E20FF31F3196FA93EA93ECA1FDA1E40FF5
:10ED2C00F51F31960C94476EECA1FDA1E40FF51F75
:10ED3C000C94476EE9A1F0E0DE0116960895ED8D76
:10ED4C00EA930E94F845E9A1EF5FE9A30895ED8BE2
:10ED5C00FE8BAB89BC8983CAA98DBA8DEA0FFB1FC8
:10ED6C00E98FFA8FEB89FC89AF89B88DEA0FFB1F0D
:10ED7C00EF8BF88FED89FE89AD89BE890E94E27A0E
:10ED8C000E94A47A0E943F7CEE87FF87688B798B68
:10ED9C00EB89FC89AB89BC890E94E27A0E94A47A37
:10EDAC000E943F7CAE85BF85888999890E94157D1C
:10EDBC00EA87FB876C877D8700E010E00895F801F7
:10EDCC000E94A47A0E943F7CEE83FF836887798738
:10EDDC00AE81BF81888599850E94C77CAA85BB8539
:10EDEC008C859D850E94C77CAE85BF858889998955
:10EDFC000E94A37B0E94727C0E94087CAF015A93F4
:10EE0C004A930C942C6BE98DFA8DE21BF30BFA935D
:10EE1C00EA930895E98DFA8DE01BF10BFA93EA93CE
:10EE2C000895F901AD8DBE8D0C94206DED8DFE8D88
:10EE3C00E01BF10BFA93EA93EA8DEA930C941D4CC8
:10EE4C00AD8DBE8D0C94206DEFE3F1E0EA1BFB0B56
:10EE5C000895EB81FC81AF81B8850895E00DF11D1B
:10EE6C00FA93EA930E942F4AE5E3EA930895E0931C
:10EE7C0065000C94E06E0E94687DEE81EA930E941E
:10EE8C005E4A8F010895E985FA85AD85BE850895A2
:10EE9C000E94784AEB85FC85FA93EA930C94904A8D
:10EEAC00ED85FE85A985BA85AE17BF070895EB855C
:10EEBC00FC85AF81B885AE17BF070895AD85BE85BB
:10EECC00E985FA85EA1BFB0B0895FA93EA930C94F7
:10EEDC00C76BAB85BC85D8CEAF81B885EB85FC857F
:10EEEC00EA1BFB0B0895D9010E94E27A0F010895E9
:10EEFC00D0010E940D7BAF01FA01AD85BE850C944B
:10EF0C00206DED85FE85E21BF30BFA93EA930895D1
:10EF1C00AD85BE850C94206DA985BA85ED85FE85E1
:10EF2C00EA1BFB0B0895E881F981FA93EA930895A3
:10EF3C005A934A93EE85FF85AFCDFA93EA93EC850D
:10EF4C00FD85FA93EA930E94FE4CE0910E04AA858B
:10EF5C00BB85E9CCD901F0E0AE17BF070895E05CA2
:10EF6C00F54F4ACAE091370CA091360CEA17089578
:10EF7C00E0911108ABE0EA9FF0010895E3E0EA9319
:10EF8C000E940263F5CFE081E05DEA930C94A562E8
:10EF9C00A091250CB091260C0895E2E5EA930E940D
:10EFAC00A5620C94E94DF096EA930E946363E2E744
:10EFBC00EA930C94A562EA930E94A562EEE0EA93B0
:10EFCC000C94A562ECEAF8E1D2CA0E94D862EBE399
:10EFDC00EA930C94A562E0E3EA930C94A562EBE34C
:10EFEC00EA930C94A5625A934A930E946E180E2FC2
:10EFFC0000340895FA93EA930C949A331A93E985A2
:10F00C00FA85FA93EA930895E552F84FA885B985E5
:10F01C00A083B183E3CBE2E5EA930C94A5621A9347
:10F02C00E0913908E0531E2FEDE3F8E0BACAE09105
:10F03C001208A0911308EA170895E3E1F8E0DACF7B
:10F04C00E0911308ABE0EA9FF0010895A091740BD6
:10F05C0041CDE093740BEAE2EA930E946363DBCF49
:10F06C00E091740BE05AA7CFD9011696EC9113CC12
:10F07C00F901A281B381BA93AA9308950E94D86230
:10F08C00EAE3EA930C94A562D9011196E0E0EC93C3
:10F09C000E947E63D2CFD901EC91FDCBE05DEA9367
:10F0AC000C94A562E05DEA930E946363B4CFEB58C5
:10F0BC00F44F69CFEEE0EA930C94A562EAE3EA938D
:10F0CC000E94A562F9010895E0935E0CF0935F0C29
:10F0DC00E2E0E0933608D9011196EC930895EA9397
:10F0EC000E94636398CF0E94D862DBCCE091190C2C
:10F0FC00D9CFE091190CF0E0DACFFA93EA9365CF0F
:10F10C000E94D862ECE2EA930E94A5620CCF3DDA31
:10F11C00AC91A0330895A0915E0BB0915F0BE0E031
:10F12C00EC930895EE81FF81E093270CF093280C6B
:10F13C001093240C0E94361CE1E3089541E050E04A
:10F14C000E94D761E887F987EAE3EA930E944C6151
:10F15C00E13008951A93E985FA85C1CDE2E2EA938C
:10F16C000C944C6112DAAC91A03208950EDAAC9189
:10F17C00AB3308950ADAEC91EA930895EAE3EA9343
:10F18C000C944C610E94D7613197E887F987E88528
:10F19C0008950E94867BE40FF51FD001ED93FC933C
:10F1AC000895E091400BF0E0ED55F94F0895E0E043
:10F1BC00E093630CE093640C08950E94D76131973F
:10F1CC00E093400BE091590BA091400BEA17089586
:10F1DC000E94DD56E091400BEA930895ECE2EA932D
:10F1EC000E944C61E0300895EC5BF44F0F01CDD9D7
:10F1FC00EC91D001EC931F5FC1CAEC5BF44FA0E023
:10F20C00A0830895EA930E944C61E1300895E09147
:10F21C00410B89CBE091410BEF5FE093410B0895DB
:10F22C00A3EABBE0E091410BF0E00C944C71AAE92D
:10F23C00BBE0E091410B0C94BD6FE091410BF0E011
:10F24C000895FA93EA930C945E53E091400BF0E02E
:10F25C00B8CBFA93EA930C94D8620E94D862ECE291
:10F26C00EA930C94A562ECE2EA930C94A5620E94DA
:10F27C005353E0E0E093410B0895E091410B0C9463
:10F28C00BD6FE091600BF091610B0895AEE5BBE0B2
:10F29C000C94706EA0915E0BB0915F0BEC93F6CF5B
:10F2AC00A0915E0BB0915F0B13970895E0E0EA9389
:10F2BC000E94B753E09335080895AA81BB81EC9165
:10F2CC00E295E07FAE2FEC810895EA0FAA81BB8115
:10F2DC00EC938ACAE091040DA091030DEA170895EE
:10F2EC00E0913B09F0E0E05CF64F08951083E0916B
:10F2FC003B09EF5FE0933B09E12FA0913D09089595
:10F30C00E0933D09E0913C09E150E0933C09E03089
:10F31C000895E05CF64FA0E0A0830895E091CF0D36
:10F32C00F091D00D0895A091CD0DB091CE0DEA17AE
:10F33C00FB070895E12FA091D40DEA0FE093D40DB3
:10F34C00E091D60D0895F0E0E85CF74F1083089536
:10F35C00E091DB0EF0E0E652F24FE081E0939C008E
:10F36C00E091DB0EEF5FE093DB0E08950ED9AC91CC
:10F37C00AA3308950F0109D9EC91E0530C94E6716E
:10F38C00EA930E94A5621F5F0895EAE5F9E1FA93FA
:10F39C00EA930895FE013196FA93EA930895E88171
:10F3AC00EA930C94A562E881F9816A817B810E94C1
:10F3BC00997B0895E05CF54FE081E0300895EA9385
:10F3CC000E940668EA930C94505EEA930E94D464FF
:10F3DC00EAE5E0933E090895EA930E949566E030D1
:10F3EC000895E0917100E87F1E2F0895E09373005B
:10F3FC00E4E8F2CF0A930E946C66E0300895FF2790
:10F40C00662777270E943F7C0895EE8DAE85BF85D9
:10F41C0088899989F4DF0E94C77CA9A1BAA18827A1
:10F42C0099270E94A07B0E94A37B0E94727C089566
:10F43C000E94A37B0E94727C0895FA93EA93E2E106
:10F44C00F0E0FA93EA9308952A93ED89FE89FA93F2
:10F45C00EA93FE017596FA93EA930C941C69EE8973
:10F46C00FF893497EE8BFF8B0895ED89FE89FA9313
:10F47C00EA93FE017596FA93EA930C941C69AE8993
:10F48C00BF8914960E94867BEE83FF83BCCAE885F5
:10F49C00F9856A857B85AC85BD858E859F850895AC
:10F4AC000E94436BE883F9836A837B830895E88128
:10F4BC00F9816A817B810895EA81FB816C817D8170
:10F4CC000895E991F991309639F080EA9FE001971F
:10F4DC00F1F7A8953197C9F708950024AF0DB01D29
:10F4EC000895EA0FFB1F681F791F0895EA1BFB0B99
:10F4FC00680B790B0895F195E195F0400895F0951E
:10F50C0060957095E195FF4F6F4F7F4F0895EE23F7
:10F51C000E2EEA2F19F0EE0F0A94E9F70895EE0F6C
:10F52C00FF1FEE0FFF1FEE0FFF1FEE0FFF1F0895C3
:10F53C00FE2FFF0FFF0B6F2F7F2F08956F2F660F7E
:10F54C00660B762F0895BA2FBB0FBB0B8B2F9B2FFF
:10F55C0008958B2F880F880B982F0895EA17FB07B7
:10F56C00E1E00CF0EE270895FA9FF02DEB9FF00DE3
:10F57C00EA9FE02DF10D08957A9F702D6B9F700D11
:10F58C00F89F700DE99F700D6A9F602D710DFB9FA8
:10F59C00600D711DE89F600D711D8827FA9FF02D7D
:10F5AC00610D781FEB9FF00D611D781FEA9FE02D18
:10F5BC00F10D681F781F089582D0D6DF0EF49BDF03
:10F5CC0008958BD0D9DF0EF49ADF0895002498E0CB
:10F5DC00AA0F001C0E1A10F40E0E01C0A1609A9511
:10F5EC00B9F7EA2FA02D08950024112490E1AA0F59
:10F5FC00BB1F001C111C0E1A1F0A18F40E0E1F1E26
:10F60C0001C0A1609A9599F7FD01D001089557D0DA
:10F61C00EBDF0EF470DF08953F934F935F9300245C
:10F62C0011244427552730E2AA0FBB1F881F991FAE
:10F63C00001C111C441F551F0E1A1F0A460B570B9A
:10F64C0028F40E0E1F1E461F571F01C0A1603A95CD
:10F65C0059F7FD01BC01D001CA015F914F913F9157
:10F66C0008953BD0D9DF0EF44ADF0895AFDFEA2FBF
:10F67C000895E894B7FF04C0A095B09511966894CE
:10F68C00F7FD39DFB1DFFD010EF435DF0895C4DF7E
:10F69C00FD01BC010895E89497FF09C0A095B095B1
:10F6AC0080959095AF5FBF4F8F4F9F4F689477FDBC
:10F6BC0026DFB2DFFD01BC010EF421DF0895E894D2
:10F6CC00F7FF02C018DF6894B7FF06C0A095B0958D
:10F6DC00119600F8039400FA0895E89477FF02C09D
:10F6EC000EDF689497FF0BC00024A095B095809511
:10F6FC0090951196801D901D00F8039400FA0895C2
:10F70C00ED91FC9111970895ED91FD916D917C9186
:10F71C0013970895ED93FD936D937C930895059045
:10F72C00F491E02D08957A936A93FA93EA930895ED
:10F73C00689401C0E89401D09DD0182E862F612DBD
:10F74C00192E972F712D1B2EBF2FF12D1A2EAE2F88
:10F75C00E12D0895119602D0FE2F1197E199FECF5D
:10F76C00FF93FFB7F894AEBBBFBBE09AEDB3FFBFFE
:10F77C00FF91089507D01196EF93EF2F03D0EF91DF
:10F78C0011970895E19B02C0A895FCCF9FB7F89400
:10F79C00AEBBBFBBE09A8DB3E81719F0EDBBE29A94
:10F7AC00E19A9FBF0895552342F4503811F4E0FFBD
:10F7BC0004C03196691F791F6BF050E8572711F47C
:10F7CC005F93CDC05F3F31F0660F000C5795679586
:10F7DC00752F08955F9300200AF0CDC0C6C050E885
:10F7EC00192E1522880F991F9527550F879550E8CC
:10F7FC00072E0522660F771F7527550F67950895FD
:10F80C00689401C0E8945F93F2DF703818F07F3F82
:10F81C0008F4A5C056E1571BAAF4519558300EF4C4
:10F82C00593030F0EFEFFFEF6FEF7FE777F91AC049
:10F83C0077275523B9F0EE0FFF1F661F771F5A95D8
:10F84C00D1F710C07727583028F0EF2FF62F672FFD
:10F85C005850F9CF552331F076956795F795E79584
:10F86C005A95D1F700200AF44ADE5F910895689406
:10F87C0001C0E894309760407040B1F0002426F04D
:10F88C00772312F400943BDE172E7EE1112032F028
:10F89C007A95EE0FFF1F661F111CF9CFEF2FF62F75
:10F8AC00612D5F938ADF5F9108954F93AF01FD0146
:10F8BC00DA01AB01BC01CA01402D012C142E4F9171
:10F8CC000895EA0FFB1F681F0895E095F095609569
:10F8DC00EF5FFF4F6F4F08955F9381DF903871F1A9
:10F8EC0050E8152604C05F937ADF903839F17038F0
:10F8FC0021F1572F591B13F112F4D7DFFACF5831DE
:10F90C0018F0AA27BB278827583028F0AB2FB82F20
:10F91C0088275850F9CF552329F08695B795A79588
:10F92C005A95D9F7502D512562F0CBDF38F46795F5
:10F93C00F795E795739513F41EC0B7DF3EDF5F9123
:10F94C000895EA1BFB0B680B51F010F40094BDDF1B
:10F95C006623A2F3EE0FFF1F661F7A95CBF7EE27F7
:10F96C00FF27662777275F910895EFEFFFEF6FE78B
:10F97C007FEF5F910895EFEFFFEF6FE77FE75F9108
:10F98C0008955F932CDF703851F3903841F30124C4
:10F99C000894791F23F41CF300203AF3ECCF0F9258
:10F9AC001F932F933F934F93112722279927689FDB
:10F9BC00A0018F9F302D410D591F6B9F300D411DA4
:10F9CC00591F8E9F27D0BF9F25D06A9F23D0BE9FE3
:10F9DC001DD0AF9F1BD0AE9F110D291F391F491F82
:10F9EC00591FE32FF42F652F522F4F913F912F91D9
:10F9FC001F910F9066232AF0550FEE1FFF1F661FF5
:10FA0C0002C073954BF2CFDE5F910895100D211D4E
:10FA1C00391F02C0200D311D491F591F08955F93D6
:10FA2C00DEDE703821F411200AF49FCFA4CF903879
:10FA3C0009F495CF01240894970B1BF4D4F3002000
:10FA4C00F3CF792F1F932F933F934F9311241127AB
:10FA5C00222733274427552790E2AE17BF07860786
:10FA6C00410730F0AE1BBF0B860B410B089401C055
:10FA7C008894551F221F331F111CAA1FBB1F881FE0
:10FA8C00441F9A9551F7F901612D4F913F912F9198
:10FA9C001F91662332F0550FEE1FFF1F661F7A95DC
:10FAAC0043F281DE5F910895309760407040089575
:10FABC0000240A160B06089500240A160B060806E5
:10FACC00090608955A934A933A932A931A930A93E0
:10FADC0008955D814C813B812A81198108810895AB
:00000001FF
